:100000000C94F50E0C94F2890C94C7890C949C897D
:100010000C9471890C9446890C941B890C94F0887B
:100020000C94C5880C94260F0C94260F0C94260F64
:100030000C94260F0C94CB6C0C94260F0C94260F6A
:100040000C94260F0C94EC720C94260F0C94260F33
:100050000C94260F0C94260F0C94CB630C94888B75
:100060000C94260F0C94D48F0C94A98C0C94260F0E
:100070000C94260F0C94260F0C94260F0C94260F2C
:100080000C94260F0C94260F0C94260F0C94260F1C
:100090000C94260F0C94260F0C94260F0C94260F0C
:1000A0000C94260F0C94260F0C94260F0C94260FFC
:1000B0000C94260F0C94260F0C94260F0C94260FEC
:1000C0000C94260F0C94260F0C94260F0C94260FDC
:1000D0000C94260F0C94260F0C94260F0C94260FCC
:1000E0000C94260F7B857E856D8571857785B5851A
:1000F000828586858C85908594859A859E85A28546
:10010000B585A885AC85B0859A8A9F8AA48AAE8A6F
:10011000B88A318BC28ACA8AD28ADC8AE68AF08A95
:10012000FF8A098B318B138B1D8B278B0A901090C4
:1001300021902C9034904990389049903C90409078
:100140004990469052945294599459945994609479
:10015000609460946D94679467946794084AD73B61
:100160003BCE016E84BCBFFDC12F3D6C74319ABD86
:1001700056833DDA3D00C77F11BED9E4BB4C3E91AA
:100180006BAAAABE000000803F05A84CCDB2D44E99
:10019000B93836A9020C50B9918688083CA6AAAA9B
:1001A0002ABE000000803F004E414E494E4954593E
:1001B000494E46CDCCCC3D0AD7233C17B7D1387732
:1001C000CC2B329595E6241FB14F0A000020410048
:1001D00000C84200401C4620BCBE4CCA1B0E5AAE92
:1001E000C59D7420746F6F206C6F6E672065787486
:1001F000727573696F6E2070726576656E74656472
:100200000A0020636F6C6420657874727573696F7F
:100210006E2070726576656E7465640A0047322FD1
:1002200047332062616420706172616D657465722C
:10023000730A00205A3A200020593A20004265648F
:1002400020583A20002569730025696D20256973BF
:10025000002569682025696D20256973002569647A
:10026000202569682025696D202569730025697935
:1002700020256964202569682025696D202569731A
:10028000005072696E742074696D653A2000000137
:1002900025301D0C1E24311C0B18232F1B0A17FFA1
:1002A000FF040806FF06222B1A4142043803FF36DA
:1002B00028294527444350726F7465637465642030
:1002C00050696E0A006F6B0020573A0020573A00C1
:1002D0004361703A454D455247454E43595F504141
:1002E000525345523A310A004361703A43415345F3
:1002F0005F4C494748545F4252494748544E455322
:10030000533A300A004361703A544F47474C455FB7
:100310004C49474854533A300A004361703A534FAE
:100320004654574152455F504F5745523A300A00A4
:100330004361703A4C4556454C494E475F444154E1
:10034000413A310A004361703A5A5F50524F424578
:100350003A310A004361703A4155544F4C45564575
:100360004C3A310A004361703A5052494E545F4A48
:100370004F423A310A004361703A50524F4752455A
:1003800053533A300A004361703A4155544F524535
:10039000504F52545F54454D503A310A00436170FA
:1003A0003A454550524F4D3A310A004649524D5751
:1003B0004152455F4E414D453A4D61726C696E2028
:1003C000204649524D574152455F56455253494F79
:1003D0004E3A312E312E352E373120455854525554
:1003E0004445525F545950453A466C657879737468
:1003F000727564657220534F555243455F434F44B5
:10040000455F55524C3A68747470733A2F2F636F7E
:1004100064652E616C6570686F626A656374732EC3
:10042000636F6D2F646966667573696F6E2F4D41DA
:10043000524C494E2050524F544F434F4C5F5645FB
:100440005253494F4E3A312E30204D414348494E88
:10045000455F545950453A4C756C7A426F74204D43
:10046000696E692045585452554445525F434F5573
:100470004E543A3120555549443A333531343837A2
:1004800062362D636139612D346331612D38373621
:10049000352D6436363862316461363538350A00B8
:1004A0002F2F20007A5F6D61783A20007A5F6D69A6
:1004B0006E3A2000795F6D61783A2000795F6D694E
:1004C0006E3A2000785F6D61783A2000785F6D6940
:1004D0006E3A20005265706F7274696E6720656EA7
:1004E0006473746F70207374617475730A00206490
:1004F0003A0020693A0020703A0020643A002069EE
:100500003A0020703A0043290A0061626C65642059
:10051000286D696E2074656D702000436F6C6420D7
:1005200065787472756465732061726520004B6430
:10053000200023646566696E652020444546415568
:100540004C545F004B69200023646566696E65202A
:100550002044454641554C545F004B7020002364B5
:100560006566696E65202044454641554C545F00E0
:10057000504944204175746F74756E652066696ECC
:100580006973686564212050757420746865206CF7
:10059000617374204B702C204B6920616E64204B7A
:1005A0006420636F6E7374616E74732066726F6D16
:1005B0002062656C6F7720696E746F20436F6E6682
:1005C000696775726174696F6E2E680A00504944DC
:1005D000204175746F74756E65206661696C656421
:1005E000212074696D656F75740A0050494420417B
:1005F00075746F74756E65206661696C6564212021
:1006000054656D706572617475726520746F6F20CA
:10061000686967680A00204B643A2000204B693AF9
:100620002000204B703A20000A20436C61737369EC
:100630006320504944200A002054753A2000204B82
:10064000753A2000206D61783A2000206D696E3A7D
:10065000200020643A200020626961733A20004241
:100660006564204C6576656C696E6720004661693B
:100670006C656420746F20656E61626C65204265F4
:1006800064204C6576656C696E670A00426564207B
:100690004C6576656C20436F7272656374696F6E2A
:1006A000204D61747269783A00546F6F20666172F0
:1006B0002066726F6D207265666572656E63652077
:1006C000706F696E740A003A20007A5F6D696E3A45
:1006D00020202D32207A5F6D61783A202035005A33
:1006E000204F6666736574200041637469766520E7
:1006F00045787472756465723A2000556E6B6E6F42
:10070000776E20636F6D6D616E643A202200434FF7
:100710004D4D554E49434154494F4E004452595254
:10072000554E004552524F525300494E464F0045D8
:1007300043484F00202F002042403A0020403A001A
:100740002F072A0723071C070E076F66660044451C
:100750004255473A00205A3A0020593A0020436F48
:10076000756E7420583A0020453A00205A3A00200D
:10077000593A00583A0053657474696E6720547290
:100780006176656C20416363656C65726174696F45
:100790006E3A200053657474696E672052657472F6
:1007A00061637420416363656C65726174696F6E27
:1007B0003A200053657474696E67205072696E74D4
:1007C00020416363656C65726174696F6E3A2000E5
:1007D00053657474696E67205072696E7420616E1F
:1007E000642054726176656C20416363656C657248
:1007F0006174696F6E3A2000205A00205900580039
:1008000020204D61783A2000205A002059005800DD
:1008100020204D696E3A20004F6E20004F66660022
:10082000536F667420656E6473746F70733A200042
:100830004E6F2063617365206C696768740A0020DD
:1008400020506C616E6E65724275666665724279A3
:100850007465733A20002046726565204D656D6FA2
:1008600072793A2000436F6D70696C65643A204A72
:10087000616E20323220323031380A00207C204133
:100880007574686F723A2028416C657068204F62F9
:100890006A6563747320496E632E2C204C756C7AE4
:1008A000426F7420476974205265706F7369746F6A
:1008B0007279290A004A616E203232203230313892
:1008C00030393A31333A343600204C617374205554
:1008D0007064617465643A2000312E312E350A004F
:1008E0004D61726C696E0020536F6674776172653A
:1008F0002052657365740A00205761746368646FE1
:10090000672052657365740A002042726F776E200B
:100910006F75742052657365740A0020457874659C
:10092000726E616C2052657365740A00506F776552
:100930007255700A0073746172740A00205A3A008A
:1009400020593A0020583A00656E6473746F7073D2
:10095000206869743A200050726F62696E67206681
:1009600061696C65640050524F4245204641494CD4
:1009700020434C45414E204E4F5A5A4C450A005296
:1009800065776970696E670A0050726F62696E6799
:10099000206661696C65640050524F4245204641B3
:1009A000494C20434C45414E204E4F5A5A4C450A23
:1009B000005265776970696E670A0050726F6269EC
:1009C0006E67206661696C65640A004572726F72B9
:1009D0003A00205A3A200020593A2000426564200B
:1009E000583A200020746F6F206C6F6E6720657816
:1009F00074727573696F6E2070726576656E74655A
:100A0000640A0020636F6C64206578747275736982
:100A10006F6E2070726576656E7465640A00204999
:100A20006E76616C69642065787472756465722095
:100A300000000040C00000E0C0000000C000002234
:100A40004300003E4300001F4320706F73697469C8
:100A50006F6E206F7574206F662072616E67652EF1
:100A60000A003F50726F626520000A0A42656420E6
:100A70004C6576656C20436F7272656374696F6E46
:100A8000204D61747269783A00202B000A436F721E
:100A900072656374656420426564204865696768AF
:100AA000742076732E2042656420546F706F6C6FD3
:100AB00067793A0A00202B000A426564204865697C
:100AC00067687420546F706F6772617068793A0A52
:100AD0002020202B2D2D2D204241434B202D2D2B2E
:100AE0000A2020207C2020202020202020202020C0
:100AF0007C0A204C207C20202020282B292020200C
:100B0000207C20520A2045207C20202020202020EC
:100B1000202020207C20490A2046207C20282D29C6
:100B2000204E20282B29207C20470A2054207C207E
:100B3000202020202020202020207C20480A202047
:100B4000207C20202020282D29202020207C20549B
:100B50000A2020207C20202020202020202020204F
:100B60007C0A2020204F2D2D2046524F4E54202D00
:100B70002D2B0A2028302C30290A004D65616E206B
:100B80006F662073616D706C656420706F696E7440
:100B9000733A200020643A200020623A2000457118
:100BA0006E20636F656666696369656E74733A206B
:100BB000613A200052756E6E696E6720696E20443E
:100BC00052592D52554E206D6F64650A00473239D7
:100BD000204175746F20426564204C6576656C69B0
:100BE0006E670A0028422961636B00284629726FEC
:100BF0006E74002852296967687400284C2965665C
:100C000074003F4E756D626572206F662070726F62
:100C1000626520706F696E747320697320696D70EE
:100C20006C61757369626C65202832206D696E692C
:100C30006D756D292E0A003F2856296572626F7303
:100C400065206C6576656C20697320696D706C61D8
:100C5000757369626C652028302D34292E0A0010C6
:100C600000C90210012C014001220170011801B0DD
:100C7000010E01F00104015002FA00B002F0003050
:100C800003E600D003DC009004D2007005C800A089
:100C900006BE000008B400B009AA00D00BA0006096
:100CA0000E960060118C000015820020197800C09B
:100CB0001D6E00A0226400B0275A00902C50000046
:100CC000314600E0343C0010383200903A28006091
:100CD0003C1E00A03D1400803E0A00203F0000455D
:100CE000303A20005A3A2000593A2000583A200061
:100CF0004D53312C4D53322050696E730A0062659A
:100D0000640A002C2073797374656D2073746F709E
:100D100070656421204865617465725F49443A20BA
:100D20000048656174696E67206661696C6564205E
:100D30004245440048656174696E67206661696C6C
:100D400065640048656174696E67206661696C65F9
:100D5000640048656174696E67206661696C6564EA
:100D6000204530001000AD0330016A0150022B0114
:100D700070030A019004F500B005E500D006D80024
:100D8000F007CE001009C500300ABE00500BB700B6
:100D9000700CB100900DAB00B00EA600D00FA200F9
:100DA000F0109D001012990030139500501492001D
:100DB00070158E0090168B00B0178700D018840035
:100DC000F0198100101B7E00301C7B00501D790043
:100DD000701E7600901F7300B0207000D0216E004E
:100DE000F0226B0010246900302566005026630055
:100DF0007027610090285E00B0295C00D02A59005D
:100E0000F02B5600102D5400302E5100502F4E0064
:100E100070304B0090314800B0324500D033420072
:100E2000F0343E0010363B00303737005038330086
:100E300070392E00903A2900B03B2300D03C1B00B3
:100E4000F03D1100103F0100F03F00004572723A82
:100E5000204D494E54454D5020424544004D494E89
:100E600054454D502074726967676572656400452A
:100E700072723A204D494E54454D5020453100453F
:100E800072723A204D494E54454D50204530004530
:100E900072723A204D415854454D5020424544000D
:100EA0004D415854454D50207472696767657265AD
:100EB00064004572723A204D415854454D502045CA
:100EC00031004572723A204D415854454D502045ED
:100ED00030004572726F722077726974696E672094
:100EE000746F20454550524F4D210A002045002087
:100EF0005A0020204D3930372058005374657070E7
:100F00006572206D6F746F722063757272656E7496
:100F1000733A0A0020204D383531205A005A2D509E
:100F2000726F6265204F666673657420286D6D2947
:100F30003A0A0020440020490020204D333034205C
:100F4000500020440020490020204D3330312050F3
:100F5000005049442073657474696E67733A0A00DF
:100F600020204D3432302053004175746F2042658B
:100F700064204C6576656C696E673A0A00205A00F9
:100F800020590020204D323036205800486F6D65C2
:100F9000206F66667365743A0A00204500205A0087
:100FA00020590020580020420020540020204D32BB
:100FB0003035205300416476616E6365643A205396
:100FC0003C6D696E5F66656564726174653E205450
:100FD0003C6D696E5F74726176656C5F66656564B1
:100FE000726174653E20423C6D696E5F7365676D2A
:100FF000656E745F74696D655F6D733E20583C6DFE
:1010000061785F78795F6A65726B3E205A3C6D61EA
:10101000785F7A5F6A65726B3E20453C6D61785FF0
:10102000655F6A65726B3E0A002054002052002002
:10103000204D323034205000416363656C6572612D
:1010400074696F6E2028756E6974732F7332293A34
:1010500020503C7072696E745F616363656C3E2002
:10106000523C726574726163745F616363656C3E68
:1010700020543C74726176656C5F616363656C3E9D
:101080000A00204500205A0020590020204D32300F
:10109000312058004D6178696D756D20416363653D
:1010A0006C65726174696F6E2028756E6974732F38
:1010B0007332293A0A00204500205A0020590020A6
:1010C000204D3230332058004D6178696D756D20A8
:1010D0006665656472617465732028756E697473E2
:1010E0002F73293A0A00204500205A002059002079
:1010F000204D39322058005374657073207065722A
:1011000020756E69743A0A0020204D323030204438
:10111000300A0020204D32303020440020446973D2
:1011200061626C65640A0046696C616D656E74206D
:1011300073657474696E67733A00202047323120FA
:101140002020203B20556E69747320696E206D6DE0
:101150000A000224F4D43050C38E20C2A240178269
:101160008B7011127A910D816CD90AA861E108C7C0
:10117000586607615143061E4B5D05C145A7041A19
:10118000411104093D9803713931034036DB026592
:10119000339102D4305402802E1D02632CEE01756F
:1011A0002AC501B028A001102781018F2564012BD9
:1011B000244B01E0223401AC211F018D200D018060
:1011C0001FFC00841EED00971DDF00B81CD200E656
:1011D0001BC600201BBC00641AB200B219A8000A8A
:1011E00019A0006A189900D117910040178B00B51B
:1011F00016840031167E00B31579003A157300C7C6
:10120000146F0058146A00EE1366008813630025FB
:10121000135E00C7125B006C12570015125400C118
:1012200011510070114F0021114B00D61049008D53
:101230001047004610440002104200C00F400080DA
:101240000F3E00420F3C00060F3B00CB0E380093D0
:101250000E37005C0E3500270E3400F30D3200C14E
:101260000D3100900D3000600D2E00320D2D000567
:101270000D2C00D90C2B00AE0C2900850C29005C2C
:101280000C2700350C27000E0C2600E80B2400C4A8
:101290000B2400A00B23007D0B23005A0B210039E7
:1012A0000B2100180B2000F80A1F00D90A1E00BBF2
:1012B0000A1E009D0A1D00800A1D00630A1C0047CB
:1012C0000A1B002C0A1B00110A1A00F7091A00DD7C
:1012D000091900C4091900AB091900920917007B0C
:1012E000091800630917004C09160036091600207A
:1012F0000916000A091500F5081500E0081400CCCD
:10130000081400B8081400A4081400900813007D05
:101310000812006B08130058081200460812003427
:10132000081100230811001208110001081100F033
:10133000071000E0071000D0071000C0071000B031
:10134000070F00A107100091070E0083070F00741C
:10135000070F0065070E0057070E0049070E003BF8
:10136000070D002E070E0020070D0013070D0006C5
:10137000070D00F9060C00ED060D00E0060C00D488
:10138000060C00C8060C00BC060C00B0060C00A43D
:10139000060B0099060C008D060B0082060B0077E9
:1013A000060B006C060B0061060A0057060B004C8A
:1013B000060A0042060A0038060A002E060A002421
:1013C000060A001A060A001006090007060A00FDB0
:1013D000050900F4050900EB050900E2050900D93B
:1013E000050900D0050900C7050900BE050900B5BB
:1013F000050800AD050800A50509009C0508009436
:101400000508008C050800840508007C05080074A8
:101410000508006C050700650508005D0507005616
:101420000508004E0507004705070040050800387D
:10143000050700310507002A050700230507001CE2
:10144000050600160507000F05070008050600023F
:10145000050700FB040600F5040700EE040600E89B
:10146000040600E2040700DB040600D5040600CFF2
:10147000040600C9040600C3040600BD040600B744
:10148000040600B1040500AC040600A6040600A092
:101490000405009B04060095040500900406008ADC
:1014A00004050085040500800406007A0405007523
:1014B000040500700405006B040500660405006166
:1014C0000405005C04050057040500520405004DA6
:1014D00004050048040500430405003E0404003AE6
:1014E00004050035040500300404002C0405002721
:1014F000040400230405001E0404001A040400165A
:10150000040500110404000D04040009040500048E
:1015100004040000040400FC030400F8030400F4C5
:10152000030400F0030400EC030400E8030400E4F7
:10153000030400E0030400DC030400D8030400D427
:10154000030400D0030400CC030400C8030300C557
:1015500003030024F404D9201BC40C5C0E9804C4BB
:10156000095F0265077101F405F900FB04B3004847
:10157000048700C10369005803550003034500BEFA
:10158000023A008402310053022A00290225000495
:10159000022000E4011C00C8011900AF01170098E7
:1015A0000114008401130071011000610110005149
:1015B000010E0043010D0036010B002B010B002032
:1015C000010B00150109000C01090003010800FBD3
:1015D000000800F3000800EB000700E4000600DE4E
:1015E000000600D8000600D2000600CC000500C7A7
:1015F000000500C2000500BD000400B9000400B5EC
:10160000000400B1000400AD000400A9000400A51E
:10161000000300A20003009F0004009B0003009849
:101620000003009500020093000300900003008D6A
:101630000002008B00030088000200860002008484
:10164000000300810002007F0002007D0002007B99
:1016500000020079000200770001007600020074A9
:1016600000020072000100710002006F0002006DB4
:101670000001006C0002006A0001006900020067BE
:1016800000010066000100650001006400020062C4
:1016900000010061000100600001005F0002005DC8
:1016A0000001005C0001005B0001005A00010059CC
:1016B00000010058000100570001005600010055CC
:1016C00000010054000100530000005300010052CB
:1016D00000010051000100500001004F0001004EC8
:1016E0000000004E0001004D0001004C0001004BC5
:1016F0000000004B0001004A0001004900010048C1
:1017000000000048000100470001004600000046BC
:1017100000010045000000450001004400010043B5
:1017200000000043000100420000004200010041AF
:1017300000000041000100400001003F0000003FA8
:101740000001003E0000003E0001003D0000003DA1
:101750000001003C0000003C0000003C0001003B98
:101760000000003B0001003A0000003A000100398F
:101770000000003900010038000000380000003887
:10178000000100370000003700010036000000367D
:101790000000003600010035000000350000003573
:1017A0000001003400000034000000340001003368
:1017B000000000330000003300010032000000325E
:1017C0000000003200010031000000310000003153
:1017D0000001003000000030000000300001002F48
:1017E0000000002F0000002F0000002F0001002E3D
:1017F0000000002E0000002E0001002D0000002D32
:101800000000002D0000002D0001002C0000002C25
:101810000000002C0000002C0001002B0000002B19
:101820000000002B0000002B0001002A0000002A0D
:101830000000002A0000002A000100290000002901
:1018400000000029000000290000002900010028F4
:1018500000000028000000280000002800000028E8
:1018600000010027000000270000002700000027DB
:1018700000000027000100260000002600000026CE
:1018800000000026000000260001002500000025C1
:1018900000000025000000250000002500000025B4
:1018A00000010024000000240000002400000024A7
:1018B000000000240001002300000023000000239A
:1018C000000000230000002300000023000000238C
:1018D000000100220000002200000022000000227F
:1018E0000000002200000022000100210000002171
:1018F0000000002100000021000000210000002164
:101900000000002100010020000000200000002055
:101910000000002000000020000000200000002047
:10192000000000200001001F0000001F0000001F39
:101930000000001F0000001F0000001F0000001F2B
:101940000001001E0000001E0000001E0000001E1E
:10195000000000290A002062797465733B206372DD
:1019600063200053657474696E67732053746F72DB
:101970006564202800202863616C63756C61746560
:101980006429210A0020213D2000454550524F4D39
:1019900020435243206D69736D61746368202D206C
:1019A0002873746F726564292000290A0020627907
:1019B0007465733B2063726320002073746F7265DB
:1019C000642073657474696E6773207265747269DC
:1019D00065766564202800204D61726C696E3D5605
:1019E0003430290A0028454550524F4D3D004545A9
:1019F00050524F4D2076657273696F6E206D69731A
:101A00006D61746368200048617264636F6465642B
:101A10002044656661756C742053657474696E67E3
:101A200073204C6F616465640A002823000028233A
:101A3000000064000000E80300000000964300007E
:101A4000964300000041000020420000C94200000F
:101A5000C9420000C8440040504400002000230058
:101A6000260029002C002F00320000010000030195
:101A700006010901656E7175657565696E672022DD
:101A8000004E6F204C696E65204E756D6265722048
:101A90007769746820636865636B73756D2C204C7F
:101AA000617374204C696E653A20005072696E74DF
:101AB00065722073746F707065642064756520743E
:101AC0006F206572726F72732E2046697820746879
:101AD00065206572726F7220616E64207573652077
:101AE0004D39393920746F20726573746172742EA8
:101AF000202854656D706572617475726520697314
:101B00002072657365742E2053657420697420619A
:101B1000667465722072657374617274696E672988
:101B20000A004E6F20436865636B73756D2077699B
:101B30007468206C696E65206E756D6265722C200C
:101B40004C617374204C696E653A2000636865636C
:101B50006B73756D206D69736D617463682C204CB7
:101B6000617374204C696E653A20004C696E652083
:101B70004E756D626572206973206E6F74204C61C2
:101B80007374204C696E65204E756D6265722B31E1
:101B90002C204C617374204C696E653A20004D31E5
:101BA0003130004B494C4C45442E20004B494C4CA5
:101BB0002063617573656420627920746F6F206D96
:101BC00075636820696E6163746976652074696DF8
:101BD00065202D2063757272656E7420636F6D6D64
:101BE000616E643A20005072696E7465722068619B
:101BF0006C7465642E206B696C6C28292063616CA1
:101C00006C6564210A00000040C000003E430000F3
:101C10001F430000F0410000F041000000410000BF
:101C200000005761726E696E673A20486F6D696E89
:101C3000672042756D702044697669736F72203C2D
:101C400020310A000202040000A0400000A0400071
:101C5000000040000025430000454300002143FFF1
:101C600001014B494C4C45442E200000000A0B0258
:101C7000090C0D0E0807030401000000000000001D
:101C80000000000000000000000000000000000054
:101C90000000000000000012111000000000000011
:101CA0000000000000000000000000000000000034
:101CB000002066697273740A005A0059005800487F
:101CC0006F6D6520006563686F3A00544845524D5A
:101CD000414C2052554E41574159204245440054F1
:101CE0006865726D616C2052756E61776179005420
:101CF0004845524D414C2052554E4157415920457F
:101D00003100544845524D414C2052554E415741A7
:101D1000592045300000002200250028002B002E0D
:101D2000003100340002010000050108010B010030
:101D3000002100240027002A002D0030003300017C
:101D4000010000040107010A010505050507050852
:101D5000080808020202020A0A080804040404012E
:101D60000101010101010103030303030303030450
:101D70000707070C0C0C0C0C0C0C0C0202020206E0
:101D8000060606060606060B0B0B0B0B0B0B0B01D0
:101D9000021020200808102040102040800201027C
:101DA0000108040201010204081020408080402044
:101DB000100804020180040201804020100804027F
:101DC00001080402010102040810204080010204FD
:101DD0000810204080526573656E643A20002042EE
:101DE000002050006F6B0000EA9011241FBECFEF5F
:101DF000D1E2DEBFCDBF00E00CBF13E0A0E0B2E057
:101E0000E4E2F1E401E00BBF02C007900D92AE31B5
:101E1000B107D9F72DE0AEE1B3E001C01D92A132C8
:101E2000B207E1F71EE0C5EFDEE000E006C0219753
:101E30000109802FFE010E9462A0C43FD10780E00B
:101E40000807A9F70E94E1340C9490A00C940000BC
:101E50002F923F924F925F926F927F928F929F92BA
:101E6000AF92BF92CF92DF92EF92FF920F931F93A8
:101E7000CF93DF93CDB7DEB7C357D1090FB6F89430
:101E8000DEBF0FBECDBF0091800320E6029F800120
:101E900011240556144F8091A40380FF1AC0E5EC6D
:101EA000FCE184917F013FEFE31AF30A811102C044
:101EB000780104C00E94D28BF701F3CFD7018D9136
:101EC0007D01882319F00E94D28BF8CF8AE00E940E
:101ED000D28B10923D0310923C038FE38093460314
:101EE0001092450310924403109238031092390364
:101EF00010923A0310923B03F80180810F5F1F4F4D
:101F00008032D1F38E34B1F4818190ED980F9A3004
:101F100020F08D3211F08B3269F43296DF01319668
:101F20002C9120532A30D0F3CD01FC010196208161
:101F30002032D9F3F093290AE093280A7F01BFEFFA
:101F4000EB1AFB0A10816AE270E0C7010E9470A0E0
:101F5000009731F0FC01319780818032E1F31182EA
:101F60001D3429F0143519F0173409F0CDC0F701EC
:101F700080812FEFE21AF20A8032C9F380538A304F
:101F800008F0C2C0109346032091440330914503EA
:101F90004AE03196429FC001439F900D1124DF011A
:101FA00011972C9130E020533109280F391F80817F
:101FB00080538A3070F33093450320934403DF014C
:101FC00031968C918032D9F31D3449F00091280A62
:101FD00040913C0350913D0361E070E058C02E31C8
:101FE000310591F03CF42731310571F02C31310588
:101FF00069F70AC0253731054CF32737310524F03E
:10200000203A43E0340711F7B0933D03A0933C031B
:102010007BC0813209F445C09FEBB92EB80E89E12F
:10202000A82EAB1408F45EC0DF01FD01908111966B
:102030009032D9F3A0EDA90FAA3008F047C04F01A4
:10204000EB2CF12C670183E0D594C7948A95E1F7D6
:10205000C601885C9C4F6C018B2D8770DB0102C030
:10206000AA0FBB1F8A95E2F7CD01D6019C91892B5F
:102070008C9381149104A1F1801AC701825E9C4F58
:10208000DC018C92808181548A3188F5DF01FD0169
:1020900031968C918111BDCF50933D0340933C0309
:1020A00033C01D3409F0B8CF2032310509F0B4CF68
:1020B000F0933D03E0933C0363E270E0CF010E94A4
:1020C00070A0009709F1DC011C921EC0A3EDA90FBE
:1020D000A23008F4B4CF9B3211F00C947E27AFCF1E
:1020E000812CCBCF4115510569F6AD01CBCFDF0176
:1020F00031969C9190539A30D0F3CD01FC0101961A
:10210000A081A032D9F3C2CF809146038D3411F45F
:102110000C94301A843511F40C942027873411F074
:102120000C94612780914403909145038A31910575
:1021300009F4E0C6A4F48430910544F4823091059A
:102140000CF020C197FF2CC00C947B2784309105A4
:1021500009F451C60C9709F48BC60C947B278E3179
:10216000910511F40C946F1944F48C31910509F424
:1021700050C70CF4C4C60C9460198B35910511F44A
:102180000C94F5198C35910511F40C94FA198A35D3
:10219000910511F00C947B27109243030C947B273C
:1021A00080912102882311F40C947B270E94D94B43
:1021B0008EE39AE00E9495900E947E8B8091A4030A
:1021C00083FD8FC0C0904A0AD0904B0AE0904C0A21
:1021D000F0904D0A2091210B3091220B4091230B5E
:1021E0005091240BC701B6010E944099882309F43D
:1021F00078C080919803811138C060911D02709160
:102200001E02072E000C880B990B0E9446999B0119
:10221000AC016091130470911404809115049091A5
:1022200016040E94409987FF20C0C092210BD092D3
:10223000220BE092230BF092240BE5ECFCE184915D
:102240008F010F5F1F4F882321F00E94D28BF8016E
:10225000F6CFE2E0F2E084918F010F5F1F4F8823F9
:1022600021F00E94D28BF801F6CFC0904A0AD0909C
:102270004B0AE0904C0AF0904D0A2091210B3091CE
:10228000220B4091230B5091240BC701B6010E94F1
:10229000729D20E030E048E453E40E94999F1816B4
:1022A00004F5C092210BD092220BE092230BF09206
:1022B000240BE5ECFCE184918F010F5F1F4F882315
:1022C00021F00E94D28BF801F6CFE3EEF1E0849189
:1022D0008F010F5F1F4F882321F00E94D28BF801DE
:1022E000F6CF20913E0A30913F0A4091400A50912A
:1022F000410A6091150B7091160B8091170B90910C
:10230000180B0E94409981111DC02091420A309102
:10231000430A4091440A5091450A6091190B70910B
:102320001A0B80911B0B90911C0B0E9440998111FC
:1023300009C06091190270911A0280911B0290915C
:102340001C021AC06091000270910102072E000C5D
:10235000880B990B0E9446992091190230911A021C
:1023600040911B0250911C020E94A5992AE037ED72
:1023700043E25CE30E94A5990E94D35C0E94C95C81
:102380000C947B2720912102222311F40C947B27AB
:1023900011E0029709F010E00E94D94B82E50E94FB
:1023A000B988882309F430C10E9457886B017C01E9
:1023B0004090150B5090160B6090170B7090180BF7
:1023C0002091190B30911A0B40911B0B50911C0B53
:1023D0002FA338A749A75AA780913E0A90913F0A98
:1023E000A091400AB091410A8BA79CA7ADA7BEA7B8
:1023F0002091420A3091430A4091440A5091450A83
:102400002BAB3CAB4DAB5EAB20E030E0A901C7018C
:10241000B6010E944099882309F4D3C4A301920114
:102420006BA57CA58DA59EA50E94409981110DC02C
:102430002FA138A549A55AA56BA97CA98DA99EA94C
:102440000E944099882309F4BCC420E030E0A9012F
:10245000C701B6010E944099881F8827881F18135A
:102460000BC080E090E0A0E8BFE323968CAF9DAF67
:10247000AEAFBFAF23970AC020E030E040E85FEB8B
:1024800023962CAF3DAF4EAF5FAF2397A3019201D0
:102490006BA57CA58DA59EA50E94729D6FAB78AFA4
:1024A00089AF9AAF2FA138A549A55AA56BA97CA9D8
:1024B0008DA99EA90E94729D6BAF7CAF8DAF9EAF20
:1024C0002FA938AD49AD5AADCA01B9010E94A599ED
:1024D0004B015C012BAD3CAD4DAD5EADCA01B90108
:1024E0000E94A5999B01AC01C501B4010E94739D96
:1024F0000E94DE9F6FA778AB89AB9AAB20E030E0FB
:1025000040E05FE30E94A5994B015C01A7019601A1
:10251000C701B6010E94A5996B017C01A501940138
:10252000C501B4010E94A5999B01AC01C701B60188
:102530000E94729D0E94DE9F9B01AC0123966CADB0
:102540007DAD8EAD9FAD23970E94A5994B015C0197
:102550002BA53CA54DA55EA5C301B2010E94739DAC
:1025600020E030E040E05FE30E94A5996B017C0130
:102570006BAD7CAD8DAD9EAD90582FA538A949A906
:102580005AA90E944F9E9B01AC01C501B4010E9453
:10259000A5999B01AC01C701B6010E94739DA301DF
:1025A00092010E94729D6B017C012BA93CA94DA94F
:1025B0005EA96FA178A589A59AA50E94739D20E0C8
:1025C00030E040E05FE30E94A5992B013C012FA57C
:1025D00038A949A95AA96FA978AD89AD9AAD0E94C9
:1025E0004F9E9B01AC01C501B4010E94A5999B01BE
:1025F000AC01C301B2010E94739D2FA138A549A56A
:102600005AA50E94729D14C089E40E94B98888234B
:1026100029F00E9457886B017C0103C0C12CD12C8A
:1026200076018AE40E94B9888823D9F00E945788ED
:102630006BAB7CAB8DAB9EAB20E030E0A901C7015A
:10264000B6010E94409981111AC020E030E0A90132
:102650006BA97CA98DA99EA90E94409981110FC0E8
:10266000B0C320E030E0A901C701B6010E94409943
:10267000882309F4A6C31BAA1CAA1DAA1EAAD70157
:10268000C601B0588FA398A7A9A7BAA72BA93CA9A0
:102690004DA95EA950582BA73CA74DA75EA79C014A
:1026A000AD01BC01CD010E94A5994B015C012BA598
:1026B0003CA54DA55EA5CA01B9010E94A5999B0143
:1026C000AC01C501B4010E94739D0E94DE9F639618
:1026D0006CAF7DAF8EAF9FAF63978091150B9091DC
:1026E000160BA091170BB091180B8FA798ABA9AB45
:1026F000BAABA7019601BC01CD010E94739D239640
:102700006CAF7DAF8EAF9FAF23972091190B3091A7
:102710001A0B40911B0B50911C0B2FAB38AF49AFDC
:102720005AAF2BA93CA94DA95EA96FA978AD89AD77
:102730009AAD0E94739D27966CAF7DAF8EAF9FAF11
:10274000279780913E0A90913F0AA091400AB0914C
:10275000410A2B968CAF9DAFAEAFBFAF2B972396A0
:102760002CAD3DAD4EAD5FAD2397BC01CD010E94B8
:10277000729D6B017C012091420A3091430A409185
:10278000440A5091450A2F962CAF3DAF4EAF5FAF34
:102790002F9727962CAD3DAD4EAD5FAD27972F9669
:1027A0006CAD7DAD8EAD9FAD2F970E94729D4B019C
:1027B0005C0180911D0B90911E0BA0911F0BB0919D
:1027C000200B6B968CAF9DAFAEAFBFAF6B979C01EC
:1027D000AD016091460A7091470A8091480A909134
:1027E000490A0E94729D6BAF7CAF8DAF9EAF209166
:1027F000210B3091220B4091230B5091240B6F96AB
:102800002CAF3DAF4EAF5FAF6F9760914A0A7091AA
:102810004B0A80914C0A90914D0A0E94729D6796D6
:102820006CAF7DAF8EAF9FAF6797A70196016FA189
:1028300078A589A59AA50E94A5992B013C01A5011F
:1028400094016BA57CA58DA59EA50E94A5999B01D1
:10285000AC01C301B2010E94739D2B013C01A50193
:1028600094016FA178A589A59AA50E94A5994B010D
:102870005C01A70196016BA57CA58DA59EA50E9474
:10288000A5999B01AC01C501B4010E94729DA301F1
:1028900092010E94E69D6B017C0120E030E0A901DD
:1028A0000E94409987FF0AC02BED3FE049EC50E4BD
:1028B000C701B6010E94739D6B017C01112351F089
:1028C0002BED3FE049EC50E4C701B6010E94729D38
:1028D0006B017C0120E030E0A901C701B6010E9434
:1028E0004099811124C02B962CAD3DAD4EAD5FAD0E
:1028F0002B976FA578A989A99AA90E94409981115F
:1029000016C02F962CAD3DAD4EAD5FAD2F976FA984
:1029100078AD89AD9AAD0E944099811108C00BED48
:10292000C02E0FE0D02E09ECE02E00E4F02E6396CE
:102930002CAD3DAD4EAD5FAD6397C701B6010E94B2
:10294000A5999B01AC010E94A5994B015C012BAD9F
:102950003CAD4DAD5EADCA01B9010E94A5999B0188
:10296000AC01C501B4010E94739D0E94DE9F4B0122
:102970005C012FE632E143E85AE30E94409987FD6B
:102980001CC2C501B4010E94E89E0E94BC9E78AFA3
:102990006FAB672B21F421E030E038AF2FABAFA84D
:1029A000B8ACB50180E090E00E9444994B015C0115
:1029B0009B01AC01C701B6010E944F9E6FA778AB87
:1029C00089AB9AABA50194016BAD7CAD8DAD9EAD8D
:1029D0000E944F9E63966CAF7DAF8EAF9FAF6397A3
:1029E000A501940167966CAD7DAD8EAD9FAD6797E7
:1029F0000E944F9E67966CAF7DAF8EAF9FAF67977B
:102A00002FA538A949A95AA9CA01B9010E94A599B7
:102A100020E030E040E05FE30E94A5999B01AC011B
:102A200060E070E080E89FE30E94729D6BAF7CAF36
:102A30008DAF9EAF6B962CAD3DAD4EAD5FAD6B9740
:102A400029873A874B875C876F968CAD9DADAEAD7D
:102A5000BFAD6F978D879E87AF87B88B609100025F
:102A600070910102072E000C880B990B0E94469969
:102A70002091190230911A0240911B0250911C02C0
:102A80000E94A5992AE037ED43E25CE30E94A599F4
:102A90002B966CAF7DAF8EAF9FAF2B970E94728B42
:102AA0009B01AC0128533F4F4F4F5F4F2F962CAFE8
:102AB0003DAF4EAF5FAF2F974FA058A469A47AA443
:102AC00022242394312C19E1D12EAFA8B8AC2A14BA
:102AD0003B0409F42EC10E9423650E94728BDC0125
:102AE000CB012F962CAD3DAD4EAD5FAD2F97821B28
:102AF000930BA40BB50BB7FD10C00E94728B9B010A
:102B0000AC0128533F4F4F4F5F4F2F962CAF3DAF37
:102B10004EAF5FAF2F970E94038EDA94DD20E9F16C
:102B20002BAD3CAD4DAD5EAD6BA57CA58DA59EA539
:102B30000E94A5994B015C012FA538A949A95AA962
:102B4000B201C3010E94A599A50194010E94739D41
:102B50007B018C012BAD3CAD4DAD5EADB201C3012F
:102B60000E94A5994B015C012FA538A949A95AA932
:102B70006BA57CA58DA59EA50E94A5999B01AC0186
:102B8000C501B4010E94729D2B013C01C701D8010F
:102B90008BA79CA7ADA7BEA74FC0B10180E090E076
:102BA0000E9444992FA538A949A95AA90E94A5991C
:102BB0004B015C010E944C9E6B017C01C501B4017C
:102BC0000E94D49F4B015C01A70196016FA178A5DB
:102BD00089A59AA50E94A5992B013C01A501940104
:102BE0006BA97CA98DA99EA90E94A5999B01AC0106
:102BF000C301B2010E94739D2B013C01A501940108
:102C00006FA178A589A59AA50E94A5994B015C01A1
:102C1000A70196016BA97CA98DA99EA90E94A599DF
:102C20009B01AC01C501B4010E94729D6BA77CA7FA
:102C30008DA79EA7A9E1DA2E9201A30123966CAD80
:102C40007DAD8EAD9FAD23970E94739D69837A837E
:102C50008B839C832BA53CA54DA55EA527966CADCB
:102C60007DAD8EAD9FAD27970E94739D6D837E8352
:102C70008F83988763962CAD3DAD4EAD5FAD639766
:102C800069857A858B859C850E94739D69877A8783
:102C90008B879C8767962CAD3DAD4EAD5FAD67973A
:102CA0006D857E858F8598890E94739D6D877E874F
:102CB0008F87988BCE0101960E949590C0908203D9
:102CC00089819A81AB81BC818E8B9F8BA88FB98FB4
:102CD0008D819E81AF81B8858A8F9B8FAC8FBD8F90
:102CE00089859A85AB85BC858E8F9F8FA8A3B9A354
:102CF000AE01425E5F4FBE01665E7F4FCE014696DB
:102D00000E94E6492B96ECACFDAC0EAD1FAD2B97A7
:102D10009E01235F3F4FAE01425E5F4FBE01665E84
:102D20007F4FCE0146960E94DE3B3FEF231A330AC7
:102D3000CCCEC090820380913E0A90913F0AA09130
:102D4000400AB091410A8E8B9F8BA88FB98F8091DA
:102D5000420A9091430AA091440AB091450A8A8F91
:102D60009B8FAC8FBD8F8091460A9091470AA091AE
:102D7000480AB091490A8E8F9F8FA8A3B9A3AE01CC
:102D8000425E5F4FBE01665E7F4FCE0146960E9457
:102D9000E6492B96ECACFDAC0EAD1FAD2B972AE4AB
:102DA0003AE0AE01425E5F4FBE01665E7F4FCE01EC
:102DB00046960E94DE3B0E94C95C0E947E8B0C946A
:102DC0007B27EBECF9E084918F010F5F1F4F882385
:102DD00021F00E94D28BF801F6CFEDE1F2E0849170
:102DE0008F010F5F1F4F882311F40C947B270E94E3
:102DF000D28BF801F4CF80E50E94B988882329F0AE
:102E00000E9417886B017C0103C0C12CD12C760174
:102E100083E50E94B988882361F00E94578820E0EA
:102E200030E04AE754E40E94A5990E94BC9E6B01E1
:102E30007C010E9474720E947E8B80912A0A90917C
:102E40002B0AA0912C0AB0912D0AC80ED91EEA1E99
:102E5000FB1E0E94728BDC01CB018C199D09AE090F
:102E6000BF09B7FD02C00C947B270E94038EF1CFEF
:102E70000E944E9281110C947B2780E50E94B988B4
:102E8000882319F00E94278801C060E06EA383E5C3
:102E90000E94B988882319F00E94278801C06CE03D
:102EA0006AA384E50E94B988882319F00E942788C4
:102EB00001C063E06E8B82E50E94B988882319F017
:102EC0000E94578804C060E070E080ED90E4698360
:102ED0007A838B839C839E012A5E3F4FAE014F5FB6
:102EE0005F4FBE016E5D7F4FCE0186960E94A76741
:102EF0000C947B2781E0809321020C947B270E9415
:102F00004E9281110C947B2780E50E94B98888231A
:102F100021F00E942788262F01C020E060911D0B20
:102F200070911E0B80911F0B9091200BC12CD12C06
:102F300040EEE42E40E4F42EC982DA82EB82FC8279
:102F4000C12CD12C54E3E52E53E4F52ECD82DE8244
:102F5000EF82F886C12CD12CE0EAEE2EE1E4FE2EC1
:102F6000C986DA86EB86FC86C12CD12CF0ECEF2EDC
:102F7000FFE7FF2ECD86DE86EF86F88A213071F1DD
:102F8000223021F51E8A1F8A188E198E20E030E02B
:102F900040EA51E40E94739D6B017C0120E030E027
:102FA0004FE153E40E94999F181634F4C12CD12CA0
:102FB0003FE1E32E33E4F32ECAA2DBA2ECA2FDA292
:102FC000BE016A5E7F4FCE01829611C020E030E0E4
:102FD00040EA51E40E94409987FF0BC01E8A1F8A75
:102FE000188E198EBE016A5E7F4FCE0109960E942F
:102FF000C15C1E8A1F8A188E198EAE014A5E5F4F11
:10300000BE016B5F7F4FCE0101960E94BC5C0C94A9
:103010007B270E9474722090170480E00E94E64C87
:103020000E94404D81E08093520388E50E948A8887
:10303000382E89E50E948A88082F8AE50E948A88AE
:10304000311005C0011105C011E0182705C001119C
:1030500002C010E001C0182F90E1E5E1FBE0AEE313
:10306000BAE001900D929A95E1F7111105C0811116
:1030700003C0311006C033C082E00E94E68C1123E9
:10308000C1F320E030E040E850E460919403709197
:10309000950380919603909197030E94739D60938E
:1030A000460A7093470A8093480A9093490A2091F0
:1030B0001D0B30911E0B40911F0B5091200B0E9455
:1030C000999F18167CF419821A821B821C82BE01F9
:1030D0006F5F7F4F86E49AE00E94C15C03C00111DC
:1030E000D0CFDFC011110DC0311003C00111D6C007
:1030F000D8C0011106C080E00E94E68C1123B1F314
:10310000CDC01092190B10921A0B10921B0B10923B
:103110001C0B1092150B1092160B1092170B10929D
:10312000180B0E94D087EFE5FCE1B490BBA6E3E565
:10313000FCE1C590D590E590F490E7E5FCE1859041
:103140009590A590B490A5019401C701B6010E9485
:10315000999F18162CF4A7019601C501B40104C06B
:10316000A5019401C701B6010E944F9E6FA378A7E5
:1031700089A79AA7B2E16B2EBCE17B2EF301659182
:1031800075918591949126E1422E2CE1522EF20107
:1031900025913591459154910E94409987FF02C035
:1031A000F30101C0F20145905590659074902FA1F4
:1031B00038A549A55AA5CA01B9010E94A59920E0E0
:1031C00030E040E85FE30E94739D0E94DE9F9B0118
:1031D000AC01C301B2010E94A5996AA37BA38CA391
:1031E0009DA3E0E6FCE124912FA320E030E040EC39
:1031F0005FE3C501B4010E94A5992B013C01AFA07A
:103200006A2DAA0C770B880B990B0E9446999B019B
:10321000AC01C301B2010E94A59969837A838B83B3
:103220009C8320E030E040EC5FE3C701B6010E94E0
:10323000A5996B017C01BBA46B2DBB0C770B880B94
:10324000990B0E9446999B01AC01C701B6010E94EF
:10325000A5996E8B7F8B888F998FAE014E5D5F4FE6
:10326000BE016F5F7F4FCE0146960E94BC5C1092FC
:10327000000B1092190B10921A0B10921B0B10924C
:103280001C0B1092150B1092160B1092170B10922C
:10329000180B111130CF31102ECF28CF81E00E94B2
:1032A000E68C0E94D0878091510380935203822D37
:1032B0000E94E64C0E94264D0E94BB2E0C947B2758
:1032C00081E08093530324982C9A149A0E94884E8C
:1032D00010925303249A2C9814980C947B2720E086
:1032E00030E0A9016091150B7091160B8091170BBE
:1032F0009091180B0E94739D6B017C0188E50E94E0
:10330000B988882321F00E9457886B017C01CE8AFE
:10331000DF8AE88EF98E20E030E0A9016091190B78
:1033200070911A0B80911B0B90911C0B0E94739D46
:103330006B017C0189E50E94B988882321F00E94F5
:1033400057886B017C01C982DA82EB82FC82409053
:10335000900350909103609092037090930320919A
:103360008C0330918D0340918E0350918F036E89B1
:103370007F89888D998D0E94729D4B015C0122E6A8
:1033800030E140E450EC0E94999F87FF02C00C940A
:103390007B2722E430E042E253E4C501B4010E94FD
:1033A0004099181614F40C947B27A3019201C701CD
:1033B000B6010E94729D6B017C0121E338E040EE72
:1033C00050EC0E94999F87FF02C00C947B2722E457
:1033D00030E04EE353E4C701B6010E94409918164D
:1033E00014F40C947B270C94882781E0809343038A
:1033F0000C947B2785E40E94B988082F811102C0B4
:103400000E947472FCEFAF2EF2E0BF2EA5E1EA2E0F
:10341000ABE0FA2ED12C10E0D5018D915D010E9418
:10342000B988882359F00E945788F7016083718317
:1034300082839383133011F0DD24D3941F5FF4E073
:10344000EF0EF11C143041F7DD2019F00E94D087F7
:1034500003C001110E94B4920E94BB2E0C947B27E2
:1034600080914403909145038B39910509F43EC343
:103470000CF085C08C35910509F4D2C3E4F58B348A
:10348000910509F4D2C2BCF48131910509F4A1C1BE
:103490002CF4029708F424C10C947B278F319105FA
:1034A00009F49DC18A32910509F469C2429711F06D
:1034B0000C947B2796C38235910509F489C37CF46B
:1034C0008D34910509F4CAC20CF4B3C2813591055B
:1034D00011F00C947B270E9420300C947B278435BC
:1034E000910509F47EC30CF477C38535910509F481
:1034F0007CC30C947B278F36910509F4BBC2DCF4A6
:103500008A36910509F44EC354F48836910509F4BE
:10351000A9C28936910509F4CFC20C947B278D3658
:10352000910509F40EC30CF0A1C28B36910509F484
:103530003DC30C947B278737910509F4F8C49CF4AC
:103540008337910509F4F5C38637910509F483C4DF
:103550008237910511F00C947B270E9474720E94AF
:10356000BB2E0C947B278937910509F4B2C50CF466
:10357000AAC58C38910509F481C20C947B2780334D
:1035800021E0920709F419C70CF049C08E3C91055F
:1035900009F415C60CF5893C910509F49FC56CF436
:1035A0008E3B910509F4E9C2883C910511F00C9419
:1035B0007B270E946E2E0C947B278C3C910509F48E
:1035C00090C50CF091C58B3C910511F00C947B27B4
:1035D0000E94272E0C947B27823E910509F40EC68B
:1035E0008CF48C3D910509F4EDC58D3D910509F4F0
:1035F000ECC5833D910511F00C947B270E94282D8A
:103600000C947B278E3241E0940709F453C70CF0E9
:10361000A5C78D32914009F432C60C947B278C3AB1
:10362000B1E09B0711F40C94132664F58039F1E0A6
:103630009F0711F40C94B425ACF48F3531E0930757
:1036400011F40C940C27833641E0940711F40C9488
:103650000E278E35914011F00C947B270E94A62CEA
:103660000C947B278239A1E09A0711F40C94BB25B6
:1036700014F40C94B725843A914011F40C94BF25AE
:103680000C947B27873FF1E09F0711F40C94CB2625
:1036900094F4853F31E0930711F40C94C52614F09F
:1036A0000C94C826843F914011F00C947B270E9413
:1036B000C2800C947B278B38A3E09A0711F40C94FA
:1036C0000A27873EB3E09B0711F40C94102783353B
:1036D000934011F00C947B27E5ECFCE10C94D92687
:1036E000E0903C03F0903D0380E50E94B988882378
:1036F00059F00E9417884B015C0111E0672B682B81
:10370000692B31F410E004C010E0812C912C54019D
:1037100083E50E94B988882399F00E94578820E0A9
:1037200030E04AE754E40E94A5990E94BC9E4B01F8
:103730005C0111110CC0672B682B692B41F436C05A
:10374000111105C0E114F10411F00C94DD2781E0A2
:1037500080934E0A0E9474720E947E8B81149104A1
:10376000A104B10479F180912A0A90912B0AA091C9
:103770002C0AB0912D0A75016401C80ED91EEA1EEB
:10378000FB1E0E94728BDC01CB018C199D09AE09D6
:10379000BF09B7FD04C010924E0A0C947B2780919C
:1037A0004E0A8823C1F30E94038EEBCFE114F1048B
:1037B00011F00C94DD2781E080934E0A0E94747210
:1037C0000E947E8B80914E0A882329F30E94038EEB
:1037D000F9CF17981698159814980C947B27809118
:1037E0008A0B813019F40E94728B08C06091930B90
:1037F0007091940B8091950B9091960B00918F0B8B
:103800001091900B2091910B3091920B601B710BDA
:10381000820B930B28EE33E040E050E00E941B9DAA
:1038200080918B0B90918C0BA0918D0BB0918E0B96
:10383000BC01CD01620F731F841F951FECE3CE2ED8
:10384000D12CE12CF12CA70196010E941B9D762E14
:10385000672ECA01B901A70196010E941B9D6B0149
:103860007C01CA01B90128E130E040E050E00E944B
:103870001B9D4B015C01C9016DE671E00E943BA0FC
:103880008E010F5F1F4F6115710599F06F927F9246
:10389000DF92CF929F928F929F938F937F936F939C
:1038A0008DE692E09F938F931F930F930E9411993F
:1038B00026C0009789F06F927F92DF92CF929F92FD
:1038C0008F929F938F938DE592E09F938F931F9399
:1038D0000F930E94119913C081149104A104B104A3
:1038E000B1F06F927F92DF92CF929F928F9281E59B
:1038F00092E09F938F931F930F930E9411990FB69D
:10390000F894DEBF0FBECDBFE5ECFCE123C0C114CF
:10391000D104E104F10469F06F927F92DF92CF92BB
:1039200089E492E09F938F931F930F930E941199C4
:10393000E6CF6F927F9285E492E09F938F931F93DF
:103940000F930E9411990F900F900F900F900F906E
:103950000F90DACF84917F01BFEFEB1AFB0A882327
:1039600021F00E94D28BF701F5CFB80181E892E0F7
:103970000E947F678AE00E94D28B0C947B2783E5AC
:103980000E94B988882311F40C947B270E94378801
:10399000E82E80E50E94B988811112C081E0E11013
:1039A00001C080E080935303882329F024982C9A47
:1039B000149A0C947B27249A2C9814980C947B27A7
:1039C00080E50E94B988882339F00E9427888B01FE
:1039D00077FF04C00C947B270DE010E0902FEEE8F9
:1039E000F2E088E28E0F2491921729F031968E131F
:1039F000FACF0C94FC27EBECF9E084918F010F5F78
:103A00001F4F882321F00E94D28BF801F6CFE6EBFE
:103A1000F2E084918F010F5F1F4F882311F40C9403
:103A20007B270E94D28BF801F4CF0E944B930C9419
:103A30007B2780918A0B813011F00C947B2782E0E8
:103A400080938A0B0E94728B6093930B7093940BFC
:103A50008093950B9093960B0C947B270E945D911D
:103A60000C947B270E946A310C947B270E94B6300D
:103A70000C947B270E9444300C947B278091A403F4
:103A800083FF02C00C947B2783E50E94B9888823BA
:103A900011F40C947B270E9457880E94B79E6739C7
:103AA000710514F066E970E07093F8036093F70312
:103AB0000E94D0610C947B2789E690E00E94855D8E
:103AC00081110C94F42BE5ECF2E084918F010F5FEF
:103AD0001F4F882321F00E94D28BF801F6CF0E945D
:103AE000E7308AE00E94D28B0C94F42B83E50E948D
:103AF000B988882311F40C947B270E94378880931F
:103B00001B0A8D3318F08CE380931B0A0E94728B82
:103B10006B017C0120911B0A30E0A8EEB3E00E940B
:103B2000639DDC01CB018C0D9D1DAE1DBF1D8093DF
:103B3000170A9093180AA093190AB0931A0A0C94C2
:103B40007B278DE690E00E94855D81110C947B2798
:103B50008091A40383FF02C00C947B2783E50E941D
:103B6000B9888BAB81110C94112882E50E94B98829
:103B700081110C9411280C947B278091A40383FF5E
:103B800002C00C947B2783E50E94B9888BAB81111E
:103B90000C94452982E50E94B98881110C9445292D
:103BA0000C947B270E94C6300C947B2780E50E94F2
:103BB000B988811106C010929F0310929E030C9445
:103BC0007B270E942788672B11F00C947B27F3CF6B
:103BD000109242030C947B2781E0809342030C9463
:103BE0007B270E94CE2F0C947B2783E50E948A8836
:103BF000882311F40C947B270E94578820E030E042
:103C00004AE754E40E94A5990E94BC9E60932E0A44
:103C100070932F0A8093300A9093310A0C947B277B
:103C20002CEFC22E22E0D22E35E2E32E3BE0F32E23
:103C300010E0D6018D916D010E948A88882309F4D5
:103C40006DC0133009F063C00E9457884B015C01BE
:103C500020E030E040EA51E40E94409987FF4EC0E6
:103C6000A50194016091310B7091320B8091330B5F
:103C70009091340B0E944F9E2B013C019B01AC01A3
:103C8000609148047091490480914A0490914B04DA
:103C90000E94A599609348047093490480934A0454
:103CA00090934B04A3019201609180047091810470
:103CB00080918204909183040E94A599609380046E
:103CC0007093810480938204909383046091A5048F
:103CD0007091A6048091A7049091A8040E94449931
:103CE000A30192010E94A5990E94BC9E6093A50425
:103CF0007093A6048093A7049093A8048092310B3C
:103D00009092320BA092330BB092340B07C00E94FA
:103D10005788F70160837183828393831F5FF4E088
:103D2000EF0EF11C143009F084CF0E94E9790C9455
:103D30007B27EBEAF3E084918F010F5F1F4F88230D
:103D400021F00E94D28BF801F6CFEDE9F3E08491E7
:103D50008F010F5F1F4F882321F00E94D28BF80143
:103D6000F6CFE6E8F3E084918F010F5F1F4F8823C1
:103D700021F00E94D28BF801F6CFE6E7F3E08491C0
:103D80008F010F5F1F4F882321F00E94D28BF80113
:103D9000F6CFE5E6F3E084918F010F5F1F4F882394
:103DA00021F00E94D28BF801F6CFE4E5F3E0849194
:103DB0008F010F5F1F4F882321F00E94D28BF801E3
:103DC000F6CFE5E4F3E084918F010F5F1F4F882366
:103DD00021F00E94D28BF801F6CFE0E3F3E084916A
:103DE0008F010F5F1F4F882321F00E94D28BF801B3
:103DF000F6CFEAE1F3E084918F010F5F1F4F882334
:103E000021F00E94D28BF801F6CFE5E0F3E0849137
:103E10008F010F5F1F4F882321F00E94D28BF80182
:103E2000F6CFE8EEF2E084918F010F5F1F4F8823F9
:103E300021F00E94D28BF801F6CFE0EDF2E0849100
:103E40008F010F5F1F4F882311F40C947B270E9472
:103E5000D28BF801F4CF85E40E948A88882381F010
:103E60000E944888882361F0E5ECFCE184918F0191
:103E70000F5F1F4F882321F00E94D28BF801F6CFED
:103E800081E40E948A88882381F00E9448888823E0
:103E900061F0E0EAF4E084918F010F5F1F4F882307
:103EA00021F00E94D28BF801F6CF00913C031091D3
:103EB0003D03D8018D918D018823A9F10E94D28BF9
:103EC000F8CF8AE50E948A88882309F496C70E9461
:103ED00057886B017C0120E030E040E050EC0E940C
:103EE000999F87FD7DC720E030E040EA50E4C7019C
:103EF000B6010E94409918160CF472C7C092010BCB
:103F0000D092020BE092030BF092040BC0922702B6
:103F1000D0922802E0922902F0922A0242E0C701E0
:103F2000B6010E94D64A8AE00E94D28BE4C781E0A3
:103F30008093530324982C9A149AE4EDF4E084912E
:103F40008F010F5F1F4F882321F00E94D28BF80151
:103F5000F6CFECECF4E084918F010F5F1F4F8823C4
:103F600021F00E94D28BF801F6CF1E9B03C000E91E
:103F700012E002C005E912E0F80181918F01882367
:103F800019F00E94D28BF8CF8AE00E94D28BE4EC29
:103F9000F4E084918F010F5F1F4F882321F00E946E
:103FA000D28BF801F6CF379B03C000E912E002C0C4
:103FB00005E912E0D8018D918D01882319F00E9446
:103FC000D28BF8CF8AE00E94D28BECEBF4E08491A4
:103FD0008F010F5F1F4F882321F00E94D28BF801C1
:103FE000F6CF1D9B03C000E912E002C005E912E014
:103FF000F80181918F01882319F00E94D28BF8CFAC
:104000008AE00E94D28BE4EBF4E084918F010F5F91
:104010001F4F882321F00E94D28BF801F6CF029B1C
:1040200003C000E912E002C005E912E0D8018D9159
:104030008D01882319F00E94D28BF8CF8AE00E946C
:10404000D28BECEAF4E084918F010F5F1F4F88233D
:1040500021F00E94D28BF801F6CF1C9B03C000E92F
:1040600012E002C005E912E0F80181918F01882376
:1040700019F00E94D28BF8CF8AE00E94D28BE4EA3A
:10408000F4E084918F010F5F1F4F882321F00E947D
:10409000D28BF801F6CF019B03C000E912E002C009
:1040A00005E912E0D8018D918D01882319F00E9455
:1040B000D28BF8CF8AE00E94D28B10925303249ABD
:1040C0002C98149818C781E0809352038093510371
:1040D00012C710925203109251030DC70E94492E2D
:1040E0000AC70E94BE2D07C783E50E948A888823DD
:1040F00051F00E9457886093540470935504809344
:1041000056049093570484E50E948A88882351F0CE
:104110000E94578860935004709351048093520416
:104120009093530482E40E948A88882351F00E946D
:10413000178860934C0470934D0480934E049093C1
:104140004F0488E50E948A88882351F00E9457888E
:1041500060933C0470933D0480933E0490933F042D
:1041600089E50E948A88882351F00E9457886093CD
:1041700040047093410480934204909343048AE581
:104180000E948A88882351F00E94578860934404D3
:1041900070934504809346049093470485E40E94FD
:1041A0008A88882309F4A7C60E9457886093480428
:1041B0007093490480934A0490934B049CC60E94D8
:1041C0007A2F99C60E941C2D96C68DED90E00E9414
:1041D000855D811190C683E50E94B988882309F422
:1041E0008AC600913E0310E00E942788000F111F2D
:1041F000F801E15EFD4F718360837DC680E50E941A
:104200008A88882309F477C60E942788F62E062F0D
:10421000172F83E50E94B988882321F00E94278800
:104220006B0103C0CC24CA94DC2CC6010196039711
:1042300008F061C617FD5FC60E947472BFEFCB160F
:10424000DB0631F0CA94CD2871F401E010E00DC016
:104250008F2D0E941D8A31E020E0892B09F030E08B
:10426000032F122F02C000E010E08F2D0E941D8A44
:104270008017910709F43FC60E94038EF6CF85E4AC
:104280000E94B988811110C080E50E948A88882325
:1042900091F00E945788609338047093390480939A
:1042A0003A0490933B0407C00E943788882361F347
:1042B000EBECF9E071C089E40E948A88882381F0E0
:1042C0000E9457882CEA35EC47E25EE30E94A599EC
:1042D00060933404709335048093360490933704CC
:1042E00084E40E948A88882381F00E9457882CEAFF
:1042F00035EC47E25EE30E944F9E6093300470937A
:1043000031048093320490933304E5ECFCE1849112
:104310008F010F5F1F4F882321F00E94D28BF8017D
:10432000F6CF409138045091390460913A0470916D
:104330003B0486EF94E00E9422672CEA35EC47E2CA
:104340005EE360913404709135048091360490915D
:1043500037040E944F9EAB01BC0182EF94E00E94A3
:10436000B4382CEA35EC47E25EE36091300470919A
:10437000310480913204909133040E94A599AB01DD
:10438000BC018EEE94E00E94B4388AE00E94D28B89
:10439000B2C50E94D28BF80184918F010F5F1F4F2D
:1043A0008111F7CF0FEA12E0D8018D918D0188239A
:1043B00009F4B9CD0E94D28BF7CF80E50E948A889C
:1043C000882351F00E94578860932C0470932D0429
:1043D00080932E0490932F0489E40E948A88882376
:1043E00081F00E9457882CEA35EC47E25EE30E9498
:1043F000A599609328047093290480932A049093CC
:104400002B0484E40E948A88882381F00E945788C4
:104410002CEA35EC47E25EE30E944F9E6093240451
:10442000709325048093260490932704E5ECFCE127
:1044300084918F010F5F1F4F882321F00E94D28B40
:10444000F801F6CF40912C0450912D0460912E0478
:1044500070912F0482E095E00E9422672CEA35ECEF
:1044600047E25EE3609128047091290480912A0458
:1044700090912B040E944F9EAB01BC018EEF94E003
:104480000E94B4382CEA35EC47E25EE360912404E4
:104490007091250480912604909127040E94A5998B
:1044A000AB01BC018AEF94E00E94B4388AE00E941C
:1044B000D28B21C583E50E948A88182F882371F04A
:1044C0000E9457880E94B79E70931E0260931D023F
:1044D00021E0672B09F020E02093980380E50E94FB
:1044E0008A88882359F020911D0230911E02232BC7
:1044F00011F00E94488880939803FDC41111FBC4F9
:10450000E5ECFCE184918F010F5F1F4F882321F0C0
:104510000E94D28BF801F6CF80919803811103C0DD
:104520006FE972E002C062E972E08BE195E00E94FF
:104530007F6760911D0270911E028AE095E00E94E3
:104540006667E6E0F5E084918F010F5F1F4F8823D7
:1045500009F4D1C40E94D28BF801F5CF85E40E9402
:10456000B988882321F00E9427881B0102C0212CD2
:10457000312C83E40E94B988882339F00E9427886F
:10458000E0967FAF6EAFE09706C0E5E0F0E0E09622
:10459000FFAFEEAFE09785E50E948A88A5968FAFC2
:1045A000A597882329F00E944888A5968FAFA597E4
:1045B00037FC07C0C12CD12CB6E1EB2EB3E4FB2EA7
:1045C00006C0C12CD12CACE8EA2EA2E4FA2E83E579
:1045D0000E94B988882321F00E9457886B017C01D2
:1045E0002114310411F410923E030E94728B2B01AE
:1045F0003C01C1010196029718F400EC12E00BC0D7
:1046000003ED12E0D8018D918D01882309F48BCC44
:104610000E94D28BF7CFF80181918F01882319F086
:104620000E94D28BF8CF8AE00E94D28B0E946662F1
:104630008FE7FFEF2F163F0619F480930F0402C097
:1046400080931104C701B6010E94B79E072E000C8B
:10465000880B990B0E94469924966FAF2497289651
:104660007FAF28972C968FAF2C9768969FAF68974F
:1046700081E080935302AA964CAE5DAE6EAE7FAEE3
:10468000AA97E4964CAE5DAE6EAE7FAEE4976C96A4
:104690001FAE6C9720E460962FAF60973CE1649664
:1046A0003FAF649746E4A0964FAFA097A1961FAE88
:1046B000A197A2961FAEA297A3961FAEA397A4960A
:1046C0001FAEA49723961CAE1DAE1EAE1FAE239741
:1046D0001BAE1CAE1DAE1EAEC12CD12C7601FFE769
:1046E0008F2E912CA12CB12C8FE790E0A0E0B0E0B0
:1046F0008FA798ABA9ABBAABAE961CAE1DAE1EAEE3
:104700001FAEAE9791E0A6969FAFA69718AE1FAAD0
:104710001FA21BA600E010E080915302882309F439
:104720001CC20E94728B6BAB7CAB8DAB9EAB80913D
:10473000FF03882309F4E4C00E941F63AFEF2A1629
:104740003A0659F4B091F303BFA3E091F403EBA749
:104750000091F5031091F6030AC0F0911304FFA332
:10476000209114042BA700911504109116042FA179
:104770003BA5A801A1966FADA197A2967FADA29788
:10478000A3968FADA397A4969FADA4970E9440993E
:1047900087FF0EC03FA1A1963FAFA1974BA5A29660
:1047A0004FAFA297A3960FAFA397A4961FAFA4975E
:1047B0002FA13BA5A8016C966FAD6C9760967FAD5D
:1047C000609764968FAD6497A0969FADA0970E9466
:1047D000999F181674F45FA16C965FAF6C978BA5C8
:1047E00060968FAF609764960FAF6497A0961FAFE7
:1047F000A097A6969FADA69724962FAD24972896AE
:104800003FAD28972C964FAD2C9768965FAD689773
:104810006FA17BA5802F992309F457C0912F0E9487
:10482000999F18160CF06CC04BA95CA96DA97EA9C4
:104830004419550966097709DB01CA018858934173
:10484000A109B109B7FD5CC08FA598A9A9A9BAA90A
:1048500088199909AA09BB09B595A79597958795D0
:10486000EFEF2E163E0619F480930F0402C08093DA
:104870001104AE964CAF5DAF6EAF7FAFAE9724968E
:10488000FFAD2497A196FFAFA19728962FAD28974B
:10489000A2962FAFA2972C963FAD2C97A3963FAF31
:1048A000A39768964FAD6897A4964FAFA4978BA92E
:1048B0009CA9ADA9BEA9AA968CAF9DAFAEAFBFAF64
:1048C000AA97A6961FAEA6971BC0912F0E9440994B
:1048D00087FF16C08BA99CA9ADA9BEA9AA962CAD2D
:1048E0003DAD4EAD5FADAA97821B930BA40BB50BEC
:1048F000AC01BD01485853416109710977FFFDC5FD
:1049000020E030E040EA51E424966FAD24972896E9
:104910007FAD28972C968FAD2C9768969FAD6897A2
:104920000E94739D9B01AC016FA17BA5C8010E94F1
:10493000999F18166CF4EBEEF5E084918F010F5FF0
:104940001F4F882309F4D7C20E94D28BF801F5CFFC
:1049500080E398EFAFEFBFEFE4962CAD3DAD4EADE9
:104960005FADE497821B930BA40BB50B2BA93CA95D
:104970004DA95EA9820F931FA41FB51FB7FD0FC0DD
:104980000E94E7308AE00E94D28B8BA99CA9ADA936
:10499000BEA9E4968CAF9DAFAEAFBFAFE4978BA935
:1049A0009CA9ADA9BEA9880F991FAA1FBB1FAA96D3
:1049B0002CAD3DAD4EAD5FADAA97821B930BA40B02
:1049C000B50B84199509A609B70981389F44A241FE
:1049D000B10568F0EDECF5E084918F010F5F1F4F9A
:1049E000882309F488C20E94D28BF801F5CF4FA921
:1049F00058ADE0968EAD9FADE097841795070CF00B
:104A00008BCEE0E7F5E084918F010F5F1F4F882385
:104A100021F00E94D28BF801F6CF9FEF29163906BC
:104A200019F008E113E002C003EA12E0B8018EE5D4
:104A300095E00E947F67B701A6018AE595E00E9494
:104A400022678AE00E94D28BB80188E495E00E9438
:104A50007F674BAD5CAD6DAD7EAD84E495E00E94AB
:104A600022678AE00E94D28BB80182E395E00E941F
:104A70007F6723964CAD5DAD6EAD7FAD23978EE223
:104A800095E00E9422678AE00E94D28BA596AFAC87
:104A9000A597AA2009F42FC22320209479F5C0926B
:104AA0002C04D0922D04E0922E04F0922F042CEAD4
:104AB00035EC47E25EE36BAD7CAD8DAD9EAD0E9403
:104AC000A599609328047093290480932A049093F5
:104AD0002B042CEA35EC47E25EE323966CAD7DAD0A
:104AE0008EAD9FAD23970E944F9E609324047093D8
:104AF00025048093260490932704FDC1C0923804B6
:104B0000D0923904E0923A04F0923B042CEA35EC5E
:104B100047E25EE36BAD7CAD8DAD9EAD0E94A59985
:104B20006093340470933504809336049093370473
:104B30002CEA35EC47E25EE323966CAD7DAD8EAD9D
:104B40009FAD23970E944F9E609330047093310471
:104B50008093320490933304CEC18091530281112B
:104B6000CAC10E946662C7C10E947472C4C181E05A
:104B70000E94424EC0C180E00E94424EBCC186E508
:104B80000E948A88882321F08CE896E00E94009495
:104B900083E50E948A88182F882319F00E9448888C
:104BA000182F83E50E948A88882319F0812F0E949C
:104BB000E64CF0901704111103C0E5ECFCE11AC0BB
:104BC000F110FBCFEBECF9E084918F010F5F1F4FE9
:104BD000882321F00E94D28BF801F6CFEDE6F6E0B3
:104BE00084918F010F5F1F4F882339F30E94D28B6E
:104BF000F801F6CF84918F010F5F1F4F882321F0BA
:104C00000E94D28BF801F6CFF11003C06BEA72E07C
:104C100002C067EA72E08FE596E00E947F678AE053
:104C20000E94D28B68C184E5C82E83E0D82E95E11E
:104C3000E92E9BE0F92E25E3222E2BE0322E00E018
:104C400010E0A22CA094AFA2D1018D911D01882368
:104C500009F48BC0F7014080518062807380F801B5
:104C6000ED5BFD4F2081318142815381F801EE5F80
:104C7000FD4F60817181828193810E94739D20E04C
:104C800030E040E05FE30E94A5999B01AC01C301C5
:104C9000B2010E94999F181644F4F801EA5FF34E9E
:104CA00085909590A590B49003C0812C912C5401CF
:104CB000F801E457FC4F2081318142815381C301C7
:104CC000B2010E94729D9B01AC01C501B4010E941A
:104CD000729D4B015C0120E030E040EA51EC0E9403
:104CE000999F87FD29C020E030E040EA51E4C501EA
:104CF000B4010E9440991816FCF0D6012D913D9107
:104D00004D915C91C501B4010E94729D9B01AC0163
:104D1000C301B2010E94739DF70160837183828396
:104D20009383D6018D929D92AD92BC9213978FA1E1
:104D3000820D0E942E5D19C0EBECF9E084918F0189
:104D40000F5F1F4F882321F00E94D28BF801F6CF0E
:104D5000E9EAF6E084918F010F5F1F4F882309F481
:104D6000CAC00E94D28BF801F5CFB4E0CB0ED11CA3
:104D70000C5F1F4FE4E0EE0EF11C0C30110509F042
:104D800063CF0E94D087F7D7B6C00E94C27BB3C062
:104D90000E945B7AB0C083E50E948A88882319F05C
:104DA0000E94488801C081E091E089270E946A6DD5
:104DB000A2C084918F010F5F1F4F882321F00E94B2
:104DC000D28BF801F6CFEFEDF6E084918F010F5F03
:104DD0001F4F882309F475C80E94D28BF801F5CFC4
:104DE000EAECF6E084918F010F5F1F4F882309F4EE
:104DF0009AC80E94D28BF801F5CF4091010B5091D7
:104E0000020B6091030B7091040B87EC96E00E94FB
:104E1000226789C8D3D56FC054D56DC037D56BC054
:104E200081E08093210283E50E948A88811103C07A
:104E30000E94DC9460C00E94488881115CC0F8CF59
:104E4000F0904403FF2021F1E5ECFCE184918F0117
:104E50000F5F1F4F882321F00E94D28BF801F6CFFD
:104E600084E50E94D28B6F2D70E080E090E04AE0F4
:104E70000E942B8C80E20E94D28B0FEA12E0D801B4
:104E80008D918D01882309F44EC80E94D28BF7CFF3
:104E900010928203E5ECFCE184918F010F5F1F4FBC
:104EA000882321F00E94D28BF801F6CF6091820313
:104EB00070E089EE96E00E9466678AE00E94D28BDD
:104EC0001AC0E5ECFCE184918F010F5F1F4F88232E
:104ED00021F00E94D28BF801F6CF6091280A7091E0
:104EE000290A8BEF96E00E947F6782E20E94D28BB4
:104EF0008AE00E94D28B0E946E9476C441155105BF
:104F000019F4AF0141505109812C912C0C942010BF
:104F100080E00E94E64C0E94404D83E50E948A8812
:104F2000882309F448C00E94488821E0482FBE0128
:104F30006F5F7F4FCE0146960E9493316B017C01DB
:104F40009B01AC010E941FA0811131C02CEA35ECFD
:104F500047E257E36E897F89888D998D0E94739D02
:104F6000AB01BC018DE392E00E94B4382CEA35EC31
:104F700047E257E369817A818B819C810E94739D0E
:104F8000AB01BC0188E392E00E94B4382CEA35EC16
:104F900047E257E3C701B6010E94739DAB01BC0114
:104FA00083E392E00E94B4388AE00E94D28B0E9490
:104FB000264DE1D6A0CF81E0B8CFD7018C918823D0
:104FC00011F40C94A71BE5ECFCE184918F010F5FB9
:104FD0001F4F882321F00E94D28BF801F6CFF701F2
:104FE00081917F01882319F00E94D28BF8CF8AE04B
:104FF0000E94D28B0C94A71B802F0E943E916E2D95
:10500000802F0E94458AF12CB701802F0E94748A5C
:105010000830110509F06FCFF0929F03E0929E03D4
:105020006ACF0E9457880E94B79E7093FC036093DA
:10503000FB0380E00E941B620E94578820E030E062
:1050400040E752E40E94409918161CF00E945D91BE
:1050500002C00E944B9381E0809353021BA61CA6C2
:105060001DA61EA61FA618AA19AA1AAA1FA21FAA21
:10507000ECE3EBAFFCE1FFAF26E424962FAF2497DF
:10508000C12CD12C60E8E62E7FEBF72E812C912CE1
:1050900054016091FB037091FC03072E000C880BF8
:1050A000990B0E944699162F072F782E692E262FCE
:1050B000372F482F592FB601C7010E9440998823E6
:1050C000D1F02091130430911404409115045091B3
:1050D0001604612F702F872D962D0E944099881FEE
:1050E0008827881F8FA33BA9332349F0882339F0F1
:1050F0008091530200CF1C2D0D2D7E2C6F2C0E9411
:10510000728B6B017C01DC01CB012FA538A949A969
:105110005AA9821B930BA40BB50BB7FD3BC0D7015B
:10512000C60188519C4FAF4FBF4F8FA798ABA9AB1B
:10513000BAAB0E94E730E8ECF2E084912F019FEFD8
:10514000491A590A882321F00E94D28BF201F5CF27
:1051500081149104A104B104B9F0D501C4018851AE
:105160009C4FAF4FBF4FBC01CD016C197D098E091B
:105170009F0928EE33E040E050E00E941B9DCA01E9
:10518000B9010E94BA4A03C08FE30E94D28B8AE021
:105190000E94D28B0E94038E0E947E8B209013046B
:1051A0003090140440901504509016049101A2010F
:1051B000612F702F872D962D0E94729D9F7720E082
:1051C00030E040E251E481149104A104B10429F4D7
:1051D0000E94409987FF07C004C00E94999F18163B
:1051E00014F446015701AFA1AA2399F12BA53CA5C0
:1051F0004DA55EA5211531054105510541F0D701A9
:10520000C601821B930BA40BB50BB7FD22C0910105
:10521000A2016FA97BAD8FAD24969FAD24970E940C
:10522000729D20E030E040EC5FE30E94409987FDF2
:105230005FCFD701C601805A9541AF4FBF4F8BA7B3
:105240009CA7ADA7BEA72FAA3BAE4FAE24965FAEDC
:10525000249780915302882309F44ACF8114910442
:10526000A104B10429F4C12ED02EE72CF62C11CFC5
:1052700098EEC91A93E0D90AE108F108C818D908CC
:10528000EA08FB08F7FE34CFEECF0E9457880E9451
:10529000B79E6739710514F066E970E07093F80302
:1052A0006093F7030E94D0610E94578820E030E0AD
:1052B00040EA50E40E94999F181614F40E944B9300
:1052C00081E0809353028091820380933E031BA66A
:1052D0001CA61DA61EA61FA618AA19AA1AAA1FA2B6
:1052E0001FAAACE3ABAFBCE1BFAFE6E42496EFAFDF
:1052F0002497C12CD12C40E8E42E5FEBF52E812CB5
:10530000912C54016091F7037091F803072E000C63
:10531000880B990B0E944699162F072F782E692E1D
:10532000262F372F482F592FB601C7010E944099C9
:105330008823D1F02091F3033091F4034091F503D9
:105340005091F603612F702F872D962D0E94409962
:10535000881F8827881F8FA3FBA9FF2349F0882374
:1053600039F080915302C7CD1C2D0D2D7E2C6F2C52
:105370000E94728B6B017C01DC01CB012FA538A947
:1053800049A95AA9821B930BA40BB50BB7FD3AC0D0
:10539000D701C60188519C4FAF4FBF4F8FA798AB25
:1053A000A9ABBAAB14D7ECECF2E084912F019FEFDC
:1053B000491A590A882321F00E94D28BF201F5CFB5
:1053C00081149104A104B104B9F0D501C40188513C
:1053D0009C4FAF4FBF4FBC01CD016C197D098E09A9
:1053E0009F0928EE33E040E050E00E941B9DCA0177
:1053F000B9010E94BA4A03C08FE30E94D28B8AE0AF
:105400000E94D28B0E94038E0E947E8B2090F30319
:105410003090F4034090F5035090F6039101A201FF
:10542000612F702F872D962D0E94729D9F7720E00F
:1054300030E040EA50E481149104A104B10429F45D
:105440000E94409987FF07C004C00E94999F1816C8
:1054500014F446015701AFA1AA2399F12BA53CA54D
:105460004DA55EA5211531054105510541F0D70136
:10547000C601821B930BA40BB50BB7FD22C0910193
:10548000A2016FA97BAD8FAD24969FAD24970E949A
:10549000729D20E030E040EC5FE30E94409987FD80
:1054A00060CFD701C601805A9541AF4FBF4F8BA740
:1054B0009CA7ADA7BEA72FAA3BAE4FAE24965FAE6A
:1054C000249780915302882309F44BCF81149104CF
:1054D000A104B10429F4C12ED02EE72CF62C12CF52
:1054E00098EEC91A93E0D90AE108F108C818D9085A
:1054F000EA08FB08F7FE35CFEECF4FA958AD1416DA
:1055000015060CF035C1AE964CAC5DAC6EAC7FAC04
:10551000AE97480E591E6A1E7B1EAE962CAD3DAD51
:105520004EAD5FADAE97281B390B4A0B5B0BCA0122
:10553000B901A50194010E940C9DA30192010E9452
:105540003D9D8FA498A8A9A8BAA8820E931EA41E58
:10555000B51E34E183169104A104B1040CF14CEEA4
:1055600084169104A104B1043CF450E8851691041A
:10557000A104B1041CF105C06BEE862E912CA12C68
:10558000B12C8FA698AAA9AABAAA8EEF90E0A0E0A3
:10559000B0E088199909AA09BB094C015D0112C044
:1055A00024E130E040E050E02FA738AB49AB5AABE4
:1055B00054E1852E912CA12CB12C04C08FA698AA61
:1055C000A9AABAAA4FA558A969A97AA987E596E018
:1055D0000E943F67B501A40182E596E00E943F6703
:1055E0006C964FAD6C9760965FAD609764966FADAB
:1055F0006497A0967FADA0978BE496E00E94226707
:10560000A1964FADA197A2965FADA297A3966FAD5D
:10561000A397A4967FADA49784E496E00E942267A6
:105620004FA958AD433051050CF4A2C0C501B401D7
:105630000E94469920E030E040E850E40E94A5999D
:105640006B017C016C962FAD6C9760963FAD6097B7
:1056500064964FAD6497A0965FADA097A1966FAD8D
:10566000A197A2967FADA297A3968FADA397A4967C
:105670009FADA4970E94729D2BED3FE049E450E45A
:105680000E94A59920E030E040E05FE30E94A599E8
:105690009B01AC01C701B6010E944F9E6B017C01CA
:1056A000C301B2010E9446992FE632E143E85AE372
:1056B0000E94A5992B013C01B701A6018EE396E05B
:1056C0000E942267B301A20188E396E00E9422674C
:1056D0002AE939E949E15FE3C701B6010E94A599CA
:1056E0006B017C019B01AC010E94739DA30192019F
:1056F0000E944F9E6BAF7CAF8DAF9EAFA301920116
:10570000C701B6010E94A59920E030E040E05EE3C9
:105710000E94A59923966CAF7DAF8EAF9FAF239764
:10572000E8E2F6E084913F015FEF651A750A88238D
:1057300021F00E94D28BF301F5CFB701A60182E2DE
:1057400096E00E9422674BAD5CAD6DAD7EAD8CE105
:1057500096E00E94226723964CAD5DAD6EAD7FADA5
:10576000239786E196E00E9422678AE00E94D28B0E
:105770008FA598A9A9A9BAA9880D991DAA1DBB1D15
:10578000B595A79597958795EFEF2E163E0619F4D8
:1057900080930F0402C0809311042FA938AD2F5FAE
:1057A0003F4F38AF2FAB24963FAD24976C963FAF59
:1057B0006C9728964FAD289760964FAF60972C96C0
:1057C0005FAD2C9764965FAF649768968FAD6897CE
:1057D000A0968FAFA0974BA85CA86DA87EA891E07B
:1057E000A6969FAFA6978CC8CD58DF4F0FB6F894FA
:1057F000DEBF0FBECDBFDF91CF911F910F91FF9004
:10580000EF90DF90CF90BF90AF909F908F907F9060
:105810006F905F904F903F902F900895EF92FF927E
:105820000F931F93CF93DF931F92CDB7DEB78C01F9
:105830007B0180E249830E94D28B49814F3F11F066
:1058400084E501C082E40E94D28B8AE30E94D28B5D
:10585000F801608171818281938142E00E94D64A81
:10586000F701408151816281738184E397E00E9456
:10587000226762E070E080E090E00F90DF91CF91CE
:105880001F910F91FF90EF900C943A8BCF93DF9381
:10589000EBECF9E08491EF012196882321F00E943E
:1058A000D28BFE01F7CFE0E3F8E08491EF0121967F
:1058B000882321F00E94D28BFE01F7CFDF91CF9198
:1058C00008950F931F93CF9383E50E94B98888238F
:1058D000C1F10E943788813031F0823091F50CEFB0
:1058E00012E0C0E01FC00CEF12E0C0E0F8018191AF
:1058F0008F010E94B988882339F00E9437884FEFC2
:10590000682F8C2F0E946471CF5FC43079F782E4D6
:105910000E94B9888823A9F00E94378812C0CF5FFF
:10592000C430A9F3F80181918F010E94B9888823BE
:10593000B1F30E943788482F6FEF8C2F0E9464715B
:10594000EECFCF911F910F910C9473660F931F931D
:10595000CF9383E50E948A88811104C00CEF12E086
:10596000C0E00EC0C0E00E943788682F8C2F0E94D4
:105970000A67CF5FC530B9F7F1CFCF5FC43071F0A0
:10598000F80181918F010E948A888823B1F30E94D7
:105990003788682F8C2F0E940A67EFCF82E40E941D
:1059A0008A88882331F00E943788682F84E00E941B
:1059B0000A67CF911F910F910C9473660F931F93F9
:1059C00088E50E948A888823F1F00E9427888B014D
:1059D000072E000C220B330B0093180410931904AC
:1059E00020931A0430931B04DB012FEF30E00E9458
:1059F0006AA020ED37E040E050E00E943D9DB901F3
:105A00008EE20E94748A8AE50E948A88882329F09F
:105A10000E94278881E00E94E37185E40E948A88C1
:105A2000882339F00E94278882E01F910F910C94FF
:105A3000E3711F910F91089583E50E94B98888232F
:105A400031F00E942788709301026093000208954C
:105A5000CF93DF93E5ECFCE18491EF01219688235D
:105A600021F00E94D28BFE01F7CF83E50E948A8845
:105A7000882321F00E94488880931802E0E2F8E031
:105A80008491EF012196882321F00E94D28BFE01A0
:105A9000F7CF80911802811103C0ECE1F8E002C059
:105AA000E8E1F8E08491EF012196882321F00E943B
:105AB000D28BFE01F7CFE0E1F8E08491EF0121966F
:105AC000882321F00E94D28BFE01F7CF4091020281
:105AD0005091030260910402709105028EE098E0FB
:105AE0000E942267409106025091070260910802CD
:105AF000709109028BE098E00E94226740910A02AF
:105B000050910B0260910C0270910D0288E098E0B8
:105B10000E942267E0E0F8E08491EF01219688235B
:105B200021F00E94D28BFE01F7CF409143025091A9
:105B3000440260914502709146028EEF97E00E9408
:105B4000226740914702509148026091490270914A
:105B50004A028BEF97E00E94226740914B025091DE
:105B60004C0260914D0270914E0288EF97E00E94C6
:105B700022678AE0DF91CF910C94D28B83E50E945B
:105B80008A888823D9F00E945788AB01BC014093D2
:105B900060045093610460936204709363044093C3
:105BA00058045093590460935A0470935B0480ED39
:105BB00097E00E9422678AE00E94D28B80E50E94D3
:105BC0008A88882399F00E945788AB01BC014093D2
:105BD000600450936104609362047093630483EBE8
:105BE00097E00E9422678AE00E94D28B82E50E94A1
:105BF0008A88882399F00E945788AB01BC014093A2
:105C00005C0450935D0460935E0470935F0484E9C8
:105C100097E00E9422678AE00E94D28B84E50E946E
:105C20008A88882399F00E945788AB01BC01409371
:105C300058045093590460935A0470935B0486E7A8
:105C400097E00E9422678AE00C94D28B0895FF921D
:105C50000F931F93CF93DF9304E714E0CCEFD2E0D0
:105C6000FC2E84E0F80E89910E948A88882339F0FE
:105C70000E945788F80160837183828393830C5F4D
:105C80001F4FFC12F0CFDF91CF911F910F91FF902A
:105C90000895FF920F931F93CF93DF9304E614E0D0
:105CA000CCEFD2E0FC2E84E0F80E89910E948A8825
:105CB000882349F00E9457880E94BC9EF8016083A7
:105CC0007183828393830C5F1F4FFC12EECFDF91B1
:105CD000CF911F910F91FF900C947F79CF93DF9319
:105CE00088EC90E00E94855D811142C084E40E94AE
:105CF0008A888823C9F10E945788C1E020E030E0FB
:105D0000A9010E944099811101C0C0E0C09388049C
:105D1000CC2351F1C0913E03D0E00E945788CC0FB4
:105D2000DD1FCC0FDD1FCC57DB4F688379838A835F
:105D30009B8320E030E0A901609184047091850488
:105D400080918604909187040E94409981110CC033
:105D500080E090E0A0E4B0E4809384049093850414
:105D6000A0938604B0938704DF91CF910C94738F36
:105D7000DF91CF9108954F925F926F927F928F92B1
:105D80009F92AF92BF92CF92DF92EF92FF92CF930A
:105D9000DF93E3E7F7E08491EF012196882321F078
:105DA0000E94D28BFE01F7CF6091150B7091160BFC
:105DB0008091170B9091180B42E00E94D64AEFE6B3
:105DC000F7E08491EF012196882321F00E94D28B85
:105DD000FE01F7CF6091190B70911A0B80911B0B8C
:105DE00090911C0B42E00E94D64AEBE6F7E08491CA
:105DF000EF012196882321F00E94D28BFE01F7CF7C
:105E000060911D0B70911E0B80911F0B9091200BC8
:105E100042E00E94D64AE7E6F7E08491EF0121963E
:105E2000882321F00E94D28BFE01F7CF6091210BD5
:105E30007091220B8091230B9091240B42E00E94E1
:105E4000D64A8FB7F8944090050B5090060B60909F
:105E5000070B7090080B8090090B90900A0BA09094
:105E60000B0BB0900C0BC0900D0BD0900E0BE09074
:105E70000F0BF090100B8FBFEDE5F7E08491EF0171
:105E80002196882321F00E94D28BFE01F7CFC30117
:105E9000B2010E94BA4AE9E5F7E08491EF01219648
:105EA000882321F00E94D28BFE01F7CFC501B401F7
:105EB0000E94BA4AE5E5F7E08491EF012196882334
:105EC00021F00E94D28BFE01F7CFC701B6010E94DC
:105ED000BA4A8AE0DF91CF91FF90EF90DF90CF90A8
:105EE000BF90AF909F908F907F906F905F904F90FA
:105EF0000C94D28B8F929F92AF92BF92CF92DF92EF
:105F0000EF92FF920F931F93CF938CEFC82E82E0F6
:105F1000D82E95E1E92E9BE0F92E04E513E0C0E0D0
:105F2000F60181916F010E948A88882309F10E94FD
:105F300057884B015C01F8012081318142815381F6
:105F40000E94729D9B01AC01F70160817181828189
:105F500093810E94739DF701608371838283938391
:105F6000F80180829182A282B3828C2F0E942E5DE2
:105F7000CF5FF4E0EF0EF11C0C5F1F4FC33081F6D2
:105F80000E94D087CF911F910F91FF90EF90DF90EB
:105F9000CF90BF90AF909F908F90EDCE83E50E9401
:105FA000B988882399F00E94578820E030E04AE7BA
:105FB00054E40E94A5990E94BC9E60934F02709386
:105FC00050028093510290935202089588E50E94F6
:105FD0008A88811113C089E50E948A8881110EC0C8
:105FE0008AE50E948A88811109C085E40E948A8816
:105FF000811104C00E9474720C94CB8D0E94747243
:1060000088E50E948A88882319F0179A10924E0317
:1060100089E50E948A88882319F0169A10924F0306
:106020008AE50E948A88882319F0159A10925003F5
:1060300085E40E948A88882311F0149A08950895AF
:10604000CF93DF930E9466620E9474720E94CB8D90
:1060500010929F0310929E03C0E0D0E062E370E0D4
:1060600080E090E00E943A8B0E9423652196C33124
:10607000D105A1F762E370E080E090E00E943A8BE6
:10608000DF91CF910C942365DF92EF92FF920F93F3
:106090001F93CF93DF9383E50E94B988882319F07B
:1060A0000E94378801C080E08093A403E5ECFCE106
:1060B0008491EF012196882321F00E94D28BFE016A
:1060C000F7CFEEE4F7E08491EF012196882321F0E9
:1060D0000E94D28BFE01F7CF8091A403882389F11F
:1060E00080E4E82E87E0F82E00E010E020E08091C8
:1060F000A40390E0002E02C0959587950A94E2F7DC
:1061000080FF16C0DD24D394D20E222319F08CE236
:106110000E94D28BF70125913491F9018491E90114
:106120002196882321F00E94D28B9E01F6CF2D2D3F
:106130000F5F1F4FF2E0EF0EF11C05301105B9F6AD
:106140000BC0EAE4F7E08491EF012196882321F067
:106150000E94D28BFE01F7CF8AE0DF91CF911F9191
:106160000F91FF90EF90DF900C94D28B8EE40E9401
:10617000B988882351F00E9427886093970B709309
:10618000980B8093990B90939A0B0895CF93DF937C
:1061900083E50E94B988882339F00E942788EB01A3
:1061A0006F3F710519F010F0CFEFD0E080E50E944D
:1061B000B988811105C0D0939F03C0939E0304C08A
:1061C0000E9437888823B9F3DF91CF9108950F9308
:1061D0001F93CF93DF93CDB7DEB728970FB6F89410
:1061E000DEBF0FBECDBF6091FB037091FC03072E95
:1061F000000C880B990B0E9446996D837E838F83D8
:1062000098878091130490911404A0911504B09183
:10621000160489839A83AB83BC834EEFBE016B5F08
:106220007F4FCE010196FADA6091F7037091F8037F
:10623000072E000C880B990B0E9446996D837E8374
:106240008F8398878091F3039091F403A091F503D5
:10625000B091F60389839A83AB83BC834FEFBE0171
:106260006B5F7F4FCE010196D9DAECE3F7E08491C2
:106270008F010F5F1F4F882321F00E94D28BF801FE
:10628000F6CFE0913E03F0E0EF5EFB4F608170E0FF
:1062900080E090E00E94BA4AE7E3F7E084918F0142
:1062A0000F5F1F4F882321F00E94D28BF801F6CF99
:1062B00060910F0470E080E090E00E94BA4A289656
:1062C0000FB6F894DEBF0FBECDBFDF91CF911F9107
:1062D0000F91089588E690E00E94855D811122C0AB
:1062E0008091A40383FD1EC083E50E94B9888823A2
:1062F000C9F00E9457880E94B79E7093FC03609378
:10630000FB0380E00E941B620E94578820E030E07F
:1063100040E752E40E944099181614F00E945D91E3
:106320000C94578808952F923F924F925F926F92EC
:106330007F928F929F92AF92BF92CF92DF92EF9215
:10634000FF920F931F93CF93DF93CDB7DEB76B9779
:106350000FB6F894DEBF0FBECDBF9F8B8E8B1B0197
:10636000488F298FFC016081718182819381698BC3
:106370007A8B8B8B9C8BF101C080D180E280F38083
:10638000CD86DE86EF86F88A409090035090910388
:10639000609092037090930320918C0330918D0351
:1063A00040918E0350918F030E94729D4B015C01BE
:1063B00022E630E140E450EC0E94999F87FD24C022
:1063C00022E430E042E253E4C501B4010E94409966
:1063D0001816D4F0A3019201C701B6010E94729D64
:1063E0006B017C0121E338E040EE50EC0E94999F64
:1063F00087FD0AC022E430E04EE353E4C701B60152
:106400000E94409918162CF4A12CB12C00EC1FE727
:1064100099C2C0901902D0901A02E0901B02F0902D
:106420001C0280918403811107C08091180280931F
:10643000830381E08093840380911402909115027C
:10644000A0911602B09117028093190290931A023C
:10645000A0931B02B0931C020E94F19219821A822F
:106460001B821C82AE014F5F5F4FBE01635F7F4F97
:10647000CE0141960E94BC5C81E00E94424E811197
:10648000EBC10E947E8B04E010E0812C912CA12CAA
:1064900041E4B42E412C512C50E2652E51E4752E6E
:1064A00060E070E080EF93E40E94B093882309F4E9
:1064B000ABC00150110909F072C0E8E9F9E084911C
:1064C0008F010F5F1F4F882321F00E94D28BF801AC
:1064D000F6CF80E090E0A0E0B1E48D839E83AF83AF
:1064E000B88780E090E0A8ECB2E489839A83AB831C
:1064F000BC83BE016B5F7F4FCE0101960E94C15CE1
:106500001092210B1092220B1092230B1092240B4D
:10651000C090820380911D0B90911E0BA0911F0BC8
:10652000B091200B4091190B50911A0B60911B0BED
:1065300070911C0B0091150B1091160B2091170BED
:106540003091180B09831A832B833C834D835E8320
:106550006F83788789879A87AB87BC87AE01475F4F
:106560005F4FBE016B5F7F4FCE0101960E94E649EF
:10657000E12CF12C00EA1FE321E23BE0AE01475F92
:106580005F4FBE016B5F7F4FCE0101960E94DE3BE5
:106590000E94B4920E94747289E899E0CAC0E1EB4B
:1065A000F9E084919F012F5F3F4F882341F02A8FAC
:1065B0003B8F0E94D28B2A8D3B8DF901F2CF8D82C9
:1065C0009E82AF82B88649825A826B827C82BE01EB
:1065D0006B5F7F4FCE0101960E94C15C1D8A1982BC
:1065E0001A821B821C82FCE0F9871D829E012B5EB1
:1065F0003F4FAE014F5F5F4FBE01675F7F4FCE01E0
:1066000005960E94A7674CCF80E090E0A0E0B1E43F
:106610008D839E83AF83B88720E030E040EA50E46A
:1066200060911D0B70911E0B80911F0B9091200BA0
:106630000E94739D69837A838B839C83BE016B5F09
:106640007F4FCE0101960E94C15C04E010E0812CD6
:10665000912C90E8A92E9FE3B92E412C512C20E2D9
:10666000622E21E4722E8BC080E090E0A0E0B1E4C5
:106670008D839E83AF83B88780E090E0A8ECB2E47E
:1066800089839A83AB83BC83BE016B5F7F4FCE014E
:1066900001960E94C15C1092210B1092220B109265
:1066A000230B1092240BC090820380911D0B9091BC
:1066B0001E0BA0911F0BB091200B4091190B509114
:1066C0001A0B60911B0B70911C0B0091150B109114
:1066D000160B2091170B3091180B09831A832B830B
:1066E0003C834D835E836F83788789879A87AB87E6
:1066F000BC87AE01475F5F4FBE016B5F7F4FCE012E
:1067000001960E94E649E12CF12C00EA1FE321E208
:106710003BE0AE01475F5F4FBE016B5F7F4FCE0135
:1067200001960E94DE3B0E94B4920E94747287E53B
:1067300099E00E94D58D8D829E82AF82B886498273
:106740005A826B827C82BE016B5F7F4FCE010196C5
:106750000E94C15C1D8A19821A821B821C828CE0F5
:1067600089871D829E012B5E3F4FAE014F5F5F4FB9
:10677000BE01675F7F4FCE0105960E94A76760E06C
:1067800070E080E792E40E94B093882309F1015001
:10679000110969F4E6E6F9E084918F010F5F1F4F5C
:1067A000882309F461CF0E94D28BF801F5CFEFE77F
:1067B000F9E084919F012F5F3F4F882309F4BBCFFD
:1067C0002A8F3B8F0E94D28B2A8D3B8DF901F1CF0E
:1067D00040901D0B50901E0B60901F0B7090200B73
:1067E0002091940330919503409196035091970323
:1067F000C301B2010E94729D2091010B3091020BE6
:106800004091030B5091040B0E94739D5B018C011E
:10681000988D91111CC080E090E0A0E0B1E48983E4
:106820009A83AB83BC8320E030E040EA50E4C301AC
:10683000B2010E94739D6D837E838F839887BE0112
:106840006F5F7F4FCE0105960E94C15C09C080E05A
:106850000E94424E882321F0A12CB12C00EC1FE7AE
:106860008091830380931802E98DE33008F440C0DF
:10687000ECEDF9E084914F019FEF891A990A882382
:1068800021F00E94D28BF401F5CFEE89FF8960815F
:1068900071818281938143E00E94D64AE7EDF9E05D
:1068A00084914F019FEF891A990A882321F00E9451
:1068B000D28BF401F5CFF1016081718182819381E6
:1068C00043E00E94D64AE2EDF9E084914F019FEF48
:1068D000891A990A882321F00E94D28BF401F5CFFE
:1068E00043E0B501C8010E94D64A8AE00E94D28BDB
:1068F000C0921902D0921A02E0921B02F0921C027E
:106900009501A801B501C8010E941FA08823D1F0FC
:10691000EBECF9E084917F019FEFE91AF90A8823F3
:1069200021F00E94D28BF701F5CFEBEBF9E08491D7
:106930007F019FEFE91AF90A882321F00E94D28B88
:10694000F701F5CFB501C8016B960FB6F894DEBF1D
:106950000FBECDBFDF91CF911F910F91FF90EF90B0
:10696000DF90CF90BF90AF909F908F907F906F906F
:106970005F904F903F902F900895FC01DB018C9128
:1069800020813181382798E0A901440F551F37FD38
:1069900006C09A019150C1F73183208308959A016E
:1069A000B1E22B27B0E13B27F5CFBC0180E090E0BE
:1069B0004AE00E942B8C8DE00E94D28B8AE00C94DE
:1069C000D28BCF93DF931F921F92CDB7DEB778940F
:1069D00084B5826084BD84B5816084BD85B58260E4
:1069E00085BD85B5816085BD80916E008160809395
:1069F0006E001092810080918100826080938100FE
:106A0000809181008160809381008091800081600D
:106A1000809380008091B10084608093B100809168
:106A2000B00081608093B00080919100826080937B
:106A300091008091910081608093910080919000FD
:106A40008160809390008091A10082608093A1007A
:106A50008091A10081608093A1008091A00081605D
:106A60008093A00080912101826080932101809118
:106A700021018160809321018091200181608093B8
:106A8000200180917A00846080937A0080917A005E
:106A9000826080937A0080917A00816080937A008E
:106AA00080917A00806880937A001092C10082E021
:106AB0008093C0001092C50087E08093C40080914D
:106AC000C10080618093C1008091C1008860809383
:106AD000C1008091C10080688093C1008091C10095
:106AE0008F7D8093C10010924703E5E3F9E0849124
:106AF0008F010F5F1F4F882321F00E94D28BF80176
:106B0000F6CFE5ECFCE184918F010F5F1F4F8823E6
:106B100021F00E94D28BF801F6CF14B710FF0DC000
:106B2000ECE2F9E084917F019FEFE91AF90A8823EA
:106B300021F00E94D28BF701F5CF11FF0DC0EBE1E0
:106B4000F9E084917F019FEFE91AF90A882321F087
:106B50000E94D28BF701F5CF12FF0DC0E9E0F9E0FA
:106B600084917F019FEFE91AF90A882321F00E949E
:106B7000D28BF701F5CF13FF0DC0E8EFF8E0849159
:106B80007F019FEFE91AF90A882321F00E94D28B36
:106B9000F701F5CF15FF0CC0E7EEF8E084918F0107
:106BA0000F5F1F4F882321F00E94D28BF801F6CF90
:106BB00014BEE0EEF8E084918F010F5F1F4F882331
:106BC00021F00E94D28BF801F6CF80E20E94D28B96
:106BD000E9EDF8E084918F010F5F1F4F882321F0CA
:106BE0000E94D28BF801F6CF8AE00E94D28BE5ECAE
:106BF000FCE184918F010F5F1F4F882321F00E94D9
:106C0000D28BF801F6CFE9ECF8E084918F010F5FA9
:106C10001F4F882321F00E94D28BF801F6CFE5EBBD
:106C2000F8E084918F010F5F1F4F882321F00E94AD
:106C3000D28BF801F6CFECE7F8E084918F010F5F7B
:106C40001F4F882321F00E94D28BF801F6CFE5EC8C
:106C5000FCE184918F010F5F1F4F882321F00E9478
:106C6000D28BF801F6CFE5E6F8E084918F010F5F53
:106C70001F4F882321F00E94D28BF801F6CFE5EC5C
:106C8000FCE184918F010F5F1F4F882321F00E9448
:106C9000D28BF801F6CF20911B0D30911C0DCE0147
:106CA00001962115310519F481529D4002C0821BC5
:106CB000930B9A83898369817A8186E598E00E94A3
:106CC000666760ED74E08FE398E00E9466678AE093
:106CD0000E94D28B81E08093600380936103809354
:106CE0006203809363030E94C27B8CE0E4E5F3E0DF
:106CF000A5E1BBE001900D928A95E1F70E94D08753
:106D00006D9A809101018061809301018091010160
:106D10008860809301019D9A809101018062809337
:106D2000010188E00E944094809101018860809375
:106D3000010186E00E94409487ED80937A001092D2
:106D40007E0010927D0080917E00816080937E00A5
:106D500080917E00846080937E0080E888BD809171
:106D60006E00846080936E006AEF70E080E090E0D7
:106D70000E943A8B85E090E090934D0380934C0302
:106D800060E080911002909111020E94316120E038
:106D900030E040EA50E40E94409987FF0AC08091A9
:106DA000100290911102409790931102809310026B
:106DB000E7CF81E391E0909313028093120260E0A9
:106DC00080914A0390914B030E94316120E030E8AA
:106DD00048E953E40E94999F181654F480914A039D
:106DE00090914B03409690934B0380934A03E7CFD7
:106DF00080910E0290910F020E94806220E030E0AC
:106E000040EA50E40E94409987FF0AC080910E0238
:106E100090910F02409790930F0280930E02E8CF5B
:106E200080914803909149030E94806220E030E005
:106E300046E153E40E94999F181654F48091480348
:106E40009091490340969093490380934803E8CF7B
:106E500098E288E10FB6F894A895809360000FBE81
:106E60009093600080910A01886080930A0180916C
:106E70000A01806180930A0180910A0180628093F7
:106E80000A010E94227280912101887F8160809393
:106E90002101999A989A809107018068809307014F
:106EA0009A9A80910701806480930701809107017D
:106EB00080628093070180910701886080930701B9
:106EC0008091070180618093070190E0E92E93E0B3
:106ED000F92E10E0F70161917F01812F0E940A676E
:106EE0001F5F1530B9F780910A01826080930A0113
:106EF00080910A01816080930A0180910A01846077
:106F000080930A0180910A01806480930A010F9A9C
:106F1000179A0E9A169A0D9A159A0C9A149A269800
:106F20002E9A25982D9A24982C9A3F98479A0A9839
:106F3000129A0998119A389A4098179A10924E030B
:106F4000399A4198169A10924F033A9A4298159A94
:106F5000109250033B9A4398149A809180008C7F42
:106F60008093800080918100877E8860809381007B
:106F7000809180008F738093800080918100887F52
:106F800082608093810080E090E4909389008093F8
:106F90008800109285001092840080916F008260BA
:106FA00080936F0011E01093520378940E947E72D8
:106FB0001092530380910101886080930101109326
:106FC00052031093510380E0E82E80E0F82E809168
:106FD0008103843010F40E944E86809181038823BF
:106FE00099F00E94280F80918103882369F08150D5
:106FF00080938103809180038F5F843018F48093A5
:10700000800302C0109280038091000B8823A9F1B5
:10701000E5ECFCE184918F010F5F1F4F882321F085
:107020000E94D28BF801F6CFE8E4F9E084918F0159
:107030000F5F1F4F882321F00E94D28BF801F6CFFB
:107040008091000B80FD22C08091000B84FD1EC04A
:107050008091000B81FD35C08091000B85FD31C012
:107060008091000B82FD48C08091000B86FD44C0DA
:107070008AE00E94D28B1092000B0E94038EE114D2
:10708000F10409F4A4CF0E940000A1CF6091740321
:107090007091750380917603909177030E944699D1
:1070A000209164033091650340916603509167031A
:1070B0000E94A599AB01BC0184E499E00E9422677B
:1070C000C7CF609178037091790380917A03909192
:1070D0007B030E9446992091680330916903409197
:1070E0006A0350916B030E94A599AB01BC0180E437
:1070F00099E00E942267B4CF60917C0370917D0378
:1071000080917E0390917F030E94469920916C03A9
:1071100030916D0340916E0350916F030E94A599C9
:10712000AB01BC018CE399E00E942267A1CFCF9212
:10713000DF92EF92FF92CF93DF936A017B01FC0114
:107140008491EF012196882321F00E94D28BFE01C9
:10715000F7CF4AE0C701B601DF91CF91FF90EF90E2
:10716000DF90CF900C942B8CCF92DF92EF92FF9216
:10717000CF93DF936A017B01FC018491EF0121969B
:10718000882321F00E94D28BFE01F7CF42E0C70195
:10719000B601DF91CF91FF90EF90DF90CF900C94EC
:1071A000D64A4F925F926F927F92AF92BF92CF92E8
:1071B000DF92EF92FF920F931F93CF93DF9300978D
:1071C00009F456C0FC01208121FD52C0EB018C0165
:1071D00047A050A461A472A4AFA0B8A4C9A4DAA423
:1071E0009501A601C301B2010E94409987FF40C0EA
:1071F000A3019201C301B2010E94A5992B013C0198
:10720000F80183A994A9A5A9B6A9BC01CD019058FC
:107210009B01AC010E94739DF80127A530A941A9EB
:1072200052A90E94A5999B01AC01C301B2010E9421
:10723000729D0E94DE9F7B018C019B01AC01B50118
:10724000C6010E94409987FF02C07501860197011F
:10725000A801B501C6010E944099882349F0A70101
:10726000B8014FA358A769A77AA78881816088834E
:10727000DF91CF911F910F91FF90EF90DF90CF9012
:10728000BF90AF907F906F905F904F9008952F9236
:107290003F924F925F926F927F928F929F92AF92A6
:1072A000BF92CF92DF92EF92FF920F931F93CF93F3
:1072B000DF93CDB7DEB768970FB6F894DEBF0FBE89
:1072C000CDBF1C015B018A01DC01D7966D917D91D8
:1072D0008D919C91DA970E9444996B017C01F50194
:1072E00020813181428153810E94A5990E94399E5B
:1072F0000E94BC9E69877A878B879C87D8012D91D5
:107300003D914D915C91C701B6010E94A5990E94E3
:10731000399E0E94BC9E6D877E878F87988B2985BA
:107320003A854B855C85283731054105510540F488
:1073300088E790E0A0E0B0E089879A87AB87BC87B8
:107340002D853E854F8558892837310541055105E2
:1073500040F488E790E0A0E0B0E08D879E87AF879B
:10736000B88B91012D5B3F4FD9018D919D910D906F
:10737000BC91A02D8D839E83AF83B887BC01CD01C6
:107380000E94469969837A838B839C8369857A8579
:107390008B859C850E944499698B7A8B8B8B9C8B07
:1073A00020E030E0A90169817A818B819C810E9473
:1073B0004099882339F1A7019601C701B6010E94BF
:1073C000A5994B015C0129893A894B895C89CA01DD
:1073D000B9010E94A5999B01AC01C501B4010E94AD
:1073E000729D4B015C0129813A814B815C81CA010C
:1073F000B9010E94739D9B01AC01C501B4010E94BB
:107400004F9E03C060E070E0CB010E94399E0E9455
:10741000B79E2B013C016D817E818F81988590956F
:107420008095709561957F4F8F4F9F4F0E94469931
:107430004B015C016D857E858F8598890E944499FA
:107440006D837E838F83988720E030E0A901C5019A
:10745000B4010E944099882349F12D813E814F81DA
:107460005885CA01B9010E94A5996D8B7E8B8F8BBF
:10747000988FA7019601C701B6010E94A5999B01AB
:10748000AC016D897E898F89988D0E94729D6B01F8
:107490007C01A5019401C501B4010E94739D9B016B
:1074A000AC01C701B6010E944F9E03C060E070E0CE
:1074B000CB010E94E89EF10182889388A488B58858
:1074C00075016401C418D508E608F7080E94B79E44
:1074D000C61AD70AE80AF90AF7FE6BC020E030E0C6
:1074E000A90169817A818B819C810E9440998823BE
:1074F00009F447C029813A814B815C81CA01B901F5
:107500000E94739D6B017C01C501B4010E944499E6
:107510009B01AC01C701B6010E94A5996B017C01DA
:1075200029893A894B895C89CA01B9010E94A599C8
:107530009B01AC01C701B6010E94729D6B017C01E9
:107540002D813E814F815885CA01B9010E94A599BC
:107550009B01AC01C701B6010E94739D6B017C01C8
:1075600020E030E040E850E469817A818B819C81A1
:107570000E94A5999B01AC01C701B6010E944F9ED4
:1075800003C060E070E0CB010E94399E0E94B79E6C
:107590002B013C0197FF03C0412C512C32014814B0
:1075A00059046A047B0410F024013501C12CD12C4C
:1075B00076018FB7F894D1019C9193FD22C0F1011F
:1075C000468A578A608E718EC40CD51CE61CF71C47
:1075D0005A96CD92DD92ED92FC925D9729853A857F
:1075E0004B855C85DB962D933D934D935C93DE97A5
:1075F000FF962D853E854F855889208331834283B0
:1076000053838FBF68960FB6F894DEBF0FBECDBF11
:10761000DF91CF911F910F91FF90EF90DF90CF906E
:10762000BF90AF909F908F907F906F905F904F90A2
:107630003F902F9008952F923F924F925F926F92BA
:107640007F928F929F92AF92BF92CF92DF92EF92F2
:10765000FF920F931F93CF93DF9300D01F92CDB76C
:10766000DEB77B016A011901A5E2BBE02D913D91D6
:107670004D915C91FC0160817181828193810E94B6
:10768000A5990E94A49F2B013C0108E71BE0D801AB
:107690006D937D938D939C9313972091290B30913B
:1076A0002A0B40912B0B50912C0BF70160817181BB
:1076B000828193810E94A5990E94A49F4B015C0145
:1076C000D80114966D937D938D939C931797209179
:1076D0002D0B30912E0B40912F0B5091300BF6015A
:1076E00060817181828193810E94A5990E94A49FEB
:1076F0006B017C01D80118966D937D938D939C93BB
:107700001B972091310B3091320B4091330B5091EC
:10771000340BF10160817181828193810E94A5996E
:107720000E94A49FD8011C966D937D938D939C938A
:107730001F9769837A838B839C830E9474722FB70F
:10774000F894E5E0FBE04082518262827382848299
:107750009582A682B782C086D186E286F386698149
:107760007A818B819C8164877587868797872FBFF5
:107770001092640B1092650B1092660B1092670BBF
:1077800080E1E8E6FBE0DF011D928A95E9F70F90C2
:107790000F900F900F90DF91CF911F910F91FF905D
:1077A000EF90DF90CF90BF90AF909F908F907F90A1
:1077B0006F905F904F903F902F9008952F923F923F
:1077C0004F925F926F927F928F929F92AF92BF92F1
:1077D000CF92DF92EF92FF920F931F93CF93DF939D
:1077E000CDB7DEB7C857D1090FB6F894DEBF0FBECC
:1077F000CDBF3B014A015901EBAAFFAA0BAF21966D
:107800001FAF21973C2C2091250B3091260B4091E6
:10781000270B5091280BDC016D917D918D919C91EE
:107820000E94A5990E94A49FE1966CAF7DAF8EAF98
:107830009FAFE1972091290B30912A0B40912B0BA0
:1078400050912C0BF30160817181828193810E94A0
:10785000A5990E94A49FE5966CAF7DAF8EAF9FAFB8
:10786000E59720912D0B30912E0B40912F0B5091CD
:10787000300BD4016D917D918D919C910E94A599C1
:107880000E94A49FE9966CAF7DAF8EAF9FAFE99742
:107890002091310B3091320B4091330B5091340BCE
:1078A000F50160817181828193810E94A5990E9476
:1078B000A49F6C966CAF7DAF8EAF9FAF6C9780919D
:1078C000780B9091790BA0917A0BB0917B0BE1969C
:1078D000CCACDDACEEACFFACE197C81AD90AEA0A31
:1078E000FB0A80917C0B90917D0BA0917E0BB09157
:1078F0007F0BE5968CAC9DACAEACBFACE597881A1F
:10790000990AAA0ABB0A8091800B9091810BA091E1
:10791000820BB091830BE9960CAD1DAD2EAD3FAD42
:10792000E997081B190B2A0B3B0B0FA718AB29ABC8
:107930003AAB8091A40383FF0EC06C962CAD3DAD95
:107940004EAD5FAD6C972093840B3093850B4093C5
:10795000860B5093870B8091840B9091850BA0919F
:10796000860BB091870B6C964CAC5DAC6EAC7FAC6B
:107970006C97481A590A6A0A7B0A09F495C08091E3
:107980009803811141C060911D0270911E02072E63
:10799000000C880B990B0E9446999B01AC016091E9
:1079A00013047091140480911504909116040E94A0
:1079B000409987FF29C06C968CAD9DADAEADBFAD33
:1079C0006C978093840B9093850BA093860BB09358
:1079D000870BE5ECFCE184918F010F5F1F4F88233B
:1079E00021F00E94D28BF801F6CFE3E0FAE0849117
:1079F0008F010F5F1F4F882321F00E94D28BF80167
:107A0000F6CF412C512C32014BA65CA66DA67EA66A
:107A100077FE0BC0002711279801041915092609C4
:107A200037090BA71CA72DA73EA76091310B7091BA
:107A3000320B8091330B9091340B0E94B79E9B01C7
:107A4000AC01A8ECB0E00E94599D2BA53CA54DA52A
:107A50005EA562177307840795074CF56C968CAD8D
:107A60009DADAEADBFAD6C978093840B9093850BAD
:107A7000A093860BB093870BE5ECFCE184918F011A
:107A80000F5F1F4F882321F00E94D28BF801F6CFA1
:107A9000E4EEF9E084918F010F5F1F4F882321F0FE
:107AA0000E94D28BF801F6CF412C512C3201D70124
:107AB000C6018827B7FD83959927AA27BB27282EBB
:107AC000B7FE03C0E82FE2602E2E0FA518A929A942
:107AD0003AA937FF03C0122D1460212E77FE03C090
:107AE000222D2860222E032D10E0C301B2010E9436
:107AF0004699F801EE0FFF1FEE0FFF1FE056FC4FF7
:107B000020813181428153810E94A5992B013C0142
:107B1000000F111FF801E15EFD4F60817181072E9A
:107B2000000C880B990B0E9446999B01AC01C30184
:107B3000B2010E94A5992AE037ED43E25CE30E947E
:107B4000A5992B013C0120E030E0A9010E94999FFA
:107B500018164CF420E030E040E05FE3C301B201CE
:107B60000E94739D08C0A301920160E070E080E074
:107B70009FE30E94729D0E94B79E6CAF7DAF8EAF57
:107B80009FAF8091880B8F5F8F70A7968FAFA7975D
:107B90008091890BA7960FADA797801303C00E9411
:107BA000038EF6CFE091880B0E2F10E01CA70BA7D9
:107BB0001DE4E19FF0011124E755FB4F108222A242
:107BC000D701C601F7FE07C088279927DC018C1969
:107BD0009D09AE09BF0982839383A483B5838DE495
:107BE0000BA51CA5809FF001819FF00D1124E75586
:107BF000FB4FD501C401B7FE07C088279927DC01D8
:107C000088199909AA09BB0986839783A087B18738
:107C10008DE40BA51CA5809FF001819FF00D112420
:107C2000E755FB4F8FA598A9A9A9BAA9B7FF07C027
:107C3000B095A095909581959F4FAF4FBF4F82878C
:107C40009387A487B5878DE40BA51CA5809FF001C1
:107C5000819FF00D1124E755FB4F2CAD3DAD4EAD8E
:107C60005FAD26873787408B518B4281538164817A
:107C70007581068117812085318504171507260730
:107C8000370714F48A019B018DE4ABA5BCA58A9F3C
:107C9000F0018B9FF00D1124E755FB4F82859385F2
:107CA000A485B58580179107A207B30764F48CAD4E
:107CB0009DADAEADBFAD80179107A207B30764F4C9
:107CC000D901C8010DC00CAD1DAD2EAD3FAD0817DB
:107CD00019072A073B0724F08CAD9DADAEADBFADB3
:107CE0002DE40BA51CA5209FF001219FF00D112470
:107CF000E755FB4F828B938BA48BB58B0697A10521
:107D0000B10510F40C945D48DF01A95BBF4F809171
:107D10009E0390919F038D939C933182452B462B1C
:107D2000472B09F017988DE40BA51CA5809FF00147
:107D3000819FF00D1124E755FB4F86819781A08527
:107D4000B185892B8A2B8B2B09F016988DE40BA516
:107D50001CA5809FF001819FF00D1124E755FB4F7A
:107D600082859385A485B585892B8A2B8B2B09F079
:107D700015982CAD3DAD4EAD5FAD232B242B252B9F
:107D800071F080919D03882319F0815080939D03A9
:107D900031100EC0149880E280939D0309C020909A
:107DA000500430905104009152041091530408C0C3
:107DB00020905404309055040091560410915704BB
:107DC0009101A8016BA97FA98BAD21969FAD219749
:107DD0000E94409987FD02C00C945548C701B60126
:107DE0000E94469920916403309165034091660397
:107DF000509167030E94A5996BAB7CAB8DAB9EAB9A
:107E0000698B7A8B8B8B9C8BC501B4010E94469940
:107E1000209168033091690340916A0350916B038C
:107E20000E94A5994B015C016D8B7E8B8F8B988F87
:107E30006FA578A989A99AA90E94469920916C03F7
:107E400030916D0340916E0350916F030E94A5998C
:107E50006B017C01698F7A8F8B8F9C8F20917003CF
:107E6000309171034091720350917303C301B201C9
:107E70000E94A5996D8F7E8F8F8F98A32DE44BA5BF
:107E80005CA5249FF001259FF00D1124E755FB4FC1
:107E9000428053806480758056E045165104610429
:107EA0007104D4F42681378140855185263031050F
:107EB000410551058CF4228533854485558526304E
:107EC00031054105510544F4DC01CB01BF7787A79B
:107ED00090ABA1ABB2AB38C02BA93CA94DA95EA910
:107EE000CA01B9010E94A5996FA778AB89AB9AAB7B
:107EF000A5019401C501B4010E94A5999B01AC01A3
:107F00006FA578A989A99AA90E94739D4B015C016C
:107F1000A7019601C701B6010E94A5999B01AC017A
:107F2000C501B4010E94739D0E94DE9F2DE4ABA5A4
:107F3000BCA52A9FF0012B9FF00D1124E755FB4FA4
:107F400067A770AB81AB92AB8DE42BA53CA5829F5C
:107F5000F001839FF00D1124E755FB4F87A590A9F1
:107F6000A1A9B2A9A6968CAF9DAFAEAFBFAFA697A1
:107F70009C01AD0160E070E080E89FE30E944F9EAD
:107F800026966CAF7DAF8EAF9FAF26979B01AC015D
:107F9000B101C8010E94A5996B017C018091880BF9
:107FA0009091890B891B8F702B968FAF2B97A70110
:107FB000960160E074E284E799E40E944F9E0E947B
:107FC000A49F4B015C012B968FAD2B97825086307E
:107FD000C0F580914C0490914D04A0914E04B09155
:107FE0004F0488169906AA06BB0658F58819990900
:107FF000AA09BB09BC01CD01660F771F881F991F15
:108000002B96AFAD2B970A2F10E020E030E0A901AE
:1080100098010E941B9DCA01B9010E9444990E94C7
:10802000A49F680D791D8A1D9B1D0E9444999B0188
:10803000AC0160E074E284E799E40E944F9E6B011A
:108040007C01A7019601A6966CAD7DAD8EAD9FAD6E
:10805000A6970E94A5992A966CAF7DAF8EAF9FAF71
:108060002A978DE4EBA5FCA58E9F80018F9F100DB4
:10807000112407551B4F2A962CAD3DAD4EAD5FAD7B
:108080002A97D80193962D933D934D935C939697A1
:1080900052962D913D914D915C9155972FA738ABFC
:1080A00049AB5AABCA01B9010E9444996BAB7CAB96
:1080B0008DAB9EABA70196010E94A5990E94399EA7
:1080C0000E94BC9E62966CAF7DAF8EAF9FAF6297F1
:1080D000F80167AB70AF81AF92AF8E010F5E1F4F9B
:1080E00022961FAF0EAF22970051110968961FAF5D
:1080F0000EAF689704E714E0A2961FAF0EAFA297E9
:108100008E010F5D1F4F1AA709A768960EAD1FAD10
:1081100068976E961FAF0EAF6E97212C312C10E82A
:108120001FAB0FE30BAF2296AEADBFAD22976D91A3
:108130007D918D919D912296BFAFAEAF2297A70101
:1081400096010E94A5996E96EEADFFAD6E97619374
:108150007193819391936E96FFAFEEAF6E974B0143
:108160005C01E894B7F8A296AEADBFADA2970D91B1
:108170001D912D913D91A296BFAFAEAFA29766968D
:108180000CAF1DAF2EAF3FAF6697A9019801C50197
:10819000B4010E94999F1816C4F4A5019401669633
:1081A0006CAD7DAD8EAD9FAD66970E944F9E5B011D
:1081B0008C019B01AC01B1018FA99BAD0E94999FDD
:1081C00018161CF415010FAB1BAF22960EAD1FAD98
:1081D000229729A53AA50217130709F0A4CF20E09A
:1081E00030E040E85FE3B1018FA99BAD0E94409968
:1081F00087FF4BC07E0131E1E30EF11C68960EADA6
:108200001FAD689791014FA95BADD8016D917D912C
:108210008D919C910E94A599F8016193719381932E
:1082200091938F01EE15FF0569F78DE42BA53CA511
:10823000829F8001839F100D112407551B4F9101D0
:108240004FA95BAD2A966CAD7DAD8EAD9FAD2A97E3
:108250000E94A599D80193966D937D938D939C93DD
:10826000969762966CAD7DAD8EAD9FAD62970E9484
:10827000449991014FA95BAD0E94A5990E94BC9EB3
:10828000F80167AB70AF81AF92AF26962CAD3DADD4
:108290004EAD5FAD26976BA97CA98DA99EA90E94C2
:1082A000A5996FAB78AF89AF9AAF411451046104BF
:1082B000710459F58DE40BA51CA5809FF001819FE9
:1082C000F00D1124E755FB4F86819781A085B1857C
:1082D000892B8A2B8B2BC9F482859385A485B58540
:1082E000892B8A2B8B2B89F420915C0430915D04BF
:1082F00040915E0450915F046FA978AD89AD9AAD4D
:108300000E94A5990E94399E27C22CAD3DAD4EAD6D
:108310005FAD232B242B252B49F0609160047091D5
:108320006104809162049091630408C060915804D4
:108330007091590480915A0490915B042FA938AD33
:1083400049AD5AAD0E94A5990E94399E0E94BC9EDB
:108350006B017C018091950490919604A091970403
:10836000B09198040FA518A929A93AA980179107D7
:10837000A207B30708F4E2C0411451046104710478
:1083800041F12091990430919A0440919B045091BD
:108390009C042C153D054E055F05D8F46FA578A902
:1083A00089A99AA90E940C9D4B015C01A701960125
:1083B000C301B2010E940C9D86169706A806B90655
:1083C00040F4C501B401A30192010E941B9D690103
:1083D0007A018DE40BA51CA5809FF001819FF00D13
:1083E0001124E755FB4F86809780A084B1848114C7
:1083F0009104A104B10441F120919D0430919E04A7
:1084000040919F045091A0042C153D054E055F0539
:10841000D8F46FA578A989A99AA90E940C9D2B016F
:108420003C01A7019601C501B4010E940C9D4616AE
:1084300057066806790640F4C301B201A50194010C
:108440000E941B9D69017A018DE40BA51CA5809FEC
:10845000F001819FF00D1124E755FB4F8284938436
:10846000A484B58481149104A104B10441F1209144
:10847000A1043091A2044091A3045091A4042C15AE
:108480003D054E055F05D8F46FA578A989A99AA97D
:108490000E940C9D2B013C01A7019601C501B4016E
:1084A0000E940C9D461657066806790640F4C301E3
:1084B000B201A50194010E941B9D69017A018DE41E
:1084C0000BA51CA5809FF001819FF00D1124E7559D
:1084D000FB4F86849784A088B18881149104A104FD
:1084E000B10409F43DC12091A5043091A604409146
:1084F000A7045091A8042C153D054E055F0508F012
:108500002FC16FA578A989A99AA90E940C9D2B015A
:108510003C01A7019601C501B4010E940C9D4616BD
:1085200057066806790608F01BC1C301B201A50110
:1085300094010E941B9D69017A0112C141145104EA
:1085400061047104A9F16091990470919A04809179
:108550009B0490919C046C157D058E059F0540F54C
:108560000E9444992BA93CA94DA95EA90E94A599F6
:108570004B015C01C301B2010E9446992B013C01F1
:10858000C701B6010E944499A30192010E94A599D6
:10859000A50194010E94999F181654F4A301920119
:1085A000C501B4010E944F9E0E94BC9E6B017C01DC
:1085B0008DE40BA51CA5809FF001819FF00D112477
:1085C000E755FB4F46805780608471844114510405
:1085D00061047104A9F160919D0470919E048091E1
:1085E0009F049091A0046C157D058E059F0540F5B4
:1085F0000E9444992BA93CA94DA95EA90E94A59966
:108600004B015C01C301B2010E9446992B013C0160
:10861000C701B6010E944499A30192010E94A59945
:10862000A50194010E94999F181654F4A301920188
:10863000C501B4010E944F9E0E94BC9E6B017C014B
:108640008DE40BA51CA5809FF001819FF00D1124E6
:10865000E755FB4F4284538464847584411451046C
:1086600061047104A9F16091A1047091A204809148
:10867000A3049091A4046C157D058E059F0540F51B
:108680000E9444992BA93CA94DA95EA90E94A599D5
:108690004B015C01C301B2010E9446992B013C01D0
:1086A000C701B6010E944499A30192010E94A599B5
:1086B000A50194010E94999F181654F4A3019201F8
:1086C000C501B4010E944F9E0E94BC9E6B017C01BB
:1086D0008DE40BA51CA5809FF001819FF00D112456
:1086E000E755FB4F86849784A088B1888114910454
:1086F000A104B104A9F16091A5047091A604809130
:10870000A7049091A8046C157D058E059F0540F582
:108710000E9444992BA93CA94DA95EA90E94A59944
:108720002B013C01C501B4010E9446994B015C013B
:10873000C701B6010E944499A50194010E94A59920
:10874000A30192010E94999F181654F4A501940167
:10875000C301B2010E944F9E0E94BC9E6B017C012E
:108760008DE42BA53CA5829F8001839F100D1124D1
:1087700007551B4FF801ED5BFF4FC082D182E282AB
:10878000F382C701B6010E9444996B017C012FA9B5
:1087900038AD49AD5AAD0E944F9EA0966CAF7DAFEB
:1087A0008EAF9FAFA097D801D3966D937D938D9395
:1087B0009C93D69720E030E040E85BE4C701B60127
:1087C0000E94A59920E034E244EF59E40E944F9EB4
:1087D0000E94B79EF801668F778F80A391A3F3A1C3
:1087E000FCAFD8019496BC91BFA7F801F5A1FBABF3
:1087F000D8019696BC91BFAB0CE314E0AD961FAFC9
:108800000EAFAD972E0111E1410E511C3CE3232E1A
:1088100034E0332E68966EAC7FAC68970CAD0BAF2E
:108820001FA521961FAF21972396FFAF2397279669
:10883000BFAF279710E0D3018D909D90AD90BD9074
:108840003D01E894B7F8F101C190D190E190F19029
:108850001F01A7019601C501B4010E94999F181636
:10886000E4F5112379F12CAD3FA54BA95FA9C70110
:10887000B6010E94A5996B017C012BAD21963FADFD
:10888000219723964FAD239727965FAD2797C50174
:10889000B4010E94A599A70196010E94999F1816FC
:1088A000DCF4A5019401C701B6010E944F9E6BAF95
:1088B00021967FAF219723968FAF239727969FAF5F
:1088C00027970AC0CBAE2196DFAE21972396EFAE55
:1088D00023972796FFAE279711E06414750409F0DB
:1088E000AACF2B960FAD2B97023008F476C13090AB
:1088F000640B2090650B1091660B0091670B27E1CC
:1089000037EB41ED58E3632D722D812F902F0E949C
:10891000999F18160CF061C121E0A1962FAFA19785
:108920002CAD3FA54BA95FA9632D722D812F902FF0
:108930000E94999F1816A4F0A1961FAEA1972CAD86
:108940003FA54BA95FA9632D722D812F902F0E9407
:108950004F9EAB966CAF7DAF8EAF9FAFAB9714C001
:10896000232D322D412F502F6CAD7FA58BA99FA9B0
:108970000E944F9EAB966CAF7DAF8EAF9FAFAB9713
:108980003CAC2FA41BA90FA948E65BE064965FAF3F
:108990004EAF649780E090E0A0E8BFE32E968CAFE6
:1089A0009DAFAEAFBFAF2E972F961FAE2F97649699
:1089B000AEADBFAD6497CD90DD90ED90FD90649627
:1089C000BFAFAEAF64976896EEADFFAD689781908C
:1089D0009190A190B1906896FFAFEEAF6897A19685
:1089E000FFADA197FF2361F0AB962CAD3DAD4EAD31
:1089F0005FADAB97C701B6010E94A5996B017C01E1
:108A00002F962FAD2F972223C1F02E962CAD3DAD82
:108A10004EAD5FAD2E97C701B6010E94A5996B01BF
:108A20007C012E962CAD3DAD4EAD5FAD2E97C501B0
:108A3000B4010E94A5994B015C01A5019401C701F5
:108A4000B6010E94999F20E030E0A90118162CF58C
:108A5000C501B4010E94999F18164CF020E030E047
:108A6000A901C701B6010E94409987FF05C0A50171
:108A70009401C701B60124C02401350177FA70942E
:108A800077F87094A3019201C701B6010E94999FE3
:108A900018165CF52601370128C0C501B4010E94F3
:108AA000409987FD09C020E030E0A901C701B60167
:108AB0000E94999F18164CF4A7019601C501B401B4
:108AC0000E94729D2B013C0110C02601370177FAEC
:108AD000709477F87094A5019401C301B2010E94CB
:108AE000999F181614F024013501AD96AEADBFADB7
:108AF000AD97CD90DD90ED90FD90AD96BFAFAEAF50
:108B0000AD97A7019601C301B2010E94999F181663
:108B1000ECF4A3019201C701B6010E944F9E9B0194
:108B2000AC012E966CAD7DAD8EAD9FAD2E970E94A3
:108B3000A5992E966CAF7DAF8EAF9FAF2E972F96D7
:108B4000BFAD2F97BF5F2F96BFAF2F976496EEAD47
:108B5000FFAD6497E857FB4009F029CF2F963FAD52
:108B60002F97332381F02E962CAD3DAD4EAD5FADEA
:108B70002E97632D722D812F902F0E94A599362E4E
:108B8000272E182F092F24EA30E74DE75FE3632DE6
:108B9000722D812F902F0E94A5996B017C019B0162
:108BA000AC016091990370919A0380919B0390911D
:108BB0009C030E94999F18163CF5A70196016BAD86
:108BC00021967FAD219723968FAD239727969FAD52
:108BD00027970E94999F1816BCF48DE40BA51CA53D
:108BE000809FF001819FF00D1124E755FB4F80819C
:108BF000846080833BAC21962FAC219723961FADD8
:108C0000239727960FAD27978DE42BA53CA5829F30
:108C1000F001839FF00D1124E755FB4F832D922D1A
:108C2000A12FB02F83A794A7A5A7B6A7A0966CAD38
:108C30007DAD8EAD9FADA09790589B01AC010E9479
:108C4000739DA6962CAD3DAD4EAD5FADA6970E942F
:108C5000A5999B01AC016BE077ED83E29BE30E9459
:108C6000729D0E94DE9F6B017C019B01AC01632D14
:108C7000722D812F902F0E94409987FD04C03C2CBB
:108C80002D2C1E2D0F2D8DE44BA55CA5849FF0018E
:108C9000859FF00D1124E755FB4F832D922DA12FB9
:108CA000B02F87A390A7A1A7B2A7B0809601A70174
:108CB0006CAD7FA58BA99FA90E944099181614F44A
:108CC00081E001C083E09DE4ABA5BCA59A9F900123
:108CD0009B9F300D1124F901E755FB4F7F01B82A06
:108CE000B08280E1FE013196A8E6BBE001900D92D2
:108CF0008A95E1F78CAD9FA5ABA9BFA98093640BC2
:108D00009093650BA093660BB093670B8BAD219688
:108D10009FAD21972396AFAD23972796BFAD279799
:108D20008093990390939A03A0939B03B0939C0321
:108D30002CAD3FA54BA95FA9BC01CD010E944F9E60
:108D40006DA37EA38FA398A72CAD3FA54BA95FA9C8
:108D5000632D722D812F902F0E944F9E69A37AA3BD
:108D60008BA39CA3AE014B5D5F4FBE016F5D7F4F38
:108D7000C7010E944739A7960FADA7970093880BAC
:108D8000E1962CAD3DAD4EAD5FADE1972093780BF4
:108D90003093790B40937A0B50937B0BE5968CAD17
:108DA0009DADAEADBFADE59780937C0B90937D0BF1
:108DB000A0937E0BB0937F0BE9960CAD1DAD2EAD4D
:108DC0003FADE9970093800B1093810B2093820BAA
:108DD0003093830B6C962CAD3DAD4EAD5FAD6C9773
:108DE0002093840B3093850B4093860B5093870B15
:108DF0008091880B9091890B891B8F70843048F487
:108E00001091890BF12C00E080E090E02DE4E22E3F
:108E10009EC04090890B8091880B83508F70F82EF4
:108E2000A12CB12C00E010E09DE4592EF41441F384
:108E30000115110521F0D8018C9182FDE1CF8FEF52
:108E40008F0D8F70F82E589EC0011124FC01E7553C
:108E5000FB4FFCA7EBA70115110509F474C0A11481
:108E6000B10409F470C0D8019B967C909B979C96A6
:108E7000CC909C979D96DC909D979E96EC909E97AB
:108E8000272D3C2D4D2D5E2D97966D917D918D91C9
:108E90009C919A970E944099882309F454C0F80144
:108EA000608061FC42C0D50197968D909D90AD90F9
:108EB000BC909A97A5019401672D7C2D8D2D9E2D38
:108EC0000E94409918168CF5A5019401C501B401C2
:108ED0000E94A5994B015C01F80183A994A9A5A959
:108EE000B6A9BC01CD0190589B01AC010E94739DB5
:108EF000D8019F962D913D914D915C91D2970E9402
:108F0000A5999B01AC01C501B4010E94729D0E940C
:108F1000DE9F1B015C019B01AC01672D7C2D8D2D1B
:108F20009E2D0E94409987FF04C0272C3C2CAD2C1D
:108F3000BE2CC101D501F80187A390A7A1A7B2A7B4
:108F4000862D8160808358010BA51CA56FCF2091D1
:108F5000880B121791F0E19E90011124A901475549
:108F60005B4F6A016F2D702F0E94D1381F5F1F70F9
:108F70008F2D902FFC2C0D2DEACF6F2D702F0E947E
:108F8000D138F090890B00E010E08DE4E82E4F2DF1
:108F90000F2C000C550B8091880B90E04817590757
:108FA00009F44DC0E49EC001E59E900D1124DC0142
:108FB000A755BB4F6D0101151105D9F1F80180814D
:108FC00080FD03C08C9180FF34C0D80193968D90B2
:108FD0009D90AD90BC909697E49EF001E59EF00DBB
:108FE0001124E755FB4FA501940167A170A581A548
:108FF00092A50E944F9E69A37AA38BA39CA3A5016F
:109000009401F80167A170A581A592A50E944F9EC9
:109010006DA37EA38FA398A7AE014F5D5F4FBE01E6
:109020006B5D7F4FC8010E944739D8018C918E7FBC
:109030008C9381E08F0D8F70F82E8601A8CF0115DB
:10904000110569F1F801C3A0D4A0E5A0F6A0A7011D
:1090500096016DEC7CEC8CE49DE30E944F9E69A32D
:109060007AA38BA39CA3A7019601D80197966D9133
:109070007D918D919C919A970E944F9E6DA37EA3A6
:109080008FA398A7AE014F5D5F4FBE016B5D7F4F11
:10909000C8010E944739F80180818E7F80838091CA
:1090A0006F00826080936F0008C02BA83FA80BADB3
:1090B00021961FAD21970C94EE3EC858DF4F0FB696
:1090C000F894DEBF0FBECDBFDF91CF911F910F91FE
:1090D000FF90EF90DF90CF90BF90AF909F908F90D8
:1090E0007F906F905F904F903F902F9008952F92B8
:1090F0003F924F925F926F927F928F929F92AF9228
:10910000BF92CF92DF92EF92FF920F931F93CF9374
:10911000DF93CDB7DEB7EC970FB6F894DEBF0FBE86
:10912000CDBF20911704222309F437C11C010091FF
:10913000440B1091450B2091460B3091470B40900A
:10914000480B5090490B60904A0B70904B0B49AA0A
:109150005AAA6BAA7CAA80904C0B90904D0BA090C1
:109160004E0BB0904F0B4091500B5091510B6091B2
:10917000520B7091530B8091540B9091550BA09111
:10918000560BB091570B8DAB9EABAFABB8AFC09049
:10919000580BD090590BE0905A0BF0905B0B8091DC
:1091A0005C0B90915D0BA0915E0BB0915F0B4090BA
:1091B000600B5090610B6090620B7090630B49AE36
:1091C0005AAE6BAE7CAE4090400B5090410B60901D
:1091D000420B7090430B49825A826B827C828D8253
:1091E0009E82AF82B886C986DA86EB86FC860D87BA
:1091F0001E872F87388B498B5A8B6B8B7C8B8D8B83
:109200009E8BAF8BB88F89A99AA9ABA9BCA9898F6E
:109210009A8FAB8FBC8F4DA85EA86FA878AC4D8E8F
:109220005E8E6F8E78A289AD9AADABADBCAD89A3D1
:109230009AA3ABA3BCA320918C0330918D034091E2
:109240008E0350918F03D1016D917D918D919C91F1
:109250000E94729D20E030E040E450E40E94739D43
:109260006DA77EA78FA798AB2091900330919103B3
:109270004091920350919303F1016481758186813D
:1092800097810E94729D20E030E04EE353E40E94FB
:10929000729D69A77AA78BA79CA720919403309110
:1092A00095034091960350919703D10118966D91C3
:1092B0007D918D919C911B970E94729D6DA37EA3C1
:1092C0008FA398A7CE0185969F938F9304969F9323
:1092D0008F9304969F938F93EDB7FEB7B4970FB615
:1092E000F894FEBF0FBEEDBFADB7BEB7119684E2D6
:1092F000FE01319601900D928A95E1F70E94516B23
:1093000020E030E040E450E46DA57EA58FA598A94B
:109310000E94729D20918C0330918D0340918E03A9
:1093200050918F030E94739DD1016D937D938D9316
:109330009C93139720E030E04EE353E469A57AA5AF
:109340008BA59CA50E94739D209190033091910361
:1093500040919203509193030E94739DF1016483A5
:109360007583868397832091940330919503409170
:109370009603509197036DA17EA18FA198A50E949D
:10938000739DD10118966D937D938D939C931B973C
:109390000FB6F894DEBF0FBECDBFEC960FB6F894B3
:1093A000DEBF0FBECDBFDF91CF911F910F91FF9018
:1093B000EF90DF90CF90BF90AF909F908F907F9075
:1093C0006F905F904F903F902F900895CF92DF92D3
:1093D000EF92FF920F931F93CF93DF93CDB7DEB73A
:1093E0002C970FB6F894DEBF0FBECDBF20911704A7
:1093F000222309F4B0C08A017B016C0120918C0307
:1094000030918D0340918E0350918F03FC01608158
:109410007181828193810E94729D20E030E040E45E
:1094200050E40E94739D69877A878B879C8720917F
:109430009003309191034091920350919303F7016F
:1094400060817181828193810E94729D20E030E071
:109450004EE353E40E94729D6D837E838F839887D1
:109460002091940330919503409196035091970376
:10947000F80160817181828193810E94729D69836C
:109480007A838B839C83CE0101969F938F9304965E
:109490009F938F9304969F938F938DB79EB78497D6
:1094A0000FB6F8949EBF0FBE8DBFADB7BEB7119675
:1094B00084E2E0E4FBE001900D928A95E1F70E94DE
:1094C000516B20E030E040E450E469857A858B857B
:1094D0009C850E94729D20918C0330918D03409158
:1094E0008E0350918F030E94739DF60160837183F8
:1094F0008283938320E030E04EE353E46D817E81EC
:109500008F8198850E94739D2091900330919103E3
:1095100040919203509193030E94739DF7016083E1
:1095200071838283938320919403309195034091BA
:1095300096035091970369817A818B819C810E9467
:10954000739DF80160837183828393830FB6F894CF
:10955000DEBF0FBECDBF2C960FB6F894DEBF0FBE98
:10956000CDBFDF91CF911F910F91FF90EF90DF90D2
:10957000CF900895CF92DF92EF92FF926B017C0122
:1095800097FF0BC08DE20E94D28BF094E094D094B0
:10959000C094C11CD11CE11CF11C4AE0C701B601FA
:1095A000FF90EF90DF90CF900C942B8C8F929F9236
:1095B000AF92BF92CF92DF92EF92FF92CF936B0167
:1095C0007C01B42E20E030E0A9010E94409987FF81
:1095D00007C08DE20E94D28BF7FAF094F7F8F0946E
:1095E000C0E060E070E080E09FE3CB1541F02DEC3F
:1095F0003CEC4CEC5DE30E94A599CF5FF6CF9B015C
:10960000AC01C701B6010E94739D6B017C010E94F1
:10961000BC9E4B015C014AE00E942B8CCC2381F163
:10962000C501B4010E9444999B01AC01C701B60178
:109630000E94729D6B017C018EE20E94D28B20E021
:1096400030E040E251E4C701B6010E94A5994B0108
:109650005C010E94B79E6B01770FEE08FF08C701FF
:10966000B60188DFC701B6010E9446999B01AC0193
:10967000C501B4010E94729D6B017C01C150F9F6D5
:10968000CF91FF90EF90DF90CF90BF90AF909F90E1
:109690008F900895EF92FF921F93CF93DF931F92C5
:1096A000CDB7DEB7182FE2E6FAE084917F012FEF05
:1096B000E21AF20A882331F099830E94D28BF701D3
:1096C0009981F3CFE12FF92F84917F019FEFE91A60
:1096D000F90A882321F00E94D28BF701F5CFE9E443
:1096E000FAE084917F012FEFE21AF20A882321F039
:1096F0000E94D28BF701F5CF0F90DF91CF911F9190
:10970000FF90EF900895CF92EF92FF920F931F93E7
:10971000CF93DF93CDB7DEB72C970FB6F894DEBFAB
:109720000FBECDBFC0908203E5E1FBE0808591854F
:10973000A285B3854481558166817781008111813D
:109740002281338109831A832B833C834D835E837B
:109750006F83788789879A87AB87BC87AE01475F1D
:109760005F4FBE016B5F7F4FCE0101962FDEE09011
:109770001902F0901A0200911B0210911C0221E2C2
:109780003BE0AE01475F5F4FBE016B5F7F4FCE0195
:1097900001960E94DE3B2C960FB6F894DEBF0FBEFA
:1097A000CDBFDF91CF911F910F91FF90EF90CF90A0
:1097B0000895BF92CF92DF92EF92FF920F931F9383
:1097C000CF93DF938EE3E82E8AE0F82E05E11BE0CD
:1097D0009FE3C92E93E0D92ECCEFD2E0BC2E84E0DB
:1097E000B80E89910E948A888823D9F00E945788F0
:1097F000F6012081211104C020914303222331F07E
:10980000F801208131814281538103C020E030E0A2
:10981000A9010E94739DF701608371838283938302
:109820000AC0F80180819181A281B381F701808310
:109830009183A283B383F4E0EF0EF11C0C5F1F4F02
:109840008FEFC81AD80ABC12CCCF86E40E94B98820
:109850008823C9F00E94578820E030E0A9010E94C7
:10986000999F181684F40E94578820E030E040E762
:1098700052E40E944F9E6093190270931A028093E3
:109880001B0290931C02DF91CF911F910F91FF90CB
:10989000EF90DF90CF90BF9008958F929F92AF92FC
:1098A000BF92CF92DF92EF92FF920F931F93CF93CD
:1098B000DF93CDB7DEB760970FB6F894DEBF0FBE6B
:1098C000CDBF490194E0890250011124F501EB5EFE
:1098D000F44F6F0110821182128213824D875E87CE
:1098E0006F87788B0E94D0874D855E856F857889DC
:1098F000F6014083518362837383C090820320E02A
:1099000030E0A901B801C4010E944099811108C04A
:10991000F501EE5EF34E85909590A590B49004C04D
:10992000C801D4014C015D0180911D0B90911E0B6B
:10993000A0911F0BB091200B4091190B50911A0B65
:1099400060911B0B70911C0B0091150B1091160B65
:109950002091170B3091180B09831A832B833C83BA
:109960004D835E836F83788789879A87AB87BC87AF
:10997000AE01475F5F4FBE016B5F7F4FCE01019627
:1099800025DD8501740121E23BE0AE01475F5F4FB9
:10999000BE016B5F7F4FCE0101960E94DE3B0E94AD
:1099A00074721092000B60960FB6F894DEBF0FBE73
:1099B000CDBFDF91CF911F910F91FF90EF90DF907E
:1099C000CF90BF90AF909F908F9008959091170483
:1099D000891771F080931704811107C00E94B88F16
:1099E00084EF9AE084DB0C94DC8C85E19BE07FCBF8
:1099F000089580E0EBDFE0E4FBE080E090E0A0E8A9
:109A0000BFE380839183A283B3831482158216827D
:109A1000178210861186128613861486158616867E
:109A20001786808B918BA28BB38B148A158A168A2A
:109A3000178A108E118E128E138E148E158E168E1E
:109A4000178E80A391A3A2A3B3A308958091A70327
:109A50009091A803A091A903B091AA038093190241
:109A600090931A02A0931B02B0931C028091A5034D
:109A70009091A60390930102809300020C947E8B38
:109A80008091190290911A02A0911B02B0911C02C0
:109A90008093A7039093A803A093A903B093AA036C
:109AA00080910002909101029093A6038093A503F8
:109AB00084E690E090930102809300020C947E8BE8
:109AC0004F925F926F927F928F929F92AF92BF92CE
:109AD000CF92DF92EF92FF920F931F93CF93DF937A
:109AE0005C014B01EA0189014090190250901A0271
:109AF00060901B0270901C02288139814A815B8131
:109B000060911D0B70911E0B80911F0B9091200B8B
:109B10000E94409987FF29C0F801C080D180E2806F
:109B2000F38020E030E0A901C701B6010E9440990E
:109B3000811106C0EAE1FCE1C590D590E590F49072
:109B4000C0921902D0921A02E0921B02F0921C02FB
:109B500088819981AA81BB8180931D0B90931E0BF4
:109B6000A0931F0BB093200BCEDDF801C080D180F5
:109B7000E280F38020E030E0A901C701B6010E9435
:109B80004099811108C0C0901402D0901502E09055
:109B90001602F0901702C0921902D0921A02E092B7
:109BA0001B02F0921C02F50180819181A281B38198
:109BB0008093150B9093160BA093170BB093180B73
:109BC000F40180819181A281B3818093190B9093DC
:109BD0001A0BA0931B0BB0931C0B95DD28813981C8
:109BE0004A815B8160911D0B70911E0B80911F0B50
:109BF0009091200B0E94999F18164CF5F801C08097
:109C0000D180E280F38020E030E0A901C701B601F5
:109C10000E944099811106C0EAE1FCE1C590D5900F
:109C2000E590F490C0921902D0921A02E0921B02C1
:109C3000F0921C0288819981AA81BB8180931D0BBF
:109C400090931E0BA0931F0BB093200B5CDD0E9422
:109C500074724092190250921A0260921B02709222
:109C60001C02DF91CF911F910F91FF90EF90DF9039
:109C7000CF90BF90AF909F908F907F906F905F90AC
:109C80004F9008951F93CF93DF93CDB7DEB72C97F6
:109C90000FB6F894DEBF0FBECDBF90915303981757
:109CA00061F1182F0E94F1928091150B9091160B83
:109CB000A091170BB091180B89879A87AB87BC8747
:109CC0008091190B90911A0BA0911B0BB0911C0B5A
:109CD0008D839E83AF83B88719821A821B821C8270
:109CE0009E012F5F3F4F4DE15BE0BE016B5F7F4FF9
:109CF000CE010996E5DE1093530380E02C960FB653
:109D0000F894DEBF0FBECDBFDF91CF911F910895B4
:109D10002F923F924F925F926F927F928F929F927B
:109D2000AF92BF92CF92DF92EF92FF920F931F9369
:109D3000CF93DF93CDB7DEB7DA950FB6F894DEBFD9
:109D40000FBECDBF0E944E9281110C94A35CFE0108
:109D500031968CE3DF011D928A95E9F70091170493
:109D6000C352DF4F0883CD5DD0408AE40E948A88C9
:109D7000882319F03EDE0C94A35C86E50E94B98826
:109D8000882349F00E942788C153DF4F7983688375
:109D9000CF5CD04006C0C153DF4F19821882CF5C20
:109DA000D040C153DF4F08811981CF5CD0400530CE
:109DB000110570F0E7E3FCE084918F010F5F1F4F06
:109DC000882311F40C94A35C0E94D28BF801F4CF89
:109DD00084E40E948A88C152DF4F8883CF5DD040DF
:109DE000882339F00E944888C152DF4F8883CF5DB5
:109DF000D040C153DF4F08811981CF5CD040033080
:109E000011056CF484E50E948A88882379F00E9409
:109E10004888C252DF4F8883CE5DD0400CC011E02D
:109E2000C252DF4F1883CE5DD04005C0C252DF4F13
:109E30001882CE5DD04088E50E94B988882321F041
:109E40000E942788162F01C012E089E50E94B98878
:109E5000882321F00E942788062F01C002E080E5B8
:109E60000E94B988811103C0212E302E04C00E94A7
:109E70002788262E362E21E0221518F0E2E0FCE09D
:109E800004C031E0331568F0F9CF84918F010F5F82
:109E90001F4F882311F40C94A35C0E94D28BF8010D
:109EA000F4CF83E50E94B988882319F00E9457886F
:109EB00004C060E070E88BEB95E420E030E040E720
:109EC00052E40E944F9E6093140270931502809397
:109ED000160290931702C0908C03D0908D03E090EF
:109EE0008E03F0908F038CE40E94B988811109C021
:109EF00020E030E040E450E4C701B6010E94729DCA
:109F000002C00E9457880E94B79E6B017C01CF520D
:109F1000DF4F79836883C15DD04080908C0390903F
:109F20008D03A0908E03B0908F0382E50E94B988C4
:109F3000811109C020E030E041E253E4C501B401E1
:109F40000E94739D02C00E9457880E94B79E4B01D9
:109F50005C01C154DF4F79836883CF5BD040409070
:109F6000900350909103609092037090930386E465
:109F70000E94B988811109C020E030E040EE50E431
:109F8000C301B2010E94729D02C00E9457880E94C4
:109F9000B79EC554DF4F688379838A839B83CB5BED
:109FA000D040C554DF4F08811981CB5BD040C752E8
:109FB000DF4F19830883C95DD040409090035090D3
:109FC0009103609092037090930382E40E94B98899
:109FD000811109C020E030E041E253E4C301B20145
:109FE0000E94739D02C00E9457880E94B79ECB5268
:109FF000DF4F688379838A839B83C55DD040CB52D2
:10A00000DF4F08811981C55DD040CD53DF4F1983E3
:10A010000883C35CD040B6010D2C000C880B990B53
:10A020000E944699CC51DF4F688379838A839B8352
:10A03000C45ED04040908C0350908D0360908E039E
:10A0400070908F0320E030E040E450E4C301B2019F
:10A050000E94729D9B01AC01CC51DF4F68817981D8
:10A060008A819B81C45ED0400E94409911E0C9540E
:10A07000DF4F1883C75BD04087FD10C0C40109972C
:10A08000CF52DF4F08811981C15DD04008171907F1
:10A090002CF4C954DF4F1882C75BD040B401990C2F
:10A0A000880B990B0E9446994B015C0120E030E03F
:10A0B00042E253E4C301B2010E94739D9B01AC01D3
:10A0C000C501B4010E94999F18167CF029E0C20EC8
:10A0D000D11C01E0C154DF4F88819981CF5BD04012
:10A0E000C816D9061CF400E001C001E0C554DF4FDA
:10A0F000A881B981CB5BD040BD01BB0F880B990B08
:10A100000E944699C851DF4F688379838A839B8375
:10A11000C85ED040C0909003D0909103E09092032D
:10A12000F090930320E030E040EE50E4C701B60128
:10A130000E94729D9B01AC01C851DF4F68817981FB
:10A140008A819B81C85ED0400E94409911E087FDC2
:10A1500011C0CB52DF4F88819981C55DD0400997EE
:10A16000C752DF4FE881F981C95DD040E817F90790
:10A170000CF410E0CB52DF4F28813981C55DD0400F
:10A18000B901330F880B990B0E9446994B015C0172
:10A1900020E030E04EE353E4C701B6010E94739D16
:10A1A0009B01AC01C501B4010E94999F1816A4F04F
:10A1B000C554DF4F88819981CB5BD0400996FF243D
:10A1C000F394CD53DF4FA881B981C35CD0408A1787
:10A1D0009B0724F4F12C02C0FF24F394C954DF4FF1
:10A1E000B881C75BD040B1110BC0002321F083EFD1
:10A1F0009BE050DA0AC0111108C0F1100BC013C067
:10A200008BEF9BE047DA0111F2CF112319F08BEEAF
:10A210009BE040DAFF2011F40C94A35C84EE9BE0F9
:10A2200039DA0C94A35CC153DF4F08811981CF5CEC
:10A23000D040012BF9F0EDECFBE084918F010F5F32
:10A240001F4F882321F00E94D28BF801F6CFC15214
:10A25000DF4F1881CF5DD040112361F0E4EBFBE0CC
:10A2600084918F010F5F1F4F882321F00E94D28BB2
:10A27000F801F6CF0E94747210921704C152DF4F9A
:10A280000881CF5DD04001110AC00E94B88F84EFD1
:10A290009AE00E9477480E94DC8C0E94D08781E07F
:10A2A000F1DC882349F0C352DF4F1881CD5DD040E7
:10A2B000109317040C94A35CE3DB85E40E948A8866
:10A2C000582E882319F00E944888582E022D10E03D
:10A2D000C351DF4F19830883CD5ED040032D10E0BA
:10A2E000C151DF4F19830883CF5ED040239C80018A
:10A2F0001124CB52DF4F19830883C55DD040122D46
:10A300001170C553DF4F1883CB5CD040CB52DF4F69
:10A3100008811981C55DD040000F111F000F111F6A
:10A32000CD50DF4F19830883C35FD040CB52DF4F3E
:10A3300008811981C55DD04023E0000F111F2A95C7
:10A34000E1F7CF50DF4F19830883C15FD040C55478
:10A35000DF4F19821882CB5BD04066246A94762C3A
:10A36000C154DF4F08811981CF5BD040CF52DF4FFE
:10A3700028813981C15DD040021B130BC154DF4FCE
:10A3800019830883CF5BD040CD53DF4F08811981FB
:10A39000C35CD040C752DF4F28813981C95DD040AE
:10A3A000021B130BCD53DF4F19830883C35CD040CE
:10A3B000C953DF4F288139814A815B81C75CD04016
:10A3C000CA01B9010E941FA08111F5C2C553DF4F18
:10A3D0000881CB5CD040002369F0CF52DF4F388238
:10A3E000C15DD04001E0C752DF4F0883C95DD04056
:10A3F000412C0FC044244A94430C1FEFC752DF4F37
:10A400001883C95DD0400FEFCF52DF4F0883C15D85
:10A41000D04081E0C553DF4F1881CB5CD040182776
:10A42000C553DF4F1883CB5CD040C3010196880F22
:10A43000991F880F991F0DE310E00C0F1D1F080FC7
:10A44000191FC954DF4F19830883C75BD040C3511C
:10A45000DF4F08811981CD5ED04001501109CB50EA
:10A46000DF4F19830883C55FD040C554DF4F888113
:10A470009981CB5BD040092E000CAA0BBB0BC950B5
:10A48000DF4F88839983AA83BB83C75FD040C151C4
:10A49000DF4F08811981CF5ED04001501109C550AE
:10A4A000DF4F19830883CB5FD040C554DF4F08814D
:10A4B0001981CB5BD040000F111FC350DF4F1983B0
:10A4C0000883CD5FD040CF52DF4F1881C15DD040AF
:10A4D000411609F45FC2C154DF4F88819981CF5B77
:10A4E000D040CB50DF4F68817981C55FD0400E945A
:10A4F0004FA0072E000C880B990B0E9446996B0108
:10A500007C01C950DF4F688179818A819B81C75F57
:10A51000D0400E9446999B01AC01C701B6010E9440
:10A52000A5999B01AC01CC51DF4F688179818A816B
:10A530009B81C45ED0400E94739D4B015C01CD5352
:10A54000DF4F88819981C35CD040C550DF4F68815F
:10A550007981CB5FD0400E944FA0072E000C880B62
:10A56000990B0E9446996B017C01642D042C000C10
:10A57000770B880B990B0E9446999B01AC01C70190
:10A58000B6010E94A5999B01AC01C851DF4F6881BB
:10A5900079818A819B81C85ED0400E94739D6B0146
:10A5A0007C0120E030E0A901C501B4010E9440997E
:10A5B00087FD05C020E030E040E05FE303C020E01D
:10A5C00030E0A901C501B4010E94739D0E94E89E7C
:10A5D000C355DF4F688379838A839B83CD5AD040EC
:10A5E00020E030E0A901C701B6010E94409987FD33
:10A5F00005C020E030E040E05FE303C020E030E051
:10A60000A901C701B6010E94739D0E94E89EC7552B
:10A61000DF4F688379838A839B83C95AD0401FEFB9
:10A62000611A710AC350DF4FE881F981CD5FD040D4
:10A63000E40DF11D47FCFA95EE0FFF1F21EA30E013
:10A640002C0F3D1FE20FF31F71826082C153DF4F59
:10A650002881CF5CD040452DBE0167557F4FCE018C
:10A6600083559F4F0E949331C953DF4F688379838D
:10A670008A839B83C75CD0409B01AC010E941FA0D2
:10A68000882341F0C352DF4F0881CD5DD040009355
:10A69000170480C1C953DF4F288139814A815B810A
:10A6A000C75CD040C052DF4F688179818A819B812D
:10A6B000C05ED0400E94739DC052DF4F6883798393
:10A6C0008A839B83C05ED040F301EE0FFF1FEE0F25
:10A6D000FF1F2DE630E02C0F3D1FE20FF31FC95383
:10A6E000DF4F88819981AA81BB81C75CD04080837C
:10A6F0009183A283B383C355DF4F88809980AA805A
:10A70000BB80CD5AD040C954DF4FA881B981C75B07
:10A71000D0408D929D92AD92BC921397C755DF4F5A
:10A72000C880D980EA80FB80C95AD040FD01CD5055
:10A73000DF4F08811981C35FD040E00FF11FC08255
:10A74000D182E282F382FD01CF50DF4F088119816F
:10A75000C15FD040E00FF11F80E090E0A0E8BFE3D0
:10A7600080839183A283B383A501940169817A8157
:10A770008B819C810E94739D69837A838B839C83E8
:10A78000A70196016D817E818F8198850E94739DBE
:10A790006D837E838F839887C953DF4F28813981EA
:10A7A0004A815B81C75CD04069857A858B859C85B1
:10A7B0000E94739D69877A878B879C87A501940186
:10A7C000C501B4010E94A5999B01AC016D857E85F0
:10A7D0008F8598890E94739D6D877E878F87988B60
:10A7E000A7019601C701B6010E94A5999B01AC0182
:10A7F00069897A898B899C890E94739D698B7A8B80
:10A800008B8B9C8BC953DF4F288139814A815B81B7
:10A81000C75CD040CA01B9010E94A5999B01AC0157
:10A820006D897E898F89988D0E94739D6D8B7E8B3B
:10A830008F8B988FA7019601C501B4010E94A5993D
:10A840009B01AC01698D7A8D8B8D9C8D0E94739DCF
:10A85000698F7A8F8B8F9C8FC953DF4F2881398105
:10A860004A815B81C75CD040C501B4010E94A599B3
:10A870009B01AC016D8D7E8D8F8D98A10E94739D83
:10A880006D8F7E8F8F8F98A3C953DF4F28813981B9
:10A890004A815B81C75CD040C701B6010E94A5997F
:10A8A0009B01AC0169A17AA18BA19CA10E94739D1F
:10A8B00069A37AA38BA39CA3E894B7F80DA1C35214
:10A8C000DF4F0883CD5DD0401EA1C451DF4F1883F8
:10A8D000CC5ED0400FA118A5C352DF4F2881CD5DBB
:10A8E000D040C451DF4F3881CC5ED040A801C501B3
:10A8F000B4010E94999F18165CF0C352DF4F888004
:10A90000CD5DD040C451DF4F9880CC5ED04058011F
:10A910008DA29EA2AFA2B8A6E894F7F8A9A4BAA403
:10A920000BA51CA59501A801C701B6010E94999F1E
:10A93000181614F065017801C9A6DAA6EBA6FCA6E4
:10A9400020E030E040E85FE369AD7AAD8BAD9CADCF
:10A950000E94739D69AF7AAF8BAF9CAF0E94038E4C
:10A96000C752DF4F0881C95DD040400EC954DF4F48
:10A9700008811981C75BD0400C5F1F4FC954DF4F5E
:10A9800019830883C75BD040C352DF4F1882CD5D67
:10A99000D04099CDC554DF4F08811981CB5BD040A1
:10A9A0000F5F1F4FC554DF4F19830883CB5BD04027
:10A9B000021508F4FDCC80E065D9882341F0C3522C
:10A9C000DF4F1881CD5DD04010931704B3C7C95332
:10A9D000DF4F288139814A815B81C75CD040CA0141
:10A9E000B9010E941FA08111A5C789AC9AACABAC7C
:10A9F000BCAC20E030E0A901C501B4010E9440993F
:10AA0000882309F408C2A501940169817A818B81A8
:10AA10009C810E944F9EC954DF4F688379838A834B
:10AA20009B83C75BD04069837A838B839C83A5011A
:10AA300094016D817E818F8198850E944F9EC554BF
:10AA4000DF4F688379838A839B83CB5BD0406D83A0
:10AA50007E838F839887A501940169857A858B858C
:10AA60009C850E944F9EC154DF4F688379838A83FF
:10AA70009B83CF5BD04069877A878B879C87A501B2
:10AA800094016D857E858F8598890E944F9E6B010C
:10AA90007C01C954DF4F288139814A815B81C75BC2
:10AAA000D040CA01B9010E94A5999B01AC01C70120
:10AAB000B6010E94729DC553DF4F688379838A83F4
:10AAC0009B83CB5CD0406D877E878F87988BA50159
:10AAD000940169897A898B899C890E944F9E6B01B8
:10AAE0007C01C554DF4F288139814A815B81CB5B72
:10AAF000D040CA01B9010E94A5999B01AC01C701D0
:10AB0000B6010E94729DCF52DF4F688379838A839A
:10AB10009B83C15DD040698B7A8B8B8B9C8BA5010D
:10AB200094016D897E898F89988D0E944F9E6B015B
:10AB30007C01C154DF4F288139814A815B81CF5B21
:10AB4000D040CA01B9010E94A5999B01AC01C7017F
:10AB5000B6010E94729D6D8B7E8B8F8B988FA501A5
:10AB60009401698D7A8D8B8D9C8D0E944F9E6B0117
:10AB70007C01C554DF4F288139814A815B81CB5BE1
:10AB8000D040C954DF4F688179818A819B81C75B3E
:10AB9000D0400E94A5999B01AC01C701B6010E945B
:10ABA000729DCD53DF4F688379838A839B83C35C17
:10ABB000D040698F7A8F8B8F9C8FA501940169A1FA
:10ABC0007AA18BA19CA10E944F9E6B017C01C15474
:10ABD000DF4F288139814A815B81CF5BD040C554EA
:10ABE000DF4F688179818A819B81CB5BD0400E9455
:10ABF000A5999B01AC01C701B6010E94729D6B0132
:10AC00007C0169A37AA38BA39CA3A50194016D8DFC
:10AC10007E8D8F8D98A10E944F9E4B015C01C15487
:10AC2000DF4F288139814A815B81CF5BD040C95495
:10AC3000DF4F688179818A819B81C75BD0400E9408
:10AC4000A5999B01AC01C501B4010E94729D4B0105
:10AC50005C016D8F7E8F8F8F98A3CF52DF4F28813D
:10AC600039814A815B81C15DD040C553DF4F688126
:10AC700079818A819B81CB5CD0400E94A5992B0170
:10AC80003C01CD53DF4F288139814A815B81C35C10
:10AC9000D040CA01B9010E94A5999B01AC01C30132
:10ACA000B2010E94729DC752DF4F688379838A8305
:10ACB0009B83C95DD0402B013C01E89477F829A51E
:10ACC0003AA54BA55CA56DA17EA18FA198A50E9478
:10ACD000739D2FEF36EE4BED5EE20E94A5999B012E
:10ACE000AC01C301B2010E94409918160CF093C048
:10ACF000CD53DF4F288139814A815B81C35CD040CD
:10AD0000C701B6010E94A5992B013C01CF52DF4F2C
:10AD1000288139814A815B81C15DD040C501B40180
:10AD20000E94A5999B01AC01C301B2010E94729DD2
:10AD3000C752DF4F288139814A815B81C95DD0408C
:10AD40000E944F9E2B013C016DA77EA78FA798AB59
:10AD5000CD53DF4F288139814A815B81C35CD0406C
:10AD6000C501B4010E94A5994B015C01C553DF4F99
:10AD7000288139814A815B81CB5CD040C701B60113
:10AD80000E94A5999B01AC01C501B4010E94729D6E
:10AD9000C752DF4F288139814A815B81C95DD0402C
:10ADA0000E944F9E6B017C0169AB7AAB8BAB9CAB75
:10ADB000C954DF4F288139814A815B81C75BD0400C
:10ADC000C301B2010E94A5999B01AC01C154DF4FA0
:10ADD000688179818A819B81CF5BD0400E94739D7D
:10ADE0004B015C01C554DF4F288139814A815B8169
:10ADF000CB5BD040C701B6010E94A5999B01AC0175
:10AE0000C501B4010E94739DDC01CB01B0588DAB2C
:10AE10009EABAFABB8AFCDA4DEA4EFA4F8A82601DB
:10AE2000370177FA709477F8709489A89AA8ABA83C
:10AE3000BCA88DA99EA9AFA9B8ADC954DF4F88831E
:10AE40009983AA83BB83C75BD040CB52DF4F088175
:10AE50001981C55DD040B801110F880B990B0E9474
:10AE600046999B01AC01C052DF4F688179818A818C
:10AE70009B81C05ED0400E944F9EC553DF4F6883C8
:10AE800079838A839B83CB5CD040C153DF4F088199
:10AE90001981CF5CD040012B09F461C0EEE9FBE0E1
:10AEA00084918F010F5F1F4F882321F00E94D28B66
:10AEB000F801F6CF48E0C301B2010E94D64AE9E9A1
:10AEC000FBE084918F010F5F1F4F882321F00E94C8
:10AED000D28BF801F6CF48E0C501B40190580E942A
:10AEE000D64AE4E9FBE084918F010F5F1F4F88236E
:10AEF00021F00E94D28BF801F6CFC954DF4F688150
:10AF000079818A819B81C75BD040905848E00E943C
:10AF1000D64A8AE00E94D28BC153DF4F0881198143
:10AF2000CF5CD04003301105D4F0EBE7FBE0849117
:10AF30008F010F5F1F4F882321F00E94D28BF801F1
:10AF4000F6CF48E0C553DF4F688179818A819B81C4
:10AF5000CB5CD0400E94D64A8AE00E94D28BC1527C
:10AF6000DF4F1881CF5DD0401111D1C1CB56DF4FDB
:10AF7000C882D982EA82FB82C559D040C756DF4FCA
:10AF800088829982AA82BB82C959D040C12CD12C17
:10AF900060E8E62E6FE3F62EC356DF4FC882D982F3
:10AFA000EA82FB82CD59D040CE018B569F4F0E9442
:10AFB000366CC757DF4FC882D982EA82FB82C958F4
:10AFC000D040C357DF4F188219821A821B82CD5896
:10AFD000D040CF56DF4F488259826A827B82C15966
:10AFE000D040CE0187579F4F0E94366CCB56DF4F23
:10AFF00088819981AA81BB81C559D040C954DF4F4E
:10B0000088839983AA83BB83C75BD040C756DF4F31
:10B01000488059806A807B80C959D040C356DF4F31
:10B0200088809980AA80BB80CD59D040C757DF4F18
:10B03000088119812A813B81C958D040C554DF4F0E
:10B04000088319832A833B83CB5BD040C357DF4FF0
:10B0500088819981AA81BB81CD58D040C154DF4FEE
:10B0600088839983AA83BB83CF5BD040CF56DF4FC1
:10B07000C880D980EA80FB80C159D040A7019601E1
:10B08000C301B2010E94A599CD53DF4F6883798334
:10B090008A839B83C35CD040C154DF4F28813981B0
:10B0A0004A815B81CF5BD040C501B4010E94A59964
:10B0B0009B01AC01CD53DF4F688179818A819B81EF
:10B0C000C35CD0400E94729DC358DF4F6883798370
:10B0D0008A839B83CD57D040C554DF4F2881398167
:10B0E0004A815B81CB5BD040C501B4010E94A59928
:10B0F0004B015C01A7019601C954DF4F688179813A
:10B100008A819B81C75BD0400E94A5999B01AC01BD
:10B11000C501B4010E94729DCF57DF4F68837983C8
:10B120008A839B83C158D040C154DF4F2881398125
:10B130004A815B81CF5BD040C954DF4F6881798100
:10B140008A819B81C75BD0400E94A5996B017C01DD
:10B15000C554DF4F288139814A815B81CB5BD04068
:10B16000C301B2010E94A5999B01AC01C701B601C0
:10B170000E94729DCB57DF4F688379838A839B83BC
:10B18000C558D040CE0183589F4F0E94366CC75798
:10B19000DF4F088119812A813B81C958D040C357AC
:10B1A000DF4F488059806A807B80CD58D040CF5691
:10B1B000DF4F88809980AA80BB80C159D040C35896
:10B1C000DF4F88819981AA81BB81CD57D040C95476
:10B1D000DF4F88839983AA83BB83C75BD040CF5757
:10B1E000DF4F88819981AA81BB81C158D040C55465
:10B1F000DF4F88839983AA83BB83CB5BD040CB5737
:10B20000DF4F88819981AA81BB81C558D040C15444
:10B21000DF4F88839983AA83BB83CF5BD040CB5613
:10B22000DF4FC880D980EA80FB80C559D040C7561F
:10B23000DF4F488159816A817B81C959D040C3560B
:10B24000DF4F88819981AA81BB81CD59D04000937D
:10B25000400B1093410B2093420B3093430B4092D1
:10B26000440B5092450B6092460B7092470B8092B4
:10B27000480B9092490BA0924A0BB0924B0BC954C9
:10B28000DF4F088119812A813B81C75BD040009341
:10B290004C0B10934D0B20934E0B30934F0BC5541A
:10B2A000DF4F088119812A813B81CB5BD04000931D
:10B2B000500B1093510B2093520B3093530BC154EE
:10B2C000DF4F088119812A813B81CF5BD0400093F9
:10B2D000540B1093550B2093560B3093570BC09281
:10B2E000580BD092590BE0925A0BF0925B0B4093A3
:10B2F0005C0B50935D0B60935E0B70935F0B8093C0
:10B30000600B9093610BA093620BB093630BC252DE
:10B31000DF4F1881CE5DD040112309F46CC2E8EBF9
:10B32000FAE084918F010F5F1F4F882321F00E9464
:10B33000D28BF801F6CFCC24CA94C30CDC2CC554B4
:10B34000DF4F1882CB5BD04000ECC154DF4F088345
:10B35000CF5BD04019E7CD53DF4F1883C35CD0409B
:10B3600004E4C252DF4F0883CE5DD0408E010B56FD
:10B370001F4FCF54DF4F19830883C15BD0400C505F
:10B380001109CD54DF4F19830883C35BD0400C50A3
:10B390001109CB54DF4F19830883C55BD040D7FC1C
:10B3A00029C10D2D000F110BCF52DF4F19830883D8
:10B3B000C15DD040C954DF4F19821882C75BD040AD
:10B3C000312CC954DF4FE881F981C75BD040CF529F
:10B3D000DF4F08811981C15DD040E00FF11F21EAE4
:10B3E00030E02C0F3D1FE20FF31F00811181780127
:10B3F000EE0CFF1CEE0CFF1CEDE6F0E0EC0FFD1F69
:10B40000EE0DFF1D4080518062807380C553DF4F79
:10B41000288139814A815B81CB5CD040C301B20174
:10B420000E94729D4B015C01E1E0F0E0EC0FFD1F1A
:10B43000EE0DFF1D84AD95ADA6ADB7ADCB56DF4F7C
:10B4400088839983AA83BB83C559D040CB52DF4FF1
:10B45000E881F981C55DD040E00FF11FEE0FFF1FBD
:10B46000EE0FFF1F81E090E08C0F9D1FE80FF91F8A
:10B4700084AD95ADA6ADB7ADC757DF4F888399832F
:10B48000AA83BB83C958D040C358DF4F18821982A2
:10B490001A821B82CD57D040CA54DF4F9881C65BB9
:10B4A000D0409F93CB54DF4FA881C55BD040AF9372
:10B4B000CC54DF4FB881C45BD040BF93CD54DF4F35
:10B4C000E881C35BD040EF93CE54DF4FF881C25B7D
:10B4D000D040FF93CF54DF4F0881C15BD0400F9322
:10B4E0002DB73EB7245231090FB6F8943EBF0FBEB8
:10B4F0002DBFADB7BEB71196E0E4FBE084E201904A
:10B500000D928A95E1F70E94516BC358DF4F288155
:10B5100039814A815B81CD57D040C301B2010E947D
:10B52000729D7B018C010FB6F894DEBF0FBECDBFBC
:10B530009B01AC01C554DF4F6881CB5BD040C15447
:10B54000DF4F7881CF5BD040CD53DF4F8881C35C24
:10B55000D040C252DF4F9881CE5DD0400E94999F6B
:10B560001816A4F4C554DF4FE882CB5BD040C15419
:10B57000DF4FF882CF5BD040CD53DF4F0883C35CF1
:10B58000D040C252DF4F1883CE5DD04020E030E083
:10B59000A901C501B4010E94999F87FD0CC0E5EB8C
:10B5A000FAE084918F010F5F1F4F882339F00E94CA
:10B5B000D28BF801F6CF80E20E94D28B45E0C50124
:10B5C000B4010E94D64A3394C954DF4F08811981CF
:10B5D000C75BD0400C5F1F4FC954DF4F19830883EE
:10B5E000C75BD040321408F4ECCE8AE00E94D28BC4
:10B5F000DA94D5CE8AE00E94D28BC153DF4F088106
:10B600001981CF5CD0400430110509F0F4C0ECE89A
:10B61000FAE084918F010F5F1F4F81110CC03E0132
:10B6200015E9610E711C2E0129E8420E511C8E0194
:10B6300003581F4F16C00E94D28BF801EACF80E258
:10B640000E94D28B45E0C501B4010E94D64AD39432
:10B65000F4E0EF0EF11CD214A0F08AE00E94D28B2D
:10B66000CA94C7FCC4C02C2D220F330BC153DF4F2B
:10B6700039832883CF5CD040E12CF12CD12C84E29B
:10B68000382EC153DF4FE881F981CF5CD040EE0DF9
:10B69000FF1D81EA90E08C0F9D1FE80FF91F80814C
:10B6A00091815C01AA0CBB1CAA0CBB1CE1E0F0E080
:10B6B000EC0FFD1FEA0DFB1D44AD55AD66AD77AD3A
:10B6C000D3014D935D936D937C931397CB52DF4FD2
:10B6D000E881F981C55DD040E80FF91FEE0FFF1F2B
:10B6E000EE0FFF1F21E030E02C0F3D1FE20FF31F94
:10B6F00084AD95ADA6ADB7ADF20180839183A283F1
:10B70000B383D8011D921D921D921C9213971F9313
:10B710000F935F924F927F926F92EDB7FEB7B497FF
:10B720000FB6F894FEBF0FBEEDBFADB7BEB7119612
:10B73000E0E4FBE0832D01900D928A95E1F70E94F1
:10B74000516BEDE6F0E0EC0FFD1FEA0DFB1DD8019B
:10B750002D913D914D915C916081718182819381A8
:10B760000E94729DC554DF4F2881CB5BD040C154ED
:10B77000DF4F3881CF5BD040CD53DF4F4881C35C72
:10B78000D040C252DF4F5881CE5DD0400E94729DA2
:10B790004B015C010FB6F894DEBF0FBECDBF20E0B9
:10B7A00030E0A9010E94999F87FD49CFE9E8FAE0BE
:10B7B00084919F012F5F3F4F882309F443CFC150ED
:10B7C000DF4F2883CF5FD040C050DF4F3883C05059
:10B7D000D1400E94D28BC150DF4F2881CF5FD04033
:10B7E000C050DF4F3881C050D140F901E1CF8AE02D
:10B7F0000E94D28B08C0C153DF4F08811981CF5CF2
:10B80000D040012B21F08AE69AE00E940094C152B8
:10B81000DF4F1881CF5DD040111185C08CE0E5E18C
:10B82000FBE0DE01A358BF4F01900D928A95E1F72E
:10B8300081E080931704CE0183589F4F0E94774880
:10B84000C355DF4F288139814A815B81CD5AD04071
:10B850006091150B7091160B8091170B9091180B3E
:10B860000E94729D6B017C012DEB37E346E855EB9E
:10B870000E94999F87FD4BC02DEB37E346E855E3C7
:10B88000C701B6010E94409918160CF440C0C75574
:10B89000DF4F288139814A815B81C95AD04060914C
:10B8A000190B70911A0B80911B0B90911C0B0E942D
:10B8B000729D6B017C012DEB37E346E855EB0E944E
:10B8C000999F87FD24C02DEB37E346E855E3C70178
:10B8D000B6010E9440991816D4F0C953DF4F288151
:10B8E00039814A815B81C75CD04060911D0B7091AA
:10B8F0001E0B80911F0B9091200B0E94729DCB57C5
:10B90000DF4F688379838A839B83C558D0408CE05E
:10B91000FE01E358FF4FA5E1BBE001900D928A952F
:10B92000E1F781E005C0C352DF4F8881CD5DD04093
:10B93000809317040E94264D0E94BB2E809117040D
:10B9400081110E94D087D3950FB6F894DEBF0FBE49
:10B95000CDBFDF91CF911F910F91FF90EF90DF90BE
:10B96000CF90BF90AF909F908F907F906F905F909F
:10B970004F903F902F9008959A014DE15BE00C9419
:10B98000604D9B01AC0169E17BE085E19BE00C949B
:10B99000604D80E1EEE3FAE0A5E1BBE001900D929D
:10B9A0008A95E1F708958F929F92AF92BF92CF92BE
:10B9B000EF92FF920F931F93CF93DF93CDB7DEB734
:10B9C0002C970FB6F894DEBF0FBECDBF4B015C01C4
:10B9D000C0908203EEE3FAE080859185A285B3856D
:10B9E0004481558166817781008111812281338173
:10B9F00009831A832B833C834D835E836F8378870F
:10BA000089879A87AB87BC87AE01475F5F4FBE01CE
:10BA10006B5F7F4FCE0101960E94E649850174015C
:10BA20002AE43AE0AE01475F5F4FBE016B5F7F4F94
:10BA3000CE0101960E94DE3B2C960FB6F894DEBF35
:10BA40000FBECDBFDF91CF911F910F91FF90EF906F
:10BA5000CF90BF90AF909F908F900895CF92DF923C
:10BA6000EF92FF920F931F93CF93DF9394E089029D
:10BA7000E0011124FE01EC5AFC4F20E030E0A90166
:10BA800060817181828193810E94739DFE01EE5CD1
:10BA9000F54F20813181428153810E94739D6B015A
:10BAA0007C01FE01E457FC4F6083718382839383A2
:10BAB000FE01EF5CF54F65917591859194918E0132
:10BAC0000E5F1D4FA70196010E94739DF8016083D0
:10BAD000718382839383FE01E35CF54F65917591D9
:10BAE00085919491CD5BDD4FA70196010E94739DD6
:10BAF000688379838A839B83DF91CF911F910F9114
:10BB0000FF90EF90DF90CF900895EF92FF920F9308
:10BB10001F93CF93DF937C0184E50E94B988D82FCF
:10BB2000882349F10E943788C82F181604F5E5ECE0
:10BB3000FCE184918F010F5F1F4F882321F00E9449
:10BB4000D28BF801F6CF8DE40E94D28BB70180E052
:10BB500090E04AE00E942B8C6C2FCC0F770B8EE18B
:10BB60009AE00E9466678AE00E94D28B08C08093A8
:10BB70003E03D0E004C08091820380933E038D2F6A
:10BB8000DF91CF911F910F91FF90EF9008956091F9
:10BB90001304709114048091150490911604089573
:10BBA0004F925F926F927F928F929F92AF92BF92CD
:10BBB000CF92DF92EF92FF92CF93DF93CDB7DEB7B4
:10BBC0002C970FB6F894DEBF0FBECDBF8091F30364
:10BBD0009091F403A091F503B091F60389839A83C1
:10BBE000AB83BC836091F7037091F803072E000CC0
:10BBF000880B990B0E94469929813A814B815C817F
:10BC00000E94729D6B017C016093D9037093DA03EB
:10BC10008093DB039093DC0320912C0430912D045E
:10BC200040912E0450912F040E94A5996D837E832C
:10BC30008F8398876093D5037093D6038093D7033F
:10BC40009093D8032091D1033091D2034091D30334
:10BC50005091D403C701B6010E94739D4B015C0152
:10BC60006093D1037093D2038093D3039093D40352
:10BC7000209128043091290440912A0450912B04EA
:10BC80000E94A59969877A878B879C876093CD03EB
:10BC90007093CE038093CF039093D00320ED3CECC0
:10BCA0004CE45DE3609124047091250480912604A6
:10BCB000909127040E94A5992B013C012091C90372
:10BCC0003091CA034091CB035091CC0369817A81B2
:10BCD0008B819C810E94729D9B01AC01C301B201CA
:10BCE0000E94A5992B013C0123E333E343E75FE383
:10BCF0006091C5037091C6038091C7039091C803FA
:10BD00000E94A5999B01AC01C301B2010E94739DE1
:10BD10002B013C016093C5037093C6038093C70356
:10BD20009093C80389819A81AB81BC818093C903B8
:10BD30009093CA03A093CB03B093CC0329853A8593
:10BD40004B855C856D817E818F8198850E94739D76
:10BD5000A30192010E94729D2B013C0120E030E082
:10BD60004FE753E40E94999F20E030E0A9011816A4
:10BD7000ACF4C701B6010E94999F18166CF5A70193
:10BD80009601C501B4010E94729D6093D103709326
:10BD9000D2038093D3039093D4031EC0C301B20196
:10BDA0000E94409987FF22C020E030E0A901C7012E
:10BDB000B6010E94409987FF16C0A7019601C501F0
:10BDC000B4010E94729D6093D1037093D20380935B
:10BDD000D3039093D40307C0412C512C8FE7682ED6
:10BDE00083E4782E03C0412C512C3201C301B201EF
:10BDF0002C960FB6F894DEBF0FBECDBFDF91CF916A
:10BE0000FF90EF90DF90CF90BF90AF909F908F907A
:10BE10007F906F905F904F9008952F923F924F9236
:10BE20005F926F927F928F929F92AF92BF92CF92CA
:10BE3000DF92EF92FF92CF93DF9300D01F92CDB7A6
:10BE4000DEB76090FB037090FC0380901304909029
:10BE50001404A0901504B0901604B301072C000C34
:10BE6000880B990B0E944699A50194010E94729D2E
:10BE70006B017C016093C1037093C2038093C30381
:10BE80009093C40320ED3CEC4CE45DE360913004FE
:10BE90007091310480913204909133040E94A599ED
:10BEA0001B012C012091BD033091BE034091BF03C3
:10BEB0005091C003C501B4010E94729D9B01AC0169
:10BEC000C201B1010E94A5991B012C0123E333E3B8
:10BED00043E75FE36091B9037091BA038091BB03BC
:10BEE0009091BC030E94A5999B01AC01C201B101D4
:10BEF0000E94739D69837A838B839C836093B903CB
:10BF00007093BA038093BB039093BC038092BD03EC
:10BF10009092BE03A092BF03B092C00320E030E035
:10BF200040E251E4C701B6010E94999F181624F41B
:10BF300081E08093B80389C020E030E040E251EC1A
:10BF4000C701B6010E94409987FD02C0672821F40D
:10BF500081E08093B8039DC08091B803882351F09D
:10BF60001092B4031092B5031092B6031092B70367
:10BF70001092B803209138043091390440913A046A
:10BF800050913B04C701B6010E94A5992B013C01C9
:10BF90006093B0037093B1038093B2039093B303A3
:10BFA0002091B4033091B5034091B6035091B7038B
:10BFB000C701B6010E94739D4B015C016093B403FD
:10BFC0007093B5038093B6039093B7032091340424
:10BFD0003091350440913604509137040E94A59960
:10BFE0009B01AC016093AC037093AD038093AE03EF
:10BFF0009093AF03C301B2010E94739D29813A81DE
:10C000004B815C810E94729D2B013C0120E030E05D
:10C010004FE753E40E94999F20E030E0A9011816F1
:10C02000DCF4C701B6010E94999F181674F4A701A9
:10C030009601C501B4010E94729D6093B403709390
:10C04000B5038093B6039093B703412C512C8FE72F
:10C05000682E83E4782E20C0C301B2010E9440996B
:10C0600087FF1AC020E030E0A901C701B6010E9495
:10C07000409987FF0EC0A7019601C501B4010E9437
:10C08000729D6093B4037093B5038093B60390934D
:10C09000B703412C512C3201C301B2010F900F9014
:10C0A0000F900F90DF91CF91FF90EF90DF90CF90A6
:10C0B000BF90AF909F908F907F906F905F904F90C8
:10C0C0003F902F9008956091F3037091F403809155
:10C0D000F5039091F6030895AF92BF92CF92DF924D
:10C0E000EF92FF920F931F93CF93DF931F92CDB7E1
:10C0F000DEB77C016B018A0159018091A109811190
:10C1000019C0F701808191810E94F69C8983F60114
:10C1100081936F01BE016F5F7F4FC5010E94BD34E7
:10C12000F701408151814F5F5F4F51834083015040
:10C13000110939F70F90DF91CF911F910F91FF9067
:10C14000EF90DF90CF90BF90AF9008958F929F9225
:10C15000AF92BF92CF92DF92EF92FF920F931F9315
:10C16000CF93DF931F921F92CDB7DEB7E091A10965
:10C17000E1114AC059016C018B017B01E40EF51EEF
:10C180000E151F0509F440C0F60180809180F8016A
:10C1900061918F016983C4016A830E94F69C6A8160
:10C1A000681729F1C4010E94FE9CC4010E94F69CFC
:10C1B00099818917E1F0E5ECFCE184918F010F5F33
:10C1C0001F4F882321F00E94D28BF801F6CFE2EDB9
:10C1D000FEE084918F010F5F1F4F882321F00E94A2
:10C1E000D28BF801F6CF81E08093A1090DC0BE018A
:10C1F0006F5F7F4FC5010E94BD34F6018081918140
:10C20000019691838083BCCF0F900F90DF91CF91E7
:10C210001F910F91FF90EF90DF90CF90BF90AF9064
:10C220009F908F9008950E947F790E94E9790E94E3
:10C23000738F80E013DC81E011DC82E00FDC809101
:10C24000010B9091020BA091030BB091040B809312
:10C25000270290932802A0932902B0932A020C94FB
:10C2600022722F923F924F925F926F927F928F92A3
:10C270009F92AF92BF92CF92DF92EF92FF920F9375
:10C280001F93CF93DF93EC0143E65CE081E090E005
:10C29000FA0125913491C217D3070CF05DC09C01BF
:10C2A00021503109220F331F220F331FD901AF59FB
:10C2B000B34FFD0165917491215A334FF901A59057
:10C2C000B490FC01EE0FFF1FEE0FFF1FEF59F34F6D
:10C2D000E590F490FD01C590D490FA010591149178
:10C2E000F90125903490072E000C880B990B0E94C1
:10C2F00046992B013C01CA19DB09BE01DD0F880BF1
:10C30000990B0E9446994B015C01B7016C197D099C
:10C31000072E000C880B990B0E9446999B01AC01DB
:10C32000C501B4010E94A5996B017C01B801621995
:10C330007309072E000C880B990B0E9446999B01EC
:10C34000AC01C701B6010E944F9E9B01AC01C30125
:10C35000B2010E94739D11C001964C5F5F4F803205
:10C36000910509F095CFEDEDFCE065917491072EF4
:10C37000000C880B990B0E944699DF91CF911F9179
:10C380000F91FF90EF90DF90CF90BF90AF909F9074
:10C390008F907F906F905F904F903F902F90089577
:10C3A000CF92DF92EF92FF92C090F303D090F4030C
:10C3B000E090F503F090F6038091F7039091F80375
:10C3C0000897BC01990F880B990B0E9446999B0115
:10C3D000AC01C701B6010E94409987FF1FC020E051
:10C3E00030E040E050E4C701B6010E94739D0E9416
:10C3F000BC9E7093F2036093F1030E94728BDC0188
:10C40000CB01805A9541AF4FBF4F8093ED0390937E
:10C41000EE03A093EF03B093F00308C01092ED0376
:10C420001092EE031092EF031092F003FF90EF9042
:10C43000DF90CF900895CF92DF92EF92FF92C0905D
:10C440001304D0901404E0901504F0901604809129
:10C45000FB039091FC030D97BC01990F880B990B7E
:10C460000E9446999B01AC01C701B6010E94409908
:10C4700087FF1FC020E030E040E050E4C701B60174
:10C480000E94739D0E94BC9E7093EC036093EB032B
:10C490000E94728BDC01CB01805E914BAF4FBF4F8E
:10C4A0008093E7039093E803A093E903B093EA0332
:10C4B00008C01092E7031092E8031092E90310926B
:10C4C000EA03FF90EF90DF90CF9008951092FC0365
:10C4D0001092FB0380E0AFDF1092F8031092F70395
:10C4E0005FDF0E945D9180E0A6DF109211047598D5
:10C4F0001092F8031092F70310920F04A598089574
:10C500002F923F924F925F926F927F928F929F9263
:10C51000AF92BF92CF92DF92EF92FF920F931F9351
:10C52000CF93DF93EC0148E65DE081E090E0FA0113
:10C5300025913491C217D3070CF05DC09C012150A6
:10C540003109220F331F220F331FD901AA59B24FCD
:10C55000FD01659174912C59324FF901A590B49069
:10C56000FC01EE0FFF1FEE0FFF1FEA59F24FE5909F
:10C57000F490FD01C590D490FA0105911491F90150
:10C5800025903490072E000C880B990B0E94469939
:10C590002B013C01CA19DB09BE01DD0F880B990B89
:10C5A0000E9446994B015C01B7016C197D09072E69
:10C5B000000C880B990B0E9446999B01AC01C501A8
:10C5C000B4010E94A5996B017C01B801621973093D
:10C5D000072E000C880B990B0E9446999B01AC0119
:10C5E000C701B6010E944F9E9B01AC01C301B2017D
:10C5F0000E94739D11C001964C5F5F4F8A33910575
:10C6000009F095CFEAE4FEE065917491072E000CE5
:10C61000880B990B0E944699DF91CF911F910F9142
:10C62000FF90EF90DF90CF90BF90AF909F908F9052
:10C630007F906F905F904F903F902F90089560E0B3
:10C640008091FD039091FE030CDE609313047093C0
:10C65000140480931504909316048091F90390912B
:10C66000FA034EDF6093F3037093F4038093F503B2
:10C670009093F603A8958FB7F8941092FF038FBF9D
:10C680000895CF92DF92FF920F931F93CF93DF9382
:10C690001F921F92CDB7DEB7F82E8A01809121023A
:10C6A000882309F444C0EBECF9E084916F019FEF1B
:10C6B000C91AD90A882341F069837A830E94D28BF0
:10C6C000F60169817A81F1CFFB0184916F019FEFBF
:10C6D000C91AD90A882321F00E94D28BF601F5CF1E
:10C6E000E3E0FDE084916F019FEFC91AD90A882326
:10C6F00021F00E94D28BF601F5CFF7FC0BC06F2D15
:10C70000FF0C770B880B990B0E94BA4A8AE00E94B3
:10C71000D28B0DC0EEEFFCE084916F019FEFC91A40
:10C72000D90A882321F00E94D28BF601F5CF80919F
:10C73000AB03811108C01092210281E08093AB030A
:10C74000C8010E94D58D0F900F90DF91CF911F915E
:10C750000F91FF90DF90CF90B9CE8F3F29F08823C3
:10C7600031F042EB5EE005C04FE85EE002C042EC13
:10C770005EE060EA7EE085CF8F3F29F0882331F0CC
:10C780004FE65EE005C04CE45EE002C04FE75EE0CD
:10C790006DE57EE076CF1F920F920FB60F921124B7
:10C7A0000BB60F921F932F933F934F935F936F930B
:10C7B0007F938F939F93AF93BF93CF93DF93EF9329
:10C7C000FF9380911204811128C181E080931204AB
:10C7D00080916E008B7F80936E007894809126020A
:10C7E0008F3790F08F5790911104909310049923F4
:10C7F00011F0759A01C0759890910F0490930E04F2
:10C80000992359F0A59A0AC090911004891708F04D
:10C81000759890910E04891708F0A5988F5F809302
:10C82000260290910D0481E0892780930D04809168
:10C830002502823079F1A0F4882341F1813009F09A
:10C8400042C080917800909179002091020430914B
:10C850000304820F931F909303048093020433C058
:10C86000833019F1843079F580910C04811103C073
:10C8700086E080930C0480910C04815080930C041A
:10C88000882309F183E0809325021DC010927B006C
:10C8900080E403C010927B0082E480937C0080914E
:10C8A0007A00806480937A000EC080917800909125
:10C8B00079002091000430910104820F931F90931E
:10C8C0000104809300041091250211115AC0909127
:10C8D00024029F5F90311CF49093240252C0109266
:10C8E00024028091FF03811113C080910204909172
:10C8F00003049093FE038093FD03809100049091C4
:10C9000001049093FA038093F90381E08093FF037D
:10C910008AE0E2E0F4E0DF011D928A95E9F71092E7
:10C92000010410920004C091FD03D091FE03D19543
:10C93000C195D10980914A0390914B0391958195BE
:10C9400091098C179D077CF1809110029091110242
:10C95000919581959109C817D9079CF1C091F90368
:10C96000D091FA0380914803909149038C179D0759
:10C97000B4F580910E0290910F02C817D9070CF000
:10C980003DC0812F90E0019665E070E00E944FA0CD
:10C9900080932502F8941092120480916E008460B6
:10C9A00080936E003AC08091FB039091FC031816AF
:10C9B000190654F642EC5EE060EA7EE080E061DE5B
:10C9C000C3CF8091FB039091FC031816190634F62F
:10C9D0004FE75EE06DE57EE080E053DEBFCF809103
:10C9E000F7039091F803181619060CF0C2CF4FE820
:10C9F0005EE060EA7EE08FEF44DEBBCF8091F7031C
:10CA00009091F803181619060CF0BBCF4CE45EE0C9
:10CA10006DE57EE08FEF35DEB4CFFF91EF91DF91D2
:10CA2000CF91BF91AF919F918F917F916F915F91C6
:10CA30004F913F912F911F910F900BBE0F900FBE02
:10CA40000F901F9018954F925F926F927F92AF92C6
:10CA5000BF92CF92DF92EF92FF920F931F93CF93EB
:10CA6000DF9300D01F92CDB7DEB78091FF03811115
:10CA700013C00F900F900F900F90DF91CF911F91E7
:10CA80000F91FF90EF90DF90CF90BF90AF907F908D
:10CA90006F905F904F900895D2DD0E94728B6983F2
:10CAA0007A838B839C8380912202909123021816B3
:10CAB00019060CF0F1C00197909323028093220293
:10CAC0004090130450901404609015047090160464
:10CAD0006091FB037091FC03072E000C880B990BEF
:10CAE0000E9446995EE1A52EB12CC12CD12C7B0170
:10CAF0008C01A301920163EE73E082EE93E00E9449
:10CB0000719160914C0370914D03072E000C880BBE
:10CB1000990B0E944699A30192010E94409987FFB8
:10CB200017C06091120270911302072E000C880B3F
:10CB3000990B0E944699A30192010E94999F181691
:10CB40003CF480E06AD90E94B79E7595679501C054
:10CB500060E0609311048091E7039091E803A09155
:10CB6000E903B091EA030097A105B10521F12981FC
:10CB70003A814B815C81281B390B4A0B5B0B57FDBB
:10CB80001AC005D86B017C018091EB039091EC03F6
:10CB9000BC0180E090E00E9444999B01AC01C70178
:10CBA000B6010E94409987FF98C042E55DE063E4CA
:10CBB0007DE080E066DD8091ED039091EE03A09131
:10CBC000EF03B091F0030097A105B10521F1498071
:10CBD0005A806B807C80481A590A6A0A7B0A77FC63
:10CBE0001AC071DA2B013C018091F1039091F2039C
:10CBF000BC0180E090E00E9444999B01AC01C3011C
:10CC0000B2010E94409987FF66C041E25DE064E3A3
:10CC10007DE08FEF36DD4090F3035090F403609099
:10CC2000F5037090F6038091F7039091F803BC012F
:10CC3000990F880B990B0E9446992AE0A22EB12CDD
:10CC4000CC24CA94DC2C7B018C01A30192016DEDF4
:10CC500073E081EE93E00E94719120E030E040EAC1
:10CC600050E4C301B2010E94999F87FD11C020E0EA
:10CC700030E046E153E4C301B2010E944099181626
:10CC80003CF00E94D05D0E94B79E7595679501C0EB
:10CC900060E060930F04EDCE4090130450901404B4
:10CCA000609015047090160420E030E848E953E4E1
:10CCB000C301B2010E94999F181694F020E030E061
:10CCC00040EA50E4C301B2010E94409987FF00CFBF
:10CCD00080E052DDFDCE64DB9ECF80E0ACDB6BCF2D
:10CCE00080E03BDDEBCFCF93DF93E0EFFCE084917E
:10CCF000EF012196882321F00E94D28BFE01F7CF0D
:10CD0000ECEEFCE08491EF012196882321F00E9453
:10CD1000D28BFE01F7CF62B36695617070E080E060
:10CD200090E00E94BA4A62B3617070E080E090E0E7
:10CD30000E94BA4A8AE00E94D28BE8EEFCE084911D
:10CD4000EF012196882321F00E94D28BFE01F7CFBC
:10CD500060910601862F660F990BAA0BBB0BBC01D5
:10CD6000CD01662797FD63957727882799270E942D
:10CD7000BA4A62B362FB662760F970E080E090E037
:10CD80000E94BA4A8AE00E94D28BE4EEFCE08491D1
:10CD9000EF012196882321F00E94D28BFE01F7CF6C
:10CDA0006091060166FB662760F970E080E090E024
:10CDB0000E94BA4A6091060165FB662760F970E03F
:10CDC00080E090E00E94BA4A8AE00E94D28BEFEDA8
:10CDD000FCE08491EF012196882321F00E94D28B00
:10CDE000FE01F7CF6091060163FB662760F970E0F2
:10CDF00080E090E00E94BA4A6091060162956170FD
:10CE000070E080E090E00E94BA4A8AE0DF91CF9122
:10CE10000C94D28B643079F028F4613041F06230A8
:10CE200041F00895683051F0603141F0089540E0DC
:10CE300003C040E004C041E060E002C041E061E0C6
:10CE40000C946471CF92DF92EF92FF92CF93DF93B5
:10CE50006A017B01FC018491EF012196882321F076
:10CE60000E94D28BFE01F7CF42E0C701B601DF91ED
:10CE7000CF91FF90EF90DF90CF900C94D64A0F9314
:10CE80001F93CF93DF9300D01F92CDB7DEB7FC0185
:10CE900084918F010F5F1F4F882361F049835A836C
:10CEA0006B837C830E94D28BF80149815A816B810C
:10CEB0007C81EECFCB01BA010F900F900F900F90B5
:10CEC000DF91CF911F910F910C94BA4A0F931F934A
:10CED000CF93DF938B01FC018491EF01219688238E
:10CEE00021F00E94D28BFE01F7CFB801110F880B01
:10CEF000990BDF91CF911F910F910C94BA4A0F9328
:10CF00001F93CF93DF931F921F92CDB7DEB7FC0123
:10CF100084918F010F5F1F4F811102C08B0108C0E8
:10CF200069837A830E94D28BF80169817A81F0CF7C
:10CF3000F80181918F01882319F00E94D28BF8CFDC
:10CF40000F900F90DF91CF911F910F9108952F9225
:10CF50003F924F925F926F927F928F929F92AF9289
:10CF6000BF92CF92DF92EF92FF920F931F93CF93D6
:10CF7000DF93CDB7DEB7EC970FB6F894DEBF0FBEE8
:10CF8000CDBFFC018081813009F469C21A018B0197
:10CF9000823009F02CC180E090E0A4E3B2E4898BF8
:10CFA0009A8BAB8BBC8B80E090E0ACE2B3E48D8BD2
:10CFB0009E8BAF8BB88F80E090E0A0E0BFEB898FB5
:10CFC0009A8FAB8FBC8F80E090E0A0ECBFE78D8F95
:10CFD0009E8FAF8FB8A3FB018081882309F43FC2E5
:10CFE0004090190B50901A0B60901B0B70901C0B0B
:10CFF00060911D0B70911E0B80911F0B9091200B67
:10D00000C090210BD090220BE090230BF090240BCA
:10D010008090150B9090160BA090170BB090180BEA
:10D0200089829A82AB82BC824D825E826F827886D0
:10D0300069877A878B879C87CD86DE86EF86F88A1C
:10D0400020E030E040E05FEB0E94999F19A21AA215
:10D050001BA21CA287FD17C0AE014F5D5F4FBE0132
:10D060006B5E7F4FCE0141960E94BC5C19A21AA252
:10D070001BA21CA2BE016F5D7F4FCE0149960E948C
:10D08000C15CD12C63C0BE016F5D7F4FCE0149965C
:10D090000E94C15C19A21AA21BA21CA2AE014F5D84
:10D0A0005F4FBE016B5E7F4FCE0141960E94BC5C1C
:10D0B000E8CFB7010F2C000C880B990B0E94469902
:10D0C00026E331E642E85DE30E94A5994B015C014D
:10D0D0000E94D49FF1014080518062807380A3013F
:10D0E00092010E94A59920E030E044E352E40E94BE
:10D0F000739D6DAB7EAB8FAB98AFC501B4010E9441
:10D100004C9EA30192010E94A59920E030E04CE2E0
:10D1100053E40E94739D69AB7AAB8BAB9CAB19A2B5
:10D120001AA21BA21CA2AE014F5D5F4FBE016F5C35
:10D130007F4FCE01C5960E94BC5CFFEFEF1AFF0A3D
:10D140008AE0E816F10409F0B4CFD394F8018081A5
:10D15000D81618F4E12CF12CACCF19A21AA21BA2FC
:10D160001CA2AE014F5D5F4FBE016B5E7F4FCE01D3
:10D1700041960E94BC5C29853A854B855C85698D0A
:10D180007A8D8B8D9C8D0E94409919A21AA21BA2A8
:10D190001CA21816B4F0BE016F5D7F4FCE01099638
:10D1A0000E94C15C19A21AA21BA21CA2AE014F5D73
:10D1B0005F4FBE016B5F7F4FCE0101960E94BC5C4A
:10D1C0004EC1AE014F5D5F4FBE016B5F7F4FCE0121
:10D1D00001960E94BC5C19A21AA21BA21CA2BE014D
:10D1E0006F5D7F4FCE0109960E94C15C38C180E01F
:10D1F00090E0A6EEB2E489A39AA3ABA3BCA3C12C92
:10D20000D12C5CE2E52E53E4F52ECDA2DEA2EFA2F6
:10D21000F8A640E050E060E07FEB49A75AA76BA773
:10D220007CA780E090E0A0ECBFE78DA79EA7AFA70A
:10D23000B8AB812C912CE4E3AE2EE2E4BE2E898AB9
:10D240009A8AAB8ABC8ACD8ADE8AEF8AF88E498FA9
:10D250005A8F6B8F7C8F8D8F9E8FAF8FB8A3C090AE
:10D26000190BD0901A0BE0901B0BF0901C0B409107
:10D270001D0B50911E0B60911F0B7091200B809124
:10D28000210B9091220BA091230BB091240B809045
:10D29000150B9090160BA090170BB090180B89826D
:10D2A0009A82AB82BC82CD82DE82EF82F886498789
:10D2B0005A876B877C878D879E87AF87B88B19AE1F
:10D2C0001AAE1BAE1CAE812C912CF9E3AF2EF3E409
:10D2D000BF2E8DAA9EAAAFAAB8AEC12CD12CE12C2C
:10D2E000A0E4FA2EC9AADAAAEBAAFCAAAE01475C0E
:10D2F0005F4FBE016B5C7F4FCE01C1960E94BC5C4C
:10D3000019AE1AAE1BAE1CAE80E090E0AEE3B3E403
:10D310008DAB9EABAFABB8AFC9AADAAAEBAAFCAA99
:10D32000AE01475C5F4FBE016B5C7F4FCE01C19683
:10D330000E94BC5C19AE1AAE1BAE1CAE8DAA9EAA92
:10D34000AFAAB8AEC9AADAAAEBAAFCAAAE01475C9A
:10D350005F4FBE016B5C7F4FCE01C1960E94BC5CEB
:10D3600019AE1AAE1BAE1CAE8DAA9EAAAFAAB8AE5D
:10D3700080E090E0A0E4B0EC89AB9AABABABBCAB87
:10D38000AE01475C5F4FBE016B5C7F4FCE01C19623
:10D390000E94BC5C19AE1AAE1BAE1CAE8DAA9EAA32
:10D3A000AFAAB8AEC9AADAAAEBAAFCAAAE01475C3A
:10D3B0005F4FBE016B5C7F4FCE01C1960E94BC5C8B
:10D3C00019AA1AAA1BAA1CAAAE014F5C5F4FBE0184
:10D3D0006B5E7F4FCE0141960E94BC5C19AA1AAACF
:10D3E0001BAA1CAABE016F5C7F4FCE0149960E940A
:10D3F000C15CF12C2F2D30E0F801808190E09595F3
:10D40000879519AA1AAA1BAA1CAA28173907D4F4A7
:10D41000AE014F5C5F4FBE016B5D7F4FCE018196C9
:10D420000E94BC5C19AA1AAA1BAA1CAAAE014F5CD6
:10D430005F4FBE016B5E7F4FCE0141960E94BC5C88
:10D44000F394D8CF9E012F5C3F4FAE01475F5F4FF3
:10D45000BE016B5F7F4FCE0101960E94604DEC963E
:10D460000FB6F894DEBF0FBECDBFDF91CF911F91F5
:10D470000F91FF90EF90DF90CF90BF90AF909F9073
:10D480008F907F906F905F904F903F902F90089576
:10D49000AF92BF92CF92DF92EF92FF920F931F93C2
:10D4A000CF93DF93A0909304B0909404F501828110
:10D4B0009381A481B581181619061A061B06C4F5B6
:10D4C00080919204409191046091900480FF14C077
:10D4D00083B1829586958695837091E08927282F60
:10D4E00021704E7F242B209391046170262301F13B
:10D4F0008091000B816018C086B150E0082E000CAE
:10D50000990B80959095990F880B982F84279527D4
:10D5100080719927482759274093910460714623C9
:10D5200039F08091000B80618093000B80E09CD7E4
:10D53000F50186819781A085B185181619061A060E
:10D540001B060CF046C090919204809191042091AA
:10D55000900491FF1EC033B190E03295369537703C
:10D5600041E0342730FBCC24C0F8D12CD194C194B5
:10D57000D108C826D926F2E0CF22DD24C826D92634
:10D58000C09291042270C22221F18091000B82602E
:10D590001CC030B190E03695369541E0342730FB21
:10D5A000EE24E0F8F12CF194E194F108E826F92654
:10D5B00030E2E322FF24E826F926E092910420726B
:10D5C000E22239F08091000B80628093000B81E0B1
:10D5D0004BD7F50182859385A485B5851816190664
:10D5E0001A061B060CF04EC0909192048091910493
:10D5F00092FF25C090915303992309F443C093B13E
:10D60000482F50E0892F82958F7091E08927082F4D
:10D61000017010E088279927801B910B842795279C
:10D6200084709927842795278093910420919004F2
:10D630002470822339F18091000B84601FC090B167
:10D64000282F30E0892F869591E089278170C82F97
:10D65000F0E0DF2F882799278C1B9D0B82279327CB
:10D660008074992782279327809391049091900446
:10D670009074892339F08091000B80648093000BB3
:10D6800082E0F2D68091910480939004DF91CF9153
:10D690001F910F91FF90EF90DF90CF90BF90AF90D0
:10D6A00008954F925F926F927F928F929F92AF9266
:10D6B000BF92CF92DF92EF92FF92CF93DF93CDB7DD
:10D6C000DEB728970FB6F894DEBF0FBECDBF249605
:10D6D000AEADBFAD24978D919D910D90BC91A02DC5
:10D6E00089839A83AB83BC832296EEADFFAD2297EC
:10D6F000C080D180E280F380AEADBFAD8D909D90B3
:10D70000AD90BC902E8D3F8D48A159A1C501B401AB
:10D710000E94A5992B013C012AA53BA54CA55DA51E
:10D72000C701B6010E94A5999B01AC01C301B201DA
:10D730000E94739D2B013C012EA93FA948AD59AD14
:10D7400069817A818B819C810E94A5999B01AC01A2
:10D75000C301B2010E94739D6D837E838F8398877E
:10D760002AA13BA14CA15DA1C501B4010E94A599CC
:10D770002B013C012EA53FA548A959A9C701B60117
:10D780000E94A5999B01AC01C301B2010E94739D47
:10D790002B013C012AAD3BAD4CAD5DAD69817A8179
:10D7A0008B819C810E94A5999B01AC01C301B201B0
:10D7B0000E94739D2B013C012A8D3B8D4C8D5D8D0C
:10D7C000C501B4010E94A5994B015C012EA13FA1A6
:10D7D00048A559A5C701B6010E94A5999B01AC01B6
:10D7E000C501B4010E94739D6B017C012AA93BA96C
:10D7F0004CA95DA969817A818B819C810E94A59940
:10D800009B01AC01C701B6010E94739DEEADFFAD57
:10D8100060837183828393838D819E81AF81B8857C
:10D820002296EEADFFAD229780839183A283B383CE
:10D830002496AEADBFAD24974D925D926D927C92D1
:10D84000139728960FB6F894DEBF0FBECDBFDF91B9
:10D85000CF91FF90EF90DF90CF90BF90AF909F90CF
:10D860008F907F906F905F904F9008954F925F924E
:10D870006F927F928F929F92AF92BF92CF92DF92E0
:10D88000EF92FF920F931F93CF93DF9300D01F92DD
:10D89000CDB7DEB78C01DC014D905D906D907C9032
:10D8A000139714968D909D90AD90BC9017971896F5
:10D8B0008D919D910D90BC91A02D89839A83AB830E
:10D8C000BC83A3019201C301B2010E94A5996B011F
:10D8D0007C01A5019401C501B4010E94A5999B0199
:10D8E000AC01C701B6010E94739D6B017C012981C7
:10D8F0003A814B815C81CA01B9010E94A5999B01C3
:10D90000AC01C701B6010E94739D0E94DE9F9B017E
:10D91000AC0160E070E080E89FE30E944F9E6B01E5
:10D920007C019B01AC01C301B2010E94A599F801E1
:10D930006083718382839383A7019601C501B4013B
:10D940000E94A599D80114966D937D938D939C9315
:10D950001797A701960169817A818B819C810E942A
:10D96000A599F80160877187828793870F900F9040
:10D970000F900F90DF91CF911F910F91FF90EF903B
:10D98000DF90CF90BF90AF909F908F907F906F90DF
:10D990005F904F9008951F920F920FB60F9211242F
:10D9A0000BB60F922F933F934F935F936F937F9399
:10D9B0008F939F93AF93BF93EF93FF9380918C04CA
:10D9C00090918D04A0918E04B0918F04892B8A2BA5
:10D9D0008B2B59F180918B04E0918904F0918A049A
:10D9E00090818927808380918C0490918D04A091EF
:10D9F0008E04B0918F04181619061A061B060CF037
:10DA000056C080918C0490918D04A0918E04B091A9
:10DA10008F040197A109B10980938C0490938D0420
:10DA2000A0938E04B0938F0442C080912B02E2E554
:10DA3000F1E1E4919FEF90932B02E230C9F050F4B2
:10DA4000EE2399F0E13081F590916F009D7F9093E6
:10DA50006F002AC0E43019F1E0F0E53029F590912B
:10DA600073009D7F909373001FC010926E001CC0C6
:10DA7000909170009D7F9093700091E09093B00022
:10DA80009091B100987F94609093B1001092B30090
:10DA90000BC0909171009D7F9093710005C0909193
:10DAA00072009D7F9093720060E00E94458AFF9112
:10DAB000EF91BF91AF919F918F917F916F915F9106
:10DAC0004F913F912F910F900BBE0F900FBE0F9073
:10DAD0001F9018950F931F93CF93C82F882319F089
:10DAE000EAE3F1E10CC0E5ECFCE184918F010F5F0A
:10DAF0001F4F8823A9F30E94D28BF801F6CF84919F
:10DB00008F010F5F1F4F882321F00E94D28BF801F5
:10DB1000F6CF8AE00E94D28BC1112CC0E5ECFCE16B
:10DB200084918F010F5F1F4F882321F00E94D28BB9
:10DB3000F801F6CFE7E2F1E184918F010F5F1F4F0B
:10DB4000882321F00E94D28BF801F6CF80918804BF
:10DB5000882321F08AE00E94D28B39C0ECE1F1E108
:10DB600084918F010F5F1F4F882389F10E94D28B10
:10DB7000F801F6CF409184045091850460918604A9
:10DB80007091870483E191E15DD98AE00E94D28B94
:10DB900080918804811127C0CC2319F0E8E0F1E1DD
:10DBA0000CC0E5ECFCE184918F010F5F1F4F8823CF
:10DBB000A9F30E94D28BF801F6CF84918F010F5FF9
:10DBC0001F4F882381F00E94D28BF801F6CFE5EC3D
:10DBD000FCE184918F010F5F1F4F882359F20E944F
:10DBE000D28BF801F6CFC11124C0E5ECFCE18491A1
:10DBF0008F010F5F1F4F882321F00E94D28BF80105
:10DC0000F6CFE7EFF0E184918F010F5F1F4F88237C
:10DC100021F00E94D28BF801F6CFE5ECFCE1849173
:10DC20008F010F5F1F4F882321F00E94D28BF801D4
:10DC3000F6CF4091250B5091260B6091270B7091E8
:10DC4000280B8FEE90E1FED84091290B50912A0BC2
:10DC500060912B0B70912C0B8CEE90E1F3D84091DE
:10DC60002D0B50912E0B60912F0B7091300B89EE84
:10DC700090E1E8D84091310B5091320B6091330B19
:10DC80007091340B86EE90E1DDD88AE00E94D28B51
:10DC9000C11124C0E5ECFCE184918F010F5F1F4F9F
:10DCA000882321F00E94D28BF801F6CFE8ECF0E156
:10DCB00084918F010F5F1F4F882321F00E94D28B28
:10DCC000F801F6CFE5ECFCE184918F010F5F1F4F67
:10DCD000882321F00E94D28BF801F6CF4091740482
:10DCE0005091750460917604709177048FEB90E108
:10DCF000A9D8409178045091790460917A04709188
:10DD00007B048CEB90E19ED840917C0450917D0483
:10DD100060917E0470917F0489EB90E193D84091EB
:10DD2000800450918104609182047091830486EB99
:10DD300090E188D88AE00E94D28BC11124C0E5EC22
:10DD4000FCE184918F010F5F1F4F882321F00E9417
:10DD5000D28BF801F6CFE4E9F0E184918F010F5FF7
:10DD60001F4F882321F00E94D28BF801F6CFE5ECFB
:10DD7000FCE184918F010F5F1F4F882321F00E94E7
:10DD8000D28BF801F6CF4091640450916504609104
:10DD90006604709167048BE890E10E949738409187
:10DDA00068045091690460916A0470916B0488E87A
:10DDB00090E10E94973840916C0450916D046091FD
:10DDC0006E0470916F0485E890E10E94973840914D
:10DDD000700450917104609172047091730482E830
:10DDE00090E10E9497388AE00E94D28BC11124C032
:10DDF000E5ECFCE184918F010F5F1F4F882321F038
:10DE00000E94D28BF801F6CFE8E3F0E184918F0114
:10DE10000F5F1F4F882321F00E94D28BF801F6CFAD
:10DE2000E5ECFCE184918F010F5F1F4F882321F007
:10DE30000E94D28BF801F6CF4091600450916104AA
:10DE400060916204709163048FE290E10E94226706
:10DE500040915C0450915D0460915E0470915F0498
:10DE60008CE290E10E94226740915804509159043D
:10DE700060915A0470915B0489E290E10E942267EC
:10DE80008AE00E94D28BC11124C0E5ECFCE18491B0
:10DE90008F010F5F1F4F882321F00E94D28BF80162
:10DEA000F6CFE5EBFFE084918F010F5F1F4F8823D2
:10DEB00021F00E94D28BF801F6CFE5ECFCE18491D1
:10DEC0008F010F5F1F4F882321F00E94D28BF80132
:10DED000F6CF4091540450915504609156047091CE
:10DEE00057048CEA9FE00E942267409150045091B1
:10DEF0005104609152047091530489EA9FE00E949A
:10DF0000226740914C0450914D0460914E047091F1
:10DF10004F0486EA9FE00E94973840913C0450915C
:10DF20003D0460913E0470913F0483EA9FE00E94AB
:10DF300022674091400450914104609142047091E5
:10DF4000430480EA9FE00E9422674091440450917C
:10DF5000450460914604709147048DE99FE00E945A
:10DF60002267409148045091490460914A0470919D
:10DF70004B048AE99FE00E9422678AE00E94D28BCC
:10DF8000C11124C0E5ECFCE184918F010F5F1F4FAC
:10DF9000882321F00E94D28BF801F6CFECE8FFE055
:10DFA00084918F010F5F1F4F882321F00E94D28B35
:10DFB000F801F6CFE5ECFCE184918F010F5F1F4F74
:10DFC000882321F00E94D28BF801F6CF40915403B0
:10DFD00050915503609156037091570383E89FE079
:10DFE0000E942267409158035091590360915A034F
:10DFF00070915B0380E89FE00E94226740915C0380
:10E0000050915D0360915E0370915F038DE79FE027
:10E010000E9422678AE00E94D28BC11124C0E5ECE5
:10E02000FCE184918F010F5F1F4F882321F00E9434
:10E03000D28BF801F6CFE9E6FFE084918F010F5F04
:10E040001F4F882321F00E94D28BF801F6CFE5EC18
:10E05000FCE184918F010F5F1F4F882321F00E9404
:10E06000D28BF801F6CF6091170470E080E69FE054
:10E070000E9466678AE00E94D28BC11124C0E5EC41
:10E08000FCE184918F010F5F1F4F882321F00E94D4
:10E09000D28BF801F6CFE1E5FFE084918F010F5FAD
:10E0A0001F4F882321F00E94D28BF801F6CFE5ECB8
:10E0B000FCE184918F010F5F1F4F882321F00E94A4
:10E0C000D28BF801F6CF4091380450913904609119
:10E0D0003A0470913B0488E49FE00E9422672CEA96
:10E0E00035EC47E25EE36091340470913504809131
:10E0F0003604909137040E944F9EAB01BC0185E429
:10E100009FE00E94B4382CEA35EC47E25EE3609170
:10E1100030047091310480913204909133040E9454
:10E12000A599AB01BC0182E49FE00E94B4388AE06B
:10E130000E94D28BC1110CC0E5ECFCE184918F01EF
:10E140000F5F1F4F882321F00E94D28BF801F6CF7A
:10E1500040912C0450912D0460912E0470912F0455
:10E1600089E39FE00E9422672CEA35EC47E25EE3F8
:10E17000609128047091290480912A0490912B04C5
:10E180000E944F9EAB01BC0186E39FE00E94B43821
:10E190002CEA35EC47E25EE360912404709125049B
:10E1A00080912604909127040E94A599AB01BC019F
:10E1B00083E39FE00E94B4388AE00E94D28BC111B1
:10E1C00024C0E5ECFCE184918F010F5F1F4F882391
:10E1D00021F00E94D28BF801F6CFEDE1FFE08491AF
:10E1E0008F010F5F1F4F882321F00E94D28BF8010F
:10E1F000F6CFE5ECFCE184918F010F5F1F4F882380
:10E2000021F00E94D28BF801F6CF4091010B509182
:10E21000020B6091030B7091040B84E19FE00E945C
:10E2200022678AE00E94D28BC11124C0E5ECFCE198
:10E2300084918F010F5F1F4F882321F00E94D28BA2
:10E24000F801F6CFEBEFFEE084918F010F5F1F4FD7
:10E25000882321F00E94D28BF801F6CFE5ECFCE197
:10E2600084918F010F5F1F4F882321F00E94D28B72
:10E27000F801F6CF409118045091190460911A04E6
:10E2800070911B0482EF9EE00E94973840911C041D
:10E2900050911D0460911E0470911F048FEE9EE04A
:10E2A0000E949738409120045091210460912204EB
:10E2B000709123048CEE9EE00E9497388AE0CF9103
:10E2C0001F910F910C94D28B67FD44C0813061F097
:10E2D00028F08230D9F0833059F13CC0662311F028
:10E2E000A19A6DC0A1986BC09FB7662329F0F894DE
:10E2F00080910801806804C0F894809108018F77AC
:10E30000809308019FBF47FF35C057C09FB7662362
:10E3100029F0F89480910801806404C0F8948091F9
:10E3200008018F7B809308019FBF47FF29C046C02B
:10E330009FB7662329F0F89480910801886004C093
:10E34000F89480910801877F809308019FBF47FF61
:10E3500027C038C047FD36C0813061F028F08230D8
:10E3600079F08330E9F00895442311F0A09A0895DC
:10E37000A0980895442311F0A29A0895A2980895B0
:10E380009FB7442329F0F89480910801806204C06B
:10E39000F894809108018F7D809308019FBF0895B4
:10E3A0009FB7442329F0F894809108018061F4CF4D
:10E3B000F894809108018F7EEFCF0895089547FF6C
:10E3C000D3CF08950895DB01833070F494E0899FE2
:10E3D000F0011124E85EFB4FAB01770F660B770B62
:10E3E0004083518362837383813089F018F08230D7
:10E3F000D9F008952FEF30E00E946AA020ED37E0B9
:10E4000040E050E00E943D9DB9018EE219C02FEF1F
:10E4100030E00E946AA020ED37E040E050E00E942A
:10E420003D9DB9018DE20CC02FEF30E00E946AA043
:10E4300020ED37E040E050E00E943D9DB9018CE2C4
:10E440000C94748ACF93DF93C8E1D4E0688179811A
:10E4500080E0B9DF6C817D8181E0B5DF68857985F9
:10E4600082E0DF91CF91AFCF24E08202C00111247E
:10E47000FC01EB5FF44F4081518162817381FC01AB
:10E48000EC58FC4F4083518362837383E091930483
:10E49000F091940482899389A489B58980939D0918
:10E4A00090939E09A0939F09B093A0090895CF93DC
:10E4B000DF932FB7F89494E08902E0011124FE0164
:10E4C000EB5FF44F60817181828193812FBF0E9445
:10E4D0004699CC59DC4F288139814A815B810E9461
:10E4E000A599DF91CF9108959091880B8091890B28
:10E4F000981719F00E94038EF7CF08958091920427
:10E500009FB780FF09C0F89480910B018D7F8093A5
:10E510000B019FBF8FEF08C0F89480910B018260C0
:10E5200080930B019FBF81E080932C028091920425
:10E530009FB781FF09C0F89480910B01816080939F
:10E540000B019FBF8FEF08C0F89480910B018E7F65
:10E5500080930B019FBF81E080932D0280919204F4
:10E560009FB782FF09C0F89480910B018B7F809345
:10E570000B019FBF8FEF08C0F89480910B0184605E
:10E5800080930B019FBF81E080932E0280919204C3
:10E590009FB783FF09C0F89480910B01806480933A
:10E5A0000B019FBF8FEF08C0F89480910B018F7B08
:10E5B00080930B019FBF81E080932F02089590917B
:10E5C000880B8091890B981731F08091890B8F5FB0
:10E5D0008F708093890B08951F920F920FB60F9240
:10E5E00011240BB60F92BF92CF92DF92EF92FF925F
:10E5F0000F931F932F933F934F935F936F937F934B
:10E600008F939F93AF93BF93EF93FF93CF93DF933A
:10E6100000D01F92CDB7DEB780916E008B7F8093C4
:10E620006E0080916F008D7F80936F007894C09012
:10E630009909D0909A09E0909B09F0909C09C11427
:10E64000D104E104F10409F442C080915203811124
:10E6500004C0809153038823D1F10E94486AF9EBEA
:10E66000CF16FBE0DF06E104F10488F008EBC01AE6
:10E670000BE0D00AE108F108C0929909D0929A09FA
:10E68000E0929B09F0929C0988EB9BE009C0C601CF
:10E690001092990910929A0910929B0910929C0964
:10E6A00090938900809388002091880030918900A0
:10E6B000809184009091850040962817390708F0D2
:10E6C00062C08091840090918500409613C0809133
:10E6D000970990919809009709F488C00197909341
:10E6E000980980939709109294041092930467DF1D
:10E6F00088EC90E0909389008093880044C0C80122
:10E700000E94D53424E630E080915203882309F436
:10E7100083C4C901293BBBE03B0708F0B7C5909310
:10E720008900809388008091890990918A09A0913D
:10E730008B09B0918C09820F931FA11DB11D80938D
:10E74000890990938A09A0938B09B0938C09209131
:10E7500088003091890080918400909185004096D6
:10E760002817390748F480918400909185004096DD
:10E770009093890080938800BB2029F01092940424
:10E78000109293041CDFF89480911204882321F0E6
:10E7900080916E008B7F03C080916E0084608093B7
:10E7A0006E0080916F00826080936F000F900F90D9
:10E7B0000F900F90DF91CF91FF91EF91BF91AF91AB
:10E7C0009F918F917F916F915F914F913F912F9189
:10E7D0001F910F91FF90EF90DF90CF90BF900F901F
:10E7E0000BBE0F900FBE0F901F901895E0919304F1
:10E7F000F0919404309709F089C19091880B809131
:10E80000890B981759F0E091890B1DE4E19FF00105
:10E810001124E755FB4F808188608083F093940436
:10E82000E0939304309709F46EC152A18091920451
:10E83000418158130AC0242F30E080913002082E05
:10E84000000C990B2817390729F050939204409334
:10E85000300254DE10929309109294091092950997
:10E8600010929609E0919304F091940487A990ADD9
:10E8700081342CE9920728F481323EE4930748F072
:10E8800002C080E49CE9969587959695879524E04B
:10E8900007C0813147E2940730F09695879522E0D2
:10E8A0002093920908C021E02093920980329105BB
:10E8B00010F480E290E07C0160E2E61AF108E114D5
:10E8C00088E0F806E0F0EF2DFF27EE0FFF1FEE0FB8
:10E8D000FF1FCF018D5A9A4EFC01329645915491FB
:10E8E000BE2DAA27B59F9001B49F210D3A1F069413
:10E8F0002A1F3A1F1124FC01859194911CC0970195
:10E90000369527952C7F2D5A3E4EF901859194918D
:10E91000F901329665917491A70147705527649F5C
:10E920009001659F300D749F300D112443E03695A2
:10E9300027954A95E1F7821B930B8436910578F46D
:10E9400005E013E0F80181918F01882319F00E94FE
:10E95000D28BF8CFC7010E94D53484E690E0909323
:10E960009109809390098091920980938F09E09199
:10E970009304F091940483AD94AD90938E098093A9
:10E980008D098134FCE99F0728F481320EE4900759
:10E9900048F002C080E49CE9969587959695879506
:10E9A00024E007C0813117E2910730F096958795F2
:10E9B00022E02093920908C021E02093920980323E
:10E9C000910510F480E290E07C0120E2E21AF10867
:10E9D000E11438E0F306E0F0EF2DFF27EE0FFF1F04
:10E9E000EE0FFF1FCF018D5A9A4EFC0132964591D2
:10E9F00054916E2DAA27659F9001649F210D3A1FA7
:10EA000006942A1F3A1F1124FC01859194911CC081
:10EA10009701369527952C7F2D5A3E4EF901859109
:10EA20009491F901329665917491A7014770552729
:10EA3000649F9001659F300D749F300D112463E039
:10EA4000369527956A95E1F7821B930B84369105DD
:10EA500078F405E013E0D8018D918D01882319F039
:10EA60000E94D28BF8CFC7010E94D53484E690E093
:10EA7000AC0160E070E04093890950938A0960938B
:10EA80008B0970938C099093890080938800E091A2
:10EA90009304F091940482899389A489B589B695E9
:10EAA000A79597958795B095A095909581959F4F3F
:10EAB000AF4FBF4F8093850990938609A093870934
:10EAC000B09388098093810990938209A093830968
:10EAD000B093840980937D0990937E09A0937F0968
:10EAE000B09380098093790990937A09A0937B0968
:10EAF000B0937C0910929D0910929E0910929F0973
:10EB00001092A00903C080ED97E0F4CD80915203EC
:10EB10008111B9C3809153038111B5C3209192092A
:10EB2000222309F4A1C1E0919304F091940440914F
:10EB3000790950917A0960917B0970917C098281F1
:10EB40009381A481B581840F951FA61FB71F809361
:10EB5000790990937A09A0937B09B0937C091816E0
:10EB600019061A061B060CF4409AE0919304F091E2
:10EB7000940440917D0950917E0960917F097091C4
:10EB8000800986819781A085B185840F951FA61F76
:10EB9000B71F80937D0990937E09A0937F09B0935E
:10EBA0008009181619061A061B060CF4419AE09102
:10EBB0009304F091940440918109509182096091ED
:10EBC00083097091840982859385A485B585840F16
:10EBD000951FA61FB71F8093810990938209A09368
:10EBE0008309B0938409181619061A061B060CF43B
:10EBF000429AE0919304F0919404409185095091D8
:10EC00008609609187097091880986859785A08912
:10EC1000B189840F951FA61FB71F80938509909314
:10EC20008609A0938709B0938809181619061A0651
:10EC30001B060CF4439A8091790990917A09A0916E
:10EC40007B09B0917C09181619061A061B0684F573
:10EC5000E0919304F0919404428953896489758901
:10EC6000841B950BA60BB70B8093790990937A09B7
:10EC7000A0937B09B0937C0980912C024091050BF5
:10EC80005091060B6091070B7091080B082E000C39
:10EC9000990BAA0BBB0B840F951FA61FB71F809360
:10ECA000050B9093060BA093070BB093080B4098AD
:10ECB00080917D0990917E09A0917F09B091800992
:10ECC000181619061A061B0684F5E0919304F091B4
:10ECD00094044289538964897589841B950BA60B1A
:10ECE000B70B80937D0990937E09A0937F09B09321
:10ECF000800980912D024091090B50910A0B60917F
:10ED00000B0B70910C0B082E000C990BAA0BBB0B74
:10ED1000840F951FA61FB71F8093090B90930A0BB2
:10ED2000A0930B0BB0930C0B4198809181099091AB
:10ED30008209A0918309B0918409181619061A0650
:10ED40001B0684F5E0919304F09194044289538961
:10ED500064897589841B950BA60BB70B8093810979
:10ED600090938209A0938309B093840980912E0225
:10ED700040910D0B50910E0B60910F0B7091100B89
:10ED8000082E000C990BAA0BBB0B840F951FA61F16
:10ED9000B71F80930D0B90930E0BA0930F0BB093A6
:10EDA000100B42988091850990918609A09187095E
:10EDB000B0918809181619061A061B0684F5E09109
:10EDC0009304F09194044289538964897589841B62
:10EDD000950BA60BB70B8093850990938609A0939A
:10EDE0008709B093880980912F024091110B5091AF
:10EDF000120B6091130B7091140B082E000C990BE1
:10EE0000AA0BBB0B840F951FA61FB71F8093110B76
:10EE10009093120BA093130BB093140B4398809113
:10EE20009D0990919E09A0919F09B091A00901961A
:10EE3000A11DB11D80939D0990939E09A0939F09E8
:10EE4000B093A0092150E0919304F0919404428979
:10EE500053896489758984179507A607B70708F44D
:10EE60005FCEBB24B39401C0B12C40919D09509159
:10EE70009E0960919F097091A009E0909304F09021
:10EE80009404F70186899789A08DB18D8417950721
:10EE9000A607B70708F4C6C04091890950918A09AE
:10EEA00060918B0970918C09068D178D20A131A17D
:10EEB000AA27419FB12D529FC001629F900D619F73
:10EEC000800D911D429FB00D811D9A1F519FB00D65
:10EED000811D9A1F609FB00D811D9A1F509FB10D1B
:10EEE0008A1F9A1FB6958A1F9A1F349F800D911D05
:10EEF000359F900D112423AD34AD820F931F909355
:10EF00008E0980938D0947A950AD61AD72ADA0E027
:10EF1000B0E0481759076A077B0720F450938E0921
:10EF200040938D0980918D0990918E098134BCE9BF
:10EF30009B0728F48132EEE49E0748F002C080E48B
:10EF40009CE9969587959695879524E007C0813131
:10EF5000F7E29F0730F09695879522E0209392097B
:10EF600008C021E0209392098032910510F480E2DC
:10EF700090E08C0100521109011528E01207E8F019
:10EF8000E12FFF27EE0FFF1FEE0FFF1FCF018D5A5E
:10EF90009A4EFC01329625913491AA27039FA00135
:10EFA000029F410D5A1F06944A1F5A1F1124FC014B
:10EFB00025913491241B350B1EC0A8015695479509
:10EFC0004C7F4D5A5E4EFA0125913491FA013296EA
:10EFD00065917491A80147705527649FC001659F92
:10EFE000900D749F900D1124B3E096958795BA9576
:10EFF000E1F7281B390B2436310508F085CBF5E005
:10F00000EF2EF3E0FF2ED7018D917D01882309F4C7
:10F0100076CB0E94D28BF7CF80915303811179CBAD
:10F02000C9017DCB40919D0950919E0960919F0936
:10F030007091A009F701828D938DA48DB58D8417F1
:10F040009507A607B70708F0EBC000919309109148
:10F050009409209195093091960909831A832B838D
:10F060003C83468D578D60A171A1AA27059FB12DC4
:10F07000169F6001269FD00C259FC00CD11C069FB7
:10F08000B00DC11CDA1E159FB00DC11CDA1E249FE5
:10F09000B00DC11CDA1E149FB10DCA1EDA1EB69542
:10F0A000CA1EDA1E709FC00CD11C719FD00C112497
:10F0B00080918D0990918E09FF96C816D90680F42B
:10F0C0008C199D0940815181628173816C01E12C11
:10F0D000F12CC416D506E606F70620F4CA0102C0D4
:10F0E0008081918181341CE9910728F481322EE4DA
:10F0F000920748F002C080E49CE996958795969522
:10F10000879524E007C0813137E2930730F0969568
:10F11000879522E02093920908C021E0209392096C
:10F120008032910510F480E290E08C0100521109C8
:10F13000011548E01407E8F0E12FFF27EE0FFF1F4D
:10F14000EE0FFF1FCF018D5A9A4EFC01329625918A
:10F150003491AA27039FA001029F410D5A1F0694D4
:10F160004A1F5A1F1124FC0125913491241B350B91
:10F170001EC0C801969587958C7F8D5A9E4EFC01C6
:10F1800025913491FC01329665917491A8014770E4
:10F190005527649FC001659F900D749F900D1124A9
:10F1A00043E0969587954A95E1F7281B390B24365D
:10F1B000310588F485E0E82E83E0F82ED7018D91A3
:10F1C0007D01882319F00E94D28BF8CFC8010E94DC
:10F1D000D53424E630E080915203811104C080913F
:10F1E0005303882339F0C901293BBBE03B0708F0F2
:10F1F00068C001C0C901909389008093880089810B
:10F200009A81AB81BC81820F931FA11DB11D809398
:10F21000930990939409A0939509B093960997CA7E
:10F22000209190093091910980915203811104C07D
:10F23000809153038823F1F0293BEBE03E07D0F0A7
:10F24000C90168EB7BE00E943BA0883E43E0940745
:10F2500008F052C08854944FA901481B590B60E034
:10F2600070E04093990950939A0960939B097093B9
:10F270009C099C01309389002093880080918F091C
:10F280008093920964CA0E94486A48CC68EB7BE08C
:10F290000E943BA0883E03E0900780F48854944F7E
:10F2A000A901481B590B60E070E040939909509305
:10F2B0009A0960939B0970939C0931CA88EB9BE083
:10F2C000EFCF68EB7BE00E943BA0883E13E0910704
:10F2D00080F48854944FA901481B590B60E070E0FA
:10F2E0004093990950939A0960939B0970939C09E4
:10F2F00082CF88EB9BE0EFCF88EB9BE0ADCF8F9286
:10F300009F92AF92BF92CF92DF92EF92FF920F93B4
:10F310001F93CF93DF9300D01F92CDB7DEB784E663
:10F32000882E84E0982E95E2A92E9BE0B92E09E95B
:10F3300014E0C12CD12C7601C394F4016191719138
:10F34000819191914F01F50121913191419151911B
:10F350005F0129833A834B835C830E94449929810E
:10F360003A814B815C810E94A5990E94BC9EF80164
:10F3700061937193819391938F01C616D706E80626
:10F38000F90610F46B017C01F4E78F16F4E09F0698
:10F39000A1F66FEF7FEFCB01A70196010E941B9DA5
:10F3A00020939504309396044093970450939804C7
:10F3B0000F900F900F900F90DF91CF911F910F91B1
:10F3C000FF90EF90DF90CF90BF90AF909F908F9085
:10F3D0000895EF92FF920F931F93CF93DF93CDB7D2
:10F3E000DEB72C970FB6F894DEBF0FBECDBF05E297
:10F3F0001BE084E6E82E83E0F82EF801219131919C
:10F40000419151918F0160E070E080E89FE30E949C
:10F410004F9EF70161937193819391937F01FBE07C
:10F4200005331F0751F78091150B9091160BA09192
:10F43000170BB091180B89839A83AB83BC8380919F
:10F44000190B90911A0BA0911B0BB0911C0B8D8383
:10F450009E83AF83B88780911D0B90911E0BA09166
:10F460001F0BB091200B89879A87AB87BC87AE01B1
:10F47000475F5F4FBE016B5F7F4FCE0101960E94D9
:10F48000E64921E23BE0AE01475F5F4FBE016B5FA3
:10F490007F4FCE0101960E941B3B31DF2C960FB6A9
:10F4A000F894DEBF0FBECDBFDF91CF911F910F91BA
:10F4B000FF90EF900895CF92DF92EF92FF920F931B
:10F4C0001F93CF93DF93CDB7DEB72C970FB6F89489
:10F4D000DEBF0FBECDBF45E25BE024E734E0A4E62B
:10F4E000B4E080E090E0FC01E65BF54EC590D5907D
:10F4F000E590F490FA01C192D192E192F192AF01BC
:10F50000FC01E65CF54EC590D590E590F490F901CC
:10F51000C192D192E192F1929F01FC01E65DF54E1C
:10F52000C590D590E590F490CD92DD92ED92FD924C
:10F53000049680319105B9F680E090E0AAEFB4E43A
:10F540008093600490936104A0936204B093630479
:10F5500040E050E86BE375E440935C0450935D0435
:10F5600060935E0470935F048093580490935904F1
:10F57000A0935A04B0935B04109254041092550463
:10F58000109256041092570480E29EE4A0E0B0E08E
:10F5900080934C0490934D04A0934E04B0934F0479
:10F5A000109250041092510410925204109253047D
:10F5B00080E090E0A0E4B1E480933C0490933D04AB
:10F5C000A0933E04B0933F04809340049093410481
:10F5D000A0934204B09343048DEC9CECACECBEE3EE
:10F5E0008093440490934504A0934604B093470449
:10F5F00080E090E0A0E2B1E4809348049093490455
:10F60000A0934A04B0934B041CE0E4E5F3E0DF016F
:10F61000812F1D928A95E9F70E94F94C89E891E4BF
:10F62000A0EBBFEB8093010B9093020BA093030B15
:10F63000B093040B8CEE91E5A6EEB1E48093380410
:10F6400090933904A0933A04B0933B0480EF98E37D
:10F65000A0EABEE38093340490933504A09336046B
:10F66000B093370488EB92E9A5E2B4E480933004C8
:10F6700090933104A0933204B093330480E090E07F
:10F68000A3E9B3E480932C0490932D04A0932E045B
:10F69000B0932F0483EC94E6AAE2B1E480932804AB
:10F6A00090932904A0932A04B0932B0480EB98EB49
:10F6B000A1E1B5E48093240490932504A09326044B
:10F6C000B09327041092880480E090E0A0E4B0E4B6
:10F6D0008093840490938504A0938604B093870458
:10F6E00081E08093520380935103E4E5F2E0DE0170
:10F6F000119601900D921A95E1F713E01150C8F0A0
:10F70000A4E01A9F90011124E1E0F0E0EC0FFD1F4E
:10F71000E20FF31F6081718182819381F901E85EBC
:10F72000FB4F6083718382839383812F0E94E371F7
:10F73000E5CF0E941361E5ECFCE184918F010F5F3E
:10F740001F4F882321F00E94D28BF801F6CFE7E00B
:10F75000FAE184918F010F5F1F4F882321F00E94EF
:10F76000D28BF801F6CF2C960FB6F894DEBF0FBE01
:10F77000CDBFDF91CF911F910F91FF90EF90DF9060
:10F78000CF9008952F923F924F925F926F927F9207
:10F790008F929F92AF92BF92CF92DF92EF92FF92A1
:10F7A0000F931F93CF93DF93CDB7DEB7CC55D1091D
:10F7B0000FB6F894DEBF0FBECDBF2DB73EB76B9628
:10F7C0003FAF2EAF6B9761961FAE1EAE619784E67A
:10F7D00090E02F969FAF8EAF2F979E01215B3F4FFA
:10F7E00044E050E0BE016F5B7F4FCE01835B9F4FD3
:10F7F0000E946C609E01215B3F4F42E050E0BE01E1
:10F80000655B7F4FCE01835B9F4F0E946C6043E03E
:10F8100050E0BE016F5B7F4F89E193E00E9482A0C0
:10F82000892B09F439C022968FAD2297863539F09D
:10F830008FE322968FAF229723961FAE2397E5EC96
:10F84000FCE184918F010F5F1F4F882321F00E94FC
:10F85000D28BF801F6CFEEEEF9E184918F010F5FC4
:10F860001F4F882321F00E94D28BF801F6CFBE01F2
:10F870006F5B7F4F85EE99E10E947F67E7EDF9E1CD
:10F8800084918F010F5F1F4F882321F00E94D28B3C
:10F89000F801F6CF10DE4CC46DB67EB621961CAED4
:10F8A0001DAE1EAE1FAE219761961FAE1EAE6197B4
:10F8B0009E01215B3F4F41E050E0BE01695A7F4FFE
:10F8C000CE01835B9F4F0E946C6080E1E0E6F2E036
:10F8D000DE01919601900D928A95E1F780E1E0E7D3
:10F8E000F2E0DE01519601900D928A95E1F780E1F8
:10F8F000E0E8F2E08E010F5F1F4FD80101900D92FA
:10F900008A95E1F76896CFAC6897D12C33E0C30EA7
:10F91000D11CCC0CDD1CCC0CDD1C8DB79EB78C191A
:10F920009D090FB6F8949EBF0FBE8DBFEDB7FEB711
:10F9300031964F012DB73EB72C193D090FB6F894FB
:10F940003EBF0FBE2DBF8DB79EB701965C01EDB7D0
:10F95000FEB7EC19FD090FB6F894FEBF0FBEEDBF60
:10F960002DB73EB72F5F3F4F79019E01215B3F4F7F
:10F97000A601B401CE01835B9F4F0E946C609E0183
:10F98000215B3F4FA601B501CE01835B9F4F0E94D3
:10F990006C609E01215B3F4FA601B701CE01835BE6
:10F9A0009F4F0E946C6068962FAD689730E02E5F85
:10F9B0003F4F84E694E06D969FAF8EAF6D97A4E7BE
:10F9C000B4E065E27BE080E090E040E050E02417A6
:10F9D000350714F0640105C0F1E2CF2ED12CCC0E16
:10F9E000DD1EC80ED91EF601208031804280538072
:10F9F000FB012192319241925192BF0124173507A8
:10FA000014F0650105C0E1E1CE2ED12CCC0EDD1E37
:10FA1000C80ED91EF60120803180428053802D927D
:10FA20003D924D925D922417350714F0670101C095
:10FA30006801C80ED91EF6012080318042805380B3
:10FA40006D96EEADFFAD6D9721923192419251923C
:10FA50006D96FFAFEEAF6D974F5F5F4F04964430EA
:10FA6000510509F0B4CF9E01215B3F4F44E050E0C7
:10FA700060E674E0CE01835B9F4F0E946C609E0144
:10FA8000215B3F4F44E050E06CE574E0CE01835BC6
:10FA90009F4F0E946C609E01215B3F4F44E050E00D
:10FAA00068E574E0CE01835B9F4F0E946C609E010D
:10FAB000215B3F4F44E050E064E574E0CE01835B9E
:10FAC0009F4F0E946C609E01215B3F4F44E050E0DD
:10FAD00060E574E0CE01835B9F4F0E946C609E01E5
:10FAE000215B3F4F44E050E06CE474E0CE01835B67
:10FAF0009F4F0E946C609E01215B3F4F40E150E0B0
:10FB00006CE374E0CE01835B9F4F0E946C609E01AA
:10FB1000215B3F4F4CE050E064E573E0CE01835B36
:10FB20009F4F0E946C609E01215B3F4F44E050E07C
:10FB3000BE01635C7F4FCE01835B9F4F0E946C6070
:10FB40009E01215B3F4F41E050E0BE016A5A7F4F6A
:10FB5000CE01835B9F4F0E946C609E01215B3F4FF3
:10FB600044E050E0BE01635C7F4FCE01835B9F4F5A
:10FB70000E946C609E01215B3F4F41E050E0BE015E
:10FB80006B5A7F4FCE01835B9F4F0E946C609E013A
:10FB9000215B3F4F41E050E0BE016C5A7F4FCE01E8
:10FBA000835B9F4F0E946C6066968FAD66976596EB
:10FBB0000FAD6597809F80011124E12CF12CE01698
:10FBC000F10689F09E01215B3F4F44E050E0BE0109
:10FBD000635C7F4FCE01835B9F4F0E946C60FFEFA1
:10FBE000EF1AFF0AECCF61960EAD1FAD61972F960D
:10FBF0008EAD9FAD2F9790933202809331029E017C
:10FC0000215B3F4F44E050E061E07BE0CE01835B4D
:10FC10009F4F0E946C6061961FAF0EAF61979E016F
:10FC2000215B3F4F44E250E060E47BE0CE01835B28
:10FC30009F4F0E946C609E01215B3F4F41E050E06E
:10FC4000BE016D5A7F4FCE01835B9F4F0E946C6057
:10FC50009E01215B3F4F41E050E0BE016E5A7F4F55
:10FC6000CE01835B9F4F0E946C609E01215B3F4FE2
:10FC700044E050E0BE016B5C7F4FCE01835B9F4F41
:10FC80000E946C609E01215B3F4F44E050E0BE014A
:10FC90006F5C7F4FCE01835B9F4F0E946C606496C8
:10FCA0008FAD649763960FAD6397809F8001112499
:10FCB000E12CF12C9E01215B3F4FE016F10671F023
:10FCC00044E050E0BE01635C7F4FCE01835B9F4FF9
:10FCD0000E946C602FEFE21AF20AECCF41E050E094
:10FCE000BE01685A7F4FCE01835B9F4F0E946C60BC
:10FCF0009E01215B3F4F44E050E0BE01635C7F4FBB
:10FD0000CE01835B9F4F0E946C609E01215B3F4F41
:10FD100041E050E0BE016F5A7F4FCE01835B9F4FA1
:10FD20000E946C6021961CAE1DAE1EAE1FAE2197C8
:10FD30001DE011509E01215B3F4F44E050E0BE01A9
:10FD4000112341F0635C7F4FCE01835B9F4F0E9484
:10FD50006C60EFCF675C7F4FCE01835B9F4F0E944B
:10FD60006C609E01215B3F4F44E050E0BE016B5C44
:10FD70007F4FCE01835B9F4F0E946C609E01215B91
:10FD80003F4F44E050E0BE016F5C7F4FCE01835B8C
:10FD90009F4F0E946C609E01215B3F4F44E050E00A
:10FDA000BE01635C7F4FCE01835B9F4F0E946C60FE
:10FDB00011113EC02196CCACDDACEEACFFAC21976E
:10FDC00020E030E84BE355E4C701B6010E944099BA
:10FDD000882371F1C0923804D0923904E0923A0439
:10FDE000F0923B049E01215B3F4F44E050E064E30E
:10FDF00074E0CE01835B9F4F0E946C609E01215B8B
:10FE00003F4F44E050E060E374E0CE01835B9F4FDE
:10FE10000E946C609E01215B3F4F44E050E0BE01B8
:10FE2000635C7F4FCE01835B9F4F0E946C6011C06B
:10FE300004E0015071F09E01215B3F4F44E050E02F
:10FE4000BE01635C7F4FCE01835B9F4F0E946C605D
:10FE5000F0CF1F5F153009F09ECF9E01215B3F4F11
:10FE600042E050E0BE01675B7F4FCE01835B9F4F56
:10FE70000E946C609E01215B3F4F44E050E0BE0158
:10FE8000635C7F4FCE01835B9F4F0E946C60219625
:10FE9000CCACDDACEEACFFAC219720E030E84BE31E
:10FEA00055E4C701B6010E944099882301F1C09230
:10FEB0002C04D0922D04E0922E04F0922F049E0187
:10FEC000215B3F4F44E050E068E274E0CE01835B89
:10FED0009F4F0E946C609E01215B3F4F44E050E0C9
:10FEE00064E274E0CE01835B9F4F0E946C609E01D0
:10FEF000215B3F4F42E050E0BE01695B7F4FCE0186
:10FF0000835B9F4F0E946C609E01215B3F4F41E0ED
:10FF100050E0BE01685A7F4FCE01835B9F4F0E9425
:10FF20006C6019E011509E01215B3F4F112359F085
:10FF300044E050E0BE01635C7F4FCE01835B9F4F86
:10FF40000E946C60EFCF41E050E068E874E0CE01C1
:10FF5000835B9F4F0E946C609E01215B3F4F44E09A
:10FF600050E0BE01635C7F4FCE01835B9F4F0E94D8
:10FF70006C6011110EC021968CAD9DADAEADBFADC4
:10FF800021978093840490938504A0938604B09372
:10FF900087041F5F153001F71BE09E01215B3F4F77
:10FFA00042E050E0BE016B5B7F4FCE01835B9F4F11
:10FFB0000E946C60115089F79E01215B3F4F44E025
:10FFC00050E0BE01635C7F4FCE01835B9F4F0E9478
:10FFD0006C609E01215B3F4F44E050E0BE01635CDA
:10FFE0007F4FCE01835B9F4F0E946C6013E01150E6
:10FFF00088F034E0139FB0011124685E7B4F9E01AE
:020000021000EC
:10000000215B3F4F44E050E0CE01835B9F4F0E9455
:100010006C60EDCF61962EAD3FAD61972D968EADA4
:100020009FAD2D972817390709F03AC00E94136138
:10003000E5ECFCE184918F010F5F1F4F811103C03C
:1000400009E113E004C00E94D28BF801F3CFF8015C
:1000500081918F01882319F00E94D28BF8CF2F96BF
:100060006EAD7FAD2F97645671098AEB99E10E94BE
:10007000666761964EAD5FAD619760E070E08DEAB6
:1000800099E10E949738EAEAF9E184918F010F5FC4
:100090001F4F882309F447C00E94D28BF801F5CF87
:1000A000EBECF9E084918F010F5F1F4F882321F063
:1000B0000E94D28BF801F6CFEAE8F9E184918F0132
:1000C0000F5F1F4F882321F00E94D28BF801F6CFDB
:1000D0002D966EAD7FAD2D9780E090E04AE00E94B6
:1000E0002B8CE5E8F9E184918F010F5F1F4F882386
:1000F00021F00E94D28BF801F6CF61966EAD7FADF4
:10010000619780E090E04AE00E942B8CE5E7F9E1FE
:1001100084918F010F5F1F4F882321F00E94D28BA3
:10012000F801F6CFC8D90FB6F8947EBE0FBE6DBEEB
:1001300080E00E946A6D9091A10981E089276B9609
:100140002EAD3FAD6B970FB6F8943EBF0FBE2DBFDF
:10015000C45ADF4F0FB6F894DEBF0FBECDBFDF919C
:10016000CF911F910F91FF90EF90DF90CF90BF90B4
:10017000AF909F908F907F906F905F904F903F9047
:100180002F9008958F929F92AF92BF92CF92DF925D
:10019000EF92FF920F931F93CF93DF93CDB7DEB70C
:1001A000C555D1090FB6F894DEBF0FBECDBF21965D
:1001B0001CAE1DAE1EAE1FAE219780E390E3A0E300
:1001C000B0E089AF9AAFABAFBCAF2D961FAE1EAEFD
:1001D0002D9784E690E02B969FAF8EAF2B971092D1
:1001E000A1099E01255B3F4F44E050E0BE01675CE2
:1001F0007F4FCE01875B9F4F0E94A6602B968EADEE
:100200009FAD2B9702962B969FAF8EAF2B972D9677
:100210001FAE1EAE2D9781E066968FAF66979E014A
:10022000255B3F4F41E050E0BE016B5A7F4FCE014E
:10023000875B9F4F0E94A6609E01255B3F4F40E178
:1002400050E065E27BE0CE01875B9F4F0E94A66095
:100250009E01255B3F4F40E150E064E774E0CE0132
:10026000875B9F4F0E94A6609E01255B3F4F40E148
:1002700050E064E674E0CE01875B9F4F0E94A66069
:100280009E01255B3F4F44E050E060E674E0CE0104
:10029000875B9F4F0E94A6609E01255B3F4F44E015
:1002A00050E06CE574E0CE01875B9F4F0E94A66032
:1002B0009E01255B3F4F44E050E068E574E0CE01CD
:1002C000875B9F4F0E94A6609E01255B3F4F44E0E5
:1002D00050E064E574E0CE01875B9F4F0E94A6600A
:1002E0009E01255B3F4F44E050E060E574E0CE01A5
:1002F000875B9F4F0E94A6609E01255B3F4F44E0B5
:1003000050E06CE474E0CE01875B9F4F0E94A660D2
:100310009E01255B3F4F40E150E06CE374E0CE016D
:10032000875B9F4F0E94A6609E01255B3F4F4CE07C
:1003300050E064E573E0CE01875B9F4F0E94A660AA
:1003400080E090E0A0E2B1E48DAB9EABAFABB8AF84
:100350009E01255B3F4F44E050E0BE016B5C7F4F48
:10036000CE01875B9F4F0E94A66065961FAE659782
:1003700021961CAE1DAE1EAE1FAE219783E0649683
:100380008FAF649763968FAF63979E01255B3F4F56
:1003900041E050E0BE016C5A7F4FCE01875B9F4F1A
:1003A0000E94A6609E01255B3F4F44E050E0BE01E5
:1003B000635C7F4FCE01875B9F4F0E94A6609E01CA
:1003C000255B3F4F41E050E0BE016D5A7F4FCE01AB
:1003D000875B9F4F0E94A6609E01255B3F4F41E0D7
:1003E00050E0BE016E5A7F4FCE01875B9F4F0E9447
:1003F000A6601AE0115071F09E01255B3F4F44E06A
:1004000050E0BE01635C7F4FCE01875B9F4F0E942F
:10041000A660F0CF2D960EAD1FAD2D972B968EAD0D
:100420009FAD2B9790933202809331029E01255B02
:100430003F4F44E050E061E07BE0CE01875B9F4F9F
:100440000E94A6602D961FAF0EAF2D979E01255BD3
:100450003F4F44E250E060E47BE0CE01875B9F4F7A
:100460000E94A66083E062968FAF629761968FAF1D
:10047000619719AA1AAA1BAA1CAA1DA61EA61FA626
:1004800018AA21961CAE1DAE1EAE1FAE21979E016E
:10049000255B3F4F41E050E0BE016F5A7F4FCE01D8
:1004A000875B9F4F0E94A6609E01255B3F4F41E006
:1004B00050E0BE01605B7F4FCE01875B9F4F0E9483
:1004C000A6609E01255B3F4F44E050E0BE01635DA6
:1004D0007F4FCE01875B9F4F0E94A6609E01255BE8
:1004E0003F4F44E050E0BE016F5C7F4FCE01875B21
:1004F0009F4F0E94A6600AE010E00150110971F0C0
:100500009E01255B3F4F44E050E0BE01635C7F4F9E
:10051000CE01875B9F4F0E94A660EFCF60961FAE13
:10052000609721961CAE1DAE1EAE1FAE21978FEFB9
:100530002F968FAF2F979E01255B3F4F41E050E0F4
:10054000BE01615B7F4FCE01875B9F4F0E94A6601B
:100550009E01255B3F4F44E050E0BE01635C7F4F4E
:10056000CE01875B9F4F0E94A6609E01255B3F4F97
:1005700041E050E0BE01625B7F4FCE01875B9F4F41
:100580000E94A66021961CAE1DAE1EAE1FAE219726
:100590001DE0115071F09E01255B3F4F44E050E09B
:1005A000BE01635C7F4FCE01875B9F4F0E94A660B8
:1005B000F0CF84EB90E09AA789A780EF90E09CA70A
:1005C0008BA786E490E09EA38DA38EE690E098A78B
:1005D0008FA31AA219A21CA21BA29E01255B3F4F4A
:1005E00044E050E0BE01675D7F4FCE01875B9F4FC7
:1005F0000E94A6609E01255B3F4F44E050E0BE0193
:100600006B5D7F4FCE01875B9F4F0E94A6609E016E
:10061000255B3F4F44E050E0BE016F5D7F4FCE0150
:10062000875B9F4F0E94A660C12C80E8D82E8BE389
:10063000E82E85E4F82E812C912C90E8A92E9FE3DA
:10064000B92E111138C09E01255B3F4F44E050E0A8
:1006500068E374E0CE01875B9F4F0E94A6609E0115
:10066000255B3F4F44E050E064E374E0CE01875BDC
:100670009F4F0E94A6609E01255B3F4F44E050E0E3
:1006800060E374E0CE01875B9F4F0E94A6602196D5
:100690008CAE9DAEAEAEBFAE21979E01255B3F4FA7
:1006A00044E050E0BE01635C7F4FCE01875B9F4F0B
:1006B0000E94A6602AC02196CCAEDDAEEEAEFFAEA3
:1006C00021979E01255B3F4F44E050E0BE01635CF3
:1006D0007F4FCE01875B9F4F0E94A66021961CAE84
:1006E0001DAE1EAE1FAE219704E0015071F09E01B9
:1006F000255B3F4F44E050E0BE01635C7F4FCE017D
:10070000875B9F4F0E94A660F0CF1F5F153009F0F6
:1007100098CF84E190E029969FAF8EAF29979E01F4
:10072000255B3F4F42E050E0BE01695B7F4FCE0149
:10073000875B9F4F0E94A6609E01255B3F4F44E070
:1007400050E06CE274E0CE01875B9F4F0E94A66090
:100750009E01255B3F4F44E050E068E274E0CE012B
:10076000875B9F4F0E94A6609E01255B3F4F44E040
:1007700050E064E274E0CE01875B9F4F0E94A66068
:1007800080E290E027969FAF8EAF27979E01255B72
:100790003F4F42E050E0BE016B5B7F4FCE01875B75
:1007A0009F4F0E94A6602E961FAE2E9780E090E08D
:1007B000A0E4B0E48D8F9E8FAF8FB8A380E090E06F
:1007C000A4E3B2E4898F9A8FAB8FBC8F1D8A1E8AF7
:1007D0001F8A188E198A1A8A1B8A1C8A1D861E86F1
:1007E0001F86188A80E090E0A0E5B1E489879A87A7
:1007F000AB87BC871D821E821F82188680E090E036
:10080000A0E0B1E489839A83AB83BC839E01255B1E
:100810003F4F41E050E0BE01635B7F4FCE01875BFD
:100820009F4F0E94A6609E01255B3F4F44E050E031
:10083000BE01635E7F4FCE01875B9F4F0E94A66023
:100840009E01255B3F4F44E050E0BE01675E7F4F55
:10085000CE01875B9F4F0E94A6609E01255B3F4FA4
:1008600044E050E0BE016B5E7F4FCE01875B9F4F3F
:100870000E94A6609E01255B3F4F44E050E0BE0110
:100880006F5E7F4FCE01875B9F4F0E94A6609E01E7
:10089000255B3F4F44E050E0BE01635F7F4FCE01D8
:1008A000875B9F4F0E94A6609E01255B3F4F44E0FF
:1008B00050E0BE01675F7F4FCE01875B9F4F0E9474
:1008C000A6609E01255B3F4F44E050E0BE016B5F98
:1008D0007F4FCE01875B9F4F0E94A6609E01255BE4
:1008E0003F4F44E050E0BE016F5F7F4FCE01875B1A
:1008F0009F4F0E94A6609E01255B3F4F41E050E064
:1009000068E874E0CE01875B9F4F0E94A66010E00C
:1009100011110EC08091840490918504A0918604E9
:10092000B091870421968CAF9DAFAEAFBFAF21973A
:100930009E01255B3F4F44E050E0BE01635C7F4F6A
:10094000CE01875B9F4F0E94A6601F5F153001F7A5
:1009500025961FAE1EAE25971CE0115071F09E012A
:10096000255B3F4F42E050E0BE016D5B7F4FCE0103
:10097000875B9F4F0E94A660F0CF21961CAE1DAEF4
:100980001EAE1FAE21979E01255B3F4F44E050E015
:10099000BE01635C7F4FCE01875B9F4F0E94A660C4
:1009A0009E01255B3F4F44E050E0BE01635C7F4FFA
:1009B000CE01875B9F4F0E94A66013E0115088F024
:1009C00084E0189FB0011124685E7B4F9E01255B77
:1009D0003F4F44E050E0CE01875B9F4F0E94A660EE
:1009E000EDCF8091A109811152C02B96EEACFFACE6
:1009F0002B972D968EAD9FAD2D9723969FAF8EAFE3
:100A0000239784E690E02B969FAF8EAF2B979E01A5
:100A1000255B3F4F44E050E069E173E0CE01875B26
:100A20009F4F0E94A6609E01255B3F4F42E050E031
:100A3000BE016F5B7F4FCE01875B9F4F0E94A66018
:100A4000E5ECFCE184918F010F5F1F4F882319F0C3
:100A5000A9D6F801F7CFB7016456710983E699E189
:100A60000E94666723964EAD5FAD239760E070E00D
:100A700086E599E10E949738E3E5F9E184918F01D9
:100A80000F5F1F4F882319F08DD6F801F7CF909193
:100A9000A10981E08927CB5ADF4F0FB6F894DEBF5A
:100AA0000FBECDBFDF91CF911F910F91FF90EF90BF
:100AB000DF90CF90BF90AF909F908F900895089552
:100AC00090E0FC013197E231F10508F04EC0882733
:100AD000EE58FF4F8F4F0C9462A0809180008F776B
:100AE00003C0809180008F7D809380000895809165
:100AF0008000877FF9CF84B58F7702C084B58F7D62
:100B000084BD08958091B0008F7703C08091B000BC
:100B10008F7D8093B0000895809190008F7707C0FB
:100B2000809190008F7D03C080919000877F80939B
:100B3000900008958091A0008F7707C08091A00059
:100B40008F7D03C08091A000877F8093A0000895CF
:100B5000809120018F7707C0809120018F7D03C095
:100B600080912001877F8093200108953FB7F894FA
:100B70008091A7099091A809A091A909B091AA090B
:100B800026B5A89B05C02F3F19F00196A11DB11DE8
:100B90003FBFBA2FA92F982F8827820F911DA11D23
:100BA000B11DBC01CD0142E0660F771F881F991F60
:100BB0004A95D1F70895EF92FF920F931F93CF9329
:100BC000DF931F92CDB7DEB7082F162FEBECF9E0BD
:100BD00084917F012FEFE21AF20A882329F099838A
:100BE000E1D5F7019981F4CFE02FF92F84917F01AE
:100BF0009FEFE91AF90A882319F0D4D5F701F6CF47
:100C00006091970B7091980B8091990B90919A0B32
:100C10000E94BA4A8AE0C6D511110E94DC94109253
:100C2000150A1092140A0F90DF91CF911F910F9126
:100C3000FF90EF900895FF920F931F93CF93DF9350
:100C4000FC0120812B3319F1D0918103D430F8F4C9
:100C5000F62EBC01C091AD090C2F10E0F0E6CF9F3D
:100C6000C00111248556944F0E947BA0F801E05AE0
:100C7000FC4FF082CF5FC43018F4C093AD0902C0BE
:100C80001092AD09DF5FD093810381E001C080E065
:100C9000DF91CF911F910F91FF900895BF92CF9256
:100CA000DF92EF92FF920F931F93CF93DF93CDB715
:100CB000DEB76E970FB6F894DEBF0FBECDBF609162
:100CC000AE097091AF096115710559F14DE150E020
:100CD000CE0101967C010E94E8981E8EF7018F01DB
:100CE0000E191F09B190BB2099F19AE0B912F7CF04
:100CF0002FC0B70184E79AE10E947F6782E252D554
:100D00008AE050D5BB2009F439C00F5F1F4F809196
:100D1000AE099091AF09080F191F1093AF09009306
:100D2000AE098091AE099091AF09892B09F028C1D5
:100D300080918103843008F023C12FB7F89480910B
:100D4000D00A9091D10A2FBF891B8F77D1F418C197
:100D5000F701E00FF11F108260E0C7016CDF88230C
:100D600001F3E5ECFCE184916F019FEFC91AD90A08
:100D7000882309F4BECF16D5F601F5CF00E010E0C8
:100D8000CCCFCFD52091140A3091150A8A3019F0B2
:100D90008D3009F0C5C01092160A2115310509F4ED
:100DA000C7CFF901EC54F64F10821092150A109239
:100DB000140A24EB39E08901F90180812F5F3F4F4C
:100DC0008032C9F378018E3411F000E010E06AE25D
:100DD00070E0C7010E9470A06C010115110509F4B3
:100DE00073C06EE97BE1C7010E94F798BB24B394FE
:100DF000892B11F4B12C09C06EE470E0C701049690
:100E00000E9470A0009709F08C014AE050E060E079
:100E100070E0C80101960E946C966093B0097093CF
:100E2000B1098093B2099093B3090091970B109187
:100E3000980B2091990B30919A0B0F5F1F4F2F4FFA
:100E40003F4F601771078207930731F0B11004C05C
:100E500061E08BE69BE13DC0C114D10401F180E06B
:100E600010E0F701E80FF11D90819A3219F08F5FC1
:100E70001927F7CF4AE050E060E070E0C601019624
:100E80000E946C96012F10E020E030E0601771079F
:100E90008207930741F061E08CE49BE11AC061E0B6
:100EA00082E29BE116C08091B0099091B109A091B6
:100EB000B209B091B3098093970B9093980BA093CC
:100EC000990BB0939A0B07C0892B29F060E081E859
:100ED0009AE171DE55C08091210281111CC067E446
:100EE00070E0C7010E9470A00097A9F04AE050E0AE
:100EF00060E070E001960E946C966430710558F4D1
:100F0000EBEAFAE184918F010F5F1F4F882319F0FC
:100F100049D4F801F7CF61E084EB99E08CDE08CF8B
:100F20002F3531050CF004CF8C35A9F42FB7F89488
:100F30008091D00A9091D10A2FBF891B8F7709F435
:100F4000F7CEEFD49091160A9111F2CE2091140AA7
:100F50003091150A09C08B3319F491E09093160A69
:100F60009091160A9111E4CEA9014F5F5F4F509303
:100F7000150A4093140AF901EC54F64F8083D8CE39
:100F80006E960FB6F894DEBF0FBECDBFDF91CF9146
:100F90001F910F91FF90EF90DF90CF90BF90089539
:100FA0000F931F93CF93DF93CDB7DEB72C970FB678
:100FB000F894DEBF0FBECDBFE5E1FBE080859185F3
:100FC000A285B38544815581668177810081118135
:100FD0002281338109831A832B833C834D835E8373
:100FE0006F83788789879A87AB87BC87AE01475F15
:100FF0005F4FBE016B5F7F4FCE0101960E94E649B5
:1010000021E23BE0AE01475F5F4FBE016B5F7F4F68
:10101000CE0101960E941B3B2C960FB6F894DEBFC2
:101020000FBECDBFDF91CF911F910F910895809199
:10103000AB099091AC09009731F04AE050E060E0D4
:1010400070E00C94949760E070E0CB01089580917B
:10105000AB099091AC09009731F04AE050E060E0B4
:1010600070E00C946C9660E070E0CB010895EFDFC7
:1010700097FD0AC0ECDF6F3F71058105910509F00E
:101080002CF4E5DF862F089580E008958FEF089512
:101090008091AB099091AC09892B31F0E8DF91E0A8
:1010A000811103C090E001C091E0892F08950F9352
:1010B0001F93CF938091AB099091AC090097F1F009
:1010C000FC018F01C1912C2F2F7D89F0C53411F0C7
:1010D000C536B9F7F801108260E070E00E9406950D
:1010E000F801C083562F472F382F292F0BC060E0FF
:1010F00070E0CF911F910F910C94069550E040E065
:1011000030E020E0652F742F832F922FCF911F9115
:101110000F91089581548A3150F5482F50E0FA011B
:1011200093E0F595E7959A95E1F7E85CFC4F20810F
:1011300030E08770B90102C0759567958A95E2F72E
:1011400060FF15C0FA01E25EFC4F2081222339F0D6
:101150008091280A9091290A820F911D02C080E097
:1011600090E09093AC098093AB0981E0089580E012
:101170000895D0DF882341F081E02091AB093091C0
:10118000AC09232B09F480E008951F920F920FB64B
:101190000F9211240BB60F922F933F934F935F93AF
:1011A0006F937F938F939F93AF93BF93EF93FF932F
:1011B000E0914102F09142021995FF91EF91BF91A8
:1011C000AF919F918F917F916F915F914F913F91DF
:1011D0002F910F900BBE0F900FBE0F901F90189580
:1011E0001F920F920FB60F9211240BB60F922F93EE
:1011F0003F934F935F936F937F938F939F93AF939F
:10120000BF93EF93FF93E0913F02F0914002199555
:10121000FF91EF91BF91AF919F918F917F916F91CE
:101220005F914F913F912F910F900BBE0F900FBE8A
:101230000F901F9018951F920F920FB60F921124C6
:101240000BB60F922F933F934F935F936F937F93C0
:101250008F939F93AF93BF93EF93FF93E0913502EA
:10126000F09136021995FF91EF91BF91AF919F9147
:101270008F917F916F915F914F913F912F910F903F
:101280000BBE0F900FBE0F901F9018951F920F92DC
:101290000FB60F9211240BB60F922F933F934F93DB
:1012A0005F936F937F938F939F93AF93BF93EF93CE
:1012B000FF93E0913302F09134021995FF91EF9181
:1012C000BF91AF919F918F917F916F915F914F915E
:1012D0003F912F910F900BBE0F900FBE0F901F905C
:1012E00018951F920F920FB60F9211240BB60F9202
:1012F0002F933F934F935F936F937F938F939F931E
:10130000AF93BF93EF93FF93E0913D02F0913E02C4
:101310001995FF91EF91BF91AF919F918F917F911F
:101320006F915F914F913F912F910F900BBE0F9056
:101330000FBE0F901F9018951F920F920FB60F922D
:1013400011240BB60F922F933F934F935F936F939C
:101350007F938F939F93AF93BF93EF93FF93E0910E
:101360003B02F0913C021995FF91EF91BF91AF9133
:101370009F918F917F916F915F914F913F912F91AD
:101380000F900BBE0F900FBE0F901F9018951F92DD
:101390000F920FB60F9211240BB60F922F933F931B
:1013A0004F935F936F937F938F939F93AF93BF936D
:1013B000EF93FF93E0913902F0913A021995FF9172
:1013C000EF91BF91AF919F918F917F916F915F91BD
:1013D0004F913F912F910F900BBE0F900FBE0F902A
:1013E0001F9018951F920F920FB60F9211240BB6F3
:1013F0000F922F933F934F935F936F937F938F93AE
:101400009F93AF93BF93EF93FF93E0913702F091D7
:1014100038021995FF91EF91BF91AF919F918F91F4
:101420007F916F915F914F913F912F910F900BBEE4
:101430000F900FBE0F901F901895CF93DF93282F1A
:1014400030E0F901E559F34E8491F901E157F24E8C
:10145000D491F901E75BF24EC491CC2389F081115C
:101460002FDBEC2FF0E0EE0FFF1FE65AF54EA591B3
:10147000B491EC91ED2381E090E021F480E002C092
:1014800080E090E0DF91CF9108951F93CF93DF9399
:10149000282F30E0F901E559F34E8491F901E15725
:1014A000F24ED491F901E75BF24EC491CC23C1F026
:1014B000162F811105DBEC2FF0E0EE0FFF1FEB5E26
:1014C000F24EA591B4918FB7F894111105C09C917B
:1014D000ED2FE095E92302C0EC91ED2BEC938FBF4B
:1014E000DF91CF911F9108951F93CF93DF93182F12
:1014F000EB01C4D6209711F460E004C0CF3FD105C2
:1015000031F461E0812FDF91CF911F91BECFE12FA8
:10151000F0E0E559F34EE4914E2F50E0FA01319797
:10152000E231F10508F09DC08827EC57FF4F8F4F3F
:101530000C9462A084B5806884BDC7BD97C084B593
:10154000806284BDC8BD92C0809180008068809315
:101550008000D0938900C093880088C0809180006B
:10156000806280938000D0938B00C0938A007EC0FD
:1015700080918000886080938000D0938D00C0931C
:101580008C0074C08091B00080688093B000C093DC
:10159000B3006CC08091B00080628093B000C093B3
:1015A000B40064C080919000806880939000D093D4
:1015B0009900C09398005AC08091900080628093F7
:1015C0009000D0939B00C0939A0050C080919000EF
:1015D000886080939000D0939D00C0939C0046C08B
:1015E0008091A00080688093A0008091A0008F7BF4
:1015F0008093A000D093A900C093A80037C0809129
:10160000A00080628093A000D093AB00C093AA009A
:101610002DC08091A00088608093A000D093AD0081
:10162000C093AC0023C0809120018068809320018A
:10163000D0932901C093280119C0809120018062B4
:1016400080932001D0932B01C0932A010FC0809179
:101650002001886080932001D0932D01C0932C013C
:1016600005C0C038D1050CF04CCF46CFDF91CF91EB
:101670001F9108958F929F92AF92BF92CF92DF9267
:10168000EF92FF926B017C0171DA4B015C01C11496
:10169000D104E104F104E9F069DADC01CB01881935
:1016A0009909AA09BB09883E9340A105B10578F3C1
:1016B00021E0C21AD108E108F10888EE880E83E023
:1016C000981EA11CB11CC114D104E104F10421F73E
:1016D000DECFFF90EF90DF90CF90BF90AF909F90C4
:1016E0008F9008952FB7F8946091A3097091A40981
:1016F0008091A5099091A6092FBF0895F3DF60930B
:101700002A0A70932B0A80932C0A90932D0A08952D
:101710001F920F920FB60F9211242F933F938F9326
:101720009F93AF93BF938091A3099091A409A09137
:10173000A509B091A6093091A20923E0230F2D3706
:1017400020F40196A11DB11D05C026E8230F0296C5
:10175000A11DB11D2093A2098093A3099093A40910
:10176000A093A509B093A6098091A7099091A80913
:10177000A091A909B091AA090196A11DB11D80935C
:10178000A7099093A809A093A909B093AA09BF91AA
:10179000AF919F918F913F912F910F900FBE0F901E
:1017A0001F90189591E0909347033FB7F8942091CC
:1017B000F20A9091F30A3FBF291304C09091C00030
:1017C00095FD3EC09091F20A9F5F9F712091F30AB0
:1017D000921325C00FB607FCF9CF2091C00025FF5A
:1017E000F5CF2091F30AE22FF0E0EE52F54F308171
:1017F0002F5F2F712093F30A3093C6002091C00011
:1018000020642093C0003091F20A2091F30A321331
:10181000DDCF2091C1002F7D2093C100D7CFE09173
:10182000F20AF0E0EE52F54F80832FB7F8949093D0
:10183000F20A8091C10080628093C1002FBF089599
:101840009FB7F8948093C6008091C0008064809315
:10185000C0009FBF08958F929F92AF92BF92EF9268
:10186000FF921F93CF93DF93CDB7DEB7A0970FB64C
:10187000F894DEBF0FBECDBF6115710581059105DE
:1018800079F110E0842E912CA12CB12CEE24E3945C
:10189000F12CEC0EFD1EE10EF11C17FDFA94A501D2
:1018A00094010E941B9DF7016083B901CA011F5F6B
:1018B000611571058105910549F7115010F1E1E0BD
:1018C000F0E0EC0FFD1FE10FF11D17FDFA9580818F
:1018D0008A3010F097E301C090E3890F63DFEDCF0A
:1018E00080E3A0960FB6F894DEBF0FBECDBFDF91A8
:1018F000CF911F91FF90EF90BF90AF909F908F90EE
:1019000051CFA0960FB6F894DEBF0FBECDBFDF91CA
:10191000CF911F91FF90EF90BF90AF909F908F90CD
:1019200008958FB7F8949091D10A2091D00A291781
:1019300059F0E92FF0E0E05BF54F208130E09F5F48
:101940009F779093D10A02C02FEF3FEF8FBFC9015D
:1019500008951F920F920FB60F9211240BB60F929B
:101960008F939F93EF93FF938091F30AE82FF0E01A
:10197000EE52F54F90818F5F8F718093F30A9093B1
:10198000C6008091C00080648093C0009091F20AEC
:101990008091F30A981305C08091C1008F7D8093D8
:1019A000C100FF91EF919F918F910F900BBE0F900F
:1019B0000FBE0F901F9018958CE0E4EFFAE0A5E1C0
:1019C000BBE001900D928A95E1F708954F925F92E6
:1019D0006F927F928F929F92AF92BF92DF92EF921F
:1019E000FF920F931F93CF93DF93D82EE82E880F8B
:1019F000FF08F701E15AF34E6491E701CC0FDD1FB8
:101A0000CC0FDD1FFE01ED5AF34E459055906590C9
:101A10007490062E000C770B880B990B0E94469948
:101A20004B015C0120E030E040EC5FE3C301B20118
:101A30000E94A599A50194010E94A599AB01BC0142
:101A400000E010E098018D2D0E944D4CFE01E95BF5
:101A5000F34E2591359145915491C501B4010E94F1
:101A6000A5994B015C0120E030E0A9010E9440995A
:101A7000882309F449C000E010E09801B501A401F1
:101A800070588D2D0E944D4CF701EC5BF34E649124
:101A9000611119C0E5ECFCE184913F019FEF691AE7
:101AA000790A882319F07EDEF301F6CFE2E2FCE149
:101AB00084913F019FEF691A790A882319F072DE39
:101AC000F301F6CF6AE0FE01EE5EF34E45905590CD
:101AD0006590749070E080E090E00E9446999B01D0
:101AE000AC01C301B2010E944F9E2B013C01A50134
:101AF0009401C501B4010E94739DAB01BC01930127
:101B000082018D2D0E944D4CF701EB5CF44F81E07A
:101B10008083F701E25BFC4F8083FE01EE5CF54FB2
:101B200010821182128213828D2D0E942E5DFE0181
:101B3000EA5FF34E65917591859194918E010B5EEC
:101B4000144FFE01E457FC4F2081318142815381C3
:101B50000E94739DF801608371838283938320DAEE
:101B6000C25CD54FF80180819181A281B3818883C5
:101B70009983AA83BB83DF91CF911F910F91FF902F
:101B8000EF90DF90BF90AF909F908F907F906F907D
:101B90005F904F900895179AEEE4F3E01082169A42
:101BA0001182159A1282149A0895EBECF9E084914F
:101BB000EF012196882319F0F5DDFE01F8CFE6EE5E
:101BC000FBE18491EF012196882319F0EBDDFE0102
:101BD000F8CF0E946662DFDF2FEF8BE49DE121509A
:101BE00080409040E1F700C00000F8942FEF84E3BC
:101BF0009CE0215080409040E1F700C000000E942E
:101C00006662A895FECFCF92DF92EF92FF920F937C
